:100000000C946B090C948A090C948A090C941C0AB0
:100010000C94520A0C948A090C948A090C948A094B
:100020000C948A090C948A090C948A090C948A0904
:100030000C948A090C948A090C948A090C947D0DFD
:100040000C948A090C948A090C948A090C948A09E4
:100050000C940B6E0C94BE650C948A090C948A095E
:100060000C948A090C9493660C948A090C94876604
:100070000C948A090C948A090C948A090C948A09B4
:100080000C943E790C948A090C948A090C948A0980
:100090000C94D1660C948A090C94C5660C948A0958
:1000A0000C948A090C948A090C948A090C948A0984
:1000B0000C948A090C948A090C948A090C948A0974
:1000C0000C948A090C948A090C948A090C948A0964
:1000D0000C948A090C948A090C948A090C948A0954
:1000E0000C948A090C94C46D0C94CE6D0C94BA6D6A
:1000F0000C947A6D0C94FF6D0C94F06D0C94E46D7F
:100100000C94D86D0C948A090C948A090C948A0971
:100110000C948A090C948A090C948A090C948A0913
:100120007582948213830284228442844A84F783F2
:10013000084AD73B3BCE016E84BCBFFDC12F3D6C4E
:1001400074319ABD56833DDA3D00C77F11BED9E4B4
:10015000BB4C3E916BAAAABE000000803F076342E1
:1001600036B79BD8A71A39685618AEBAAB558C1D4E
:100170003CB7CC5763BD6DEDFD753EF6177231BFD0
:10018000000000803F08000000BE922449123EABF0
:10019000AAAA2ABECDCCCC4C3E00000080BEABAAA1
:1001A000AAAA3E00000000BF000000803F0000003F
:1001B0000000084178D3BB4387D1133D190E3CC3DF
:1001C000BD4282AD2B3E68EC8276BED98FE1A93E5E
:1001D0004C80EFFFBE01C4FF7F3F00000000000025
:1001E00025730A005854414C5F5452494D3D2564D3
:1001F0000025730A0025730A0054657374203620A5
:1002000025730A005465737420352025730A005441
:1002100065737420342025730A0054657374203389
:100220002025730A005465737420322025730A0058
:100230005465737420312025730A006368616E3D34
:1002400025640A0074787077723D25640A003530A1
:10025000306B0A003235306B0A003131356B0A00E1
:1002600035366B0A0033386B0A0025730A00765F57
:100270006C6F773D252D332E32660A0025730A00F8
:1002800073656E743D252D75206475703D252D7543
:100290002069676E6F7265643D252D752074746CDE
:1002A0005F7A65726F3D252D750A0025372E3366FE
:1002B0002025372E33660025352E32662000457204
:1002C000726F72203020566F6C74004E6F74207302
:1002D0007570706F727465640A004572726F722077
:1002E0003020566F6C74004572726F722030205649
:1002F0006F6C74007062323D25730A00256C7500C6
:10030000416C6C6F77656420737065656420312F74
:1003100031302F3130302F343030206B6269742F00
:10032000730025630074746C3D252D642000747483
:100330006C3D252D6420004E65772074746C3D253E
:100340002D6420002563004D533536313120503D5A
:10035000252D372E326620252D372E32666D0A0068
:10036000424D5030383520256C64205061202025C6
:100370002D372E32666D00256300545F4845415489
:100380005F4944583D252D352E32662000545F4488
:1003900045573D252D352E3266200041483D252DFF
:1003A000352E32662000545F53485432583D252D77
:1003B000352E3266200052485F53485432583D254E
:1003C0002D352E32662000545F52483D252D342EA7
:1003D0003166200052483D252D342E3166200025FF
:1003E00063002563002563002563002563007265B3
:1003F000706F72745F616C6C3D007265706F7274C7
:100400003D00256300256300256300256300204F20
:10041000534343414C3D2564200020467573653AA3
:100420002065653D253032782068663D253032787C
:10043000206C663D25303278206C623D2530327864
:10044000004D43553D2530366C78002563007478A7
:100450005F6C656E3D252D6C752C765F6C6F773DFE
:10046000252D6C752C73687432783D252D6C750ABA
:10047000002563004F4B0A002563002563002563B8
:1004800000256300256300256300256300256300C4
:1004900064656275675F616C6C3D00646562756779
:1004A0003D0064656275673D0025730A00646565FB
:1004B000700A006E6F6E650A00707772733D00708F
:1004C00062323D25730A007062313D25730A00696E
:1004D0006E74725F7365635F70313D252D372E3307
:1004E000660A00696E74725F70313D252D6C640A76
:1004F00000696E74725F7365635F70303D252D37E0
:100500002E33660A00696E74725F70303D252D6C63
:10051000640A00765F6D63753D252D352E32660ABF
:1005200000745F6D63753D252D352E32660A0070AF
:100530007077723D25730A0064656275673D0072CD
:10054000636D643D25730A0025730A006175746F3D
:100550000A006C6F675F6D6F64653D007573625F65
:100560007077723D25730A0072656C61793D257361
:100570000A0074746C3D252D640A0052494D455F94
:10058000616464723D252D642E252D640A006E651C
:10059000696768626F725F7461626C655F73697AC4
:1005A000653D25640A00765F6C6F773D252D332EFF
:1005B00032660A00747870773D25640A00636861CA
:1005C0006E3D25640A0069643D006932635F6275AF
:1005D000733D006932635F73706565643D252D6C02
:1005E000750A007478743D25730A00537973746535
:1005F0006D2053756D6D6172790A002530366C7807
:100600000041744D656761323536524652320041C1
:10061000744D656761313238524652320041744D33
:100620006567613634524652320041744D656761E8
:1006300031323852464131004D43553D006D6173B2
:100640006B3D002C00696E74657276616C3D252DE2
:10065000750023252D642C00745F686561745F69E3
:10066000647800745F64657700616800705F6D7323
:10067000353631310072685F736874327800745FA8
:1006800073687432780070610070006164340061D6
:1006900064330061643200616431006133006132AF
:1006A00000613100765F696E0072680065727200E9
:1006B000757074696D650070315F6C7374007031B2
:1006C0005F740070310070305F6C73740070305F65
:1006D0007400703000765F6D637500745F6D6375D4
:1006E00000743100740069640065363400747874F5
:1006F000002D002B006175746F006E6F6E650070C9
:100700006F7765725F736176655F6C65647279009F
:1007100072656C61795F6C65647900636F6D70619F
:10072000737300616363656C007072657300705F62
:10073000707772006165730070315F6C6564790079
:1007400070305F6C656472006576656E74006C6510
:1007500064006F7700706B740074785F6C65647907
:100760000072785F6C656472006F706572006E6F06
:100770006E65002530327800765F6164343D252D4A
:10078000382E3666002000765F6164333D252D38B3
:100790002E3666002000765F6164323D252D382EAE
:1007A0003666002000765F6164313D252D382E3697
:1007B00066002000765F6C696768743D252D382ED1
:1007C0003666002000765F61323D252D372E336678
:1007D000002000765F61313D252D372E33660020E5
:1007E00000765F696E3D252D352E326600204E6500
:1007F0007665722D7573656420737461636B203E3A
:100800002025642062797465730A00757074696DBF
:10081000653D252D642D646179732D253032643A50
:10082000253032643A253032642D686F7572730A50
:100830000074657374205B6F66667C317C327C3338
:100840007C347C355D20202020202020202D207429
:10085000657374206D6F6465730A0D007478205B96
:10086000706B74207061796C6F61645D2020202052
:1008700020202020202020202D2073656E642072EF
:100880006164696F20706B74206B6579626F61724F
:10089000640A0D00776474205B6F6E7C6F66667C03
:1008A000746573745D2020202020202020202020CB
:1008B0002D207761746368646F670A0D00765F6C42
:1008C0006F77205B765F6C6F775D20202020202083
:1008D0002020202020202020202D206C6F77657381
:1008E00074207265706F727420766F6C74616765C6
:1008F0000A0D007570677220202020202020202003
:100900002020202020202020202020202020202DDA
:10091000207265626F6F742076696120626F6F74F8
:100920006C6F616465720A0D0075617274205B33CF
:10093000386B7C35366B7C3131356B7C3235306BC6
:100940007C3530306B5D202D2073657420746572AA
:100950006D2F756172742073706565640A0D006295
:100960006F6F742020202020202020202020202095
:1009700020202020202020202020202D2072656291
:100980006F6F740A0D0070777273205B6465657019
:100990007C6E6F6E655D202020202020202020208E
:1009A00020202D206D637520736C656570206D6F40
:1009B00064650A0D007265737420656570726F6DF1
:1009C0002020202020202020202020202020202027
:1009D000202D20726573746F726520656570726F6B
:1009E0006D0A0D0070707772205B6F6E7C6F6666AB
:1009F0005D202020202020202020202020202020BA
:100A00002D2070726F6772616D6D61626C65207010
:100A100077720A0D0070623220205B6F6E7C6F6609
:100A2000665D202020202020202020202020202043
:100A3000202D2070726F6772616D6D61626C652030
:100A400070696E2062320A0D00747874205B7374D2
:100A500072696E675D202020202020202020202029
:100A600020202020202D20536574207265706F7225
:100A700074207465787420737472696E670A0D004F
:100A800074787077205B31352D305D202020202058
:100A90002020202020202020202020202D205458DD
:100AA000205077722E204869676865737420302063
:100AB000283364426D290A0D0074746C205B302D5C
:100AC00031355D20202020202020202020202020C3
:100AD00020202020202D2074696D652D746F2D6CD1
:100AE00069766520666F72207061636B6574730A46
:100AF0000D00737320202020202020202020202083
:100B000020202020202020202020202020202D20D8
:100B100073797374656D2073756D6D6172790A0DEB
:100B20000072732020202020202020202020202040
:100B3000202020202020202020202020202D207256
:100B40006164696F2073746174730A0D00726920A7
:100B50005B236E5D205B696E745D20202020202069
:100B60002020202020202020202D207265706F72F0
:100B70007420696E74657276616C0A0D0072636D23
:100B800064205B6F6E7C6F66665D202020202020D5
:100B90002020202020202020202D20616C6C6F77C9
:100BA00020636D642066726F6D206E65746F726B6A
:100BB0000A0D007265205B236E5D205B2B7C2D5D32
:100BC000205B6D61736B7C6175746F2C6D61736BF1
:100BD0005D202D206D6F7465207265706F727420BA
:100BE0007365742F6D6F646966790A0D006F7720E5
:100BF00020202020202020202020202020202020F5
:100C00002020202020202020202D206F6E652D7791
:100C10006972652073656E736F72730A0D006C6F75
:100C200067205B6175746F7C6F6E7C6F66665D209C
:100C3000202020202020202020202D206D6F746572
:100C4000732064617461206F6E205553420A0D0059
:100C50006E65205B666C7573685D20202020202007
:100C60002020202020202020202020202D206E65E4
:100C7000696768626F72207461626C650A0D006555
:100C800072722020202020202020202020202020C0
:100C900020202020202020202020202D206572725E
:100CA0006F722073746174730A0D006D6375202078
:100CB0002020202020202020202020202020202034
:100CC000202020202020202D206D637520696E6655
:100CD0006F0A0D00693263205B70726F62657C730E
:100CE0007065656420236E5D202020202020202058
:100CF0002D206932632070726F6265206275737C8B
:100D0000736574206275732073706565640A0D00E5
:100D10006964205B72657365745D2020202020204B
:100D20002020202020202020202020202D20696429
:100D30002068616E646C696E670A0D0068756D20CD
:100D400020202020202020202020202020202020A3
:100D500020202020202020202D2068756D696469C6
:100D600074792073656E736F720A0D0072656C6121
:100D700079205B6F6E7C6F66667C73746174735DE3
:100D800020202020202020202D2072656C617920D9
:100D90006E6574776F726B207265706F7274730A10
:100DA0000D006465205B6D61736B5D202020202049
:100DB00020202020202020202020202020202D2026
:100DC00064656275670A0D006368616E205B31318E
:100DD0002D32365D202020202020202020202020A1
:100DE000202020202D206368616E2031312D323685
:100DF0002028322E3430352D32343830204D687A68
:100E0000290A0D0063616C69205B5B765F696E7C0B
:100E100061317C61325D20766F6C747C72657365C4
:100E2000747C6E6F6E655D202D2063616C696272EB
:100E30006174650A0D006164632020202020202059
:100E400020202020202020202020202020202020A2
:100E500020202D2073686F7720765F696E2C2061CB
:100E6000312C20613220766F6C74616765730A0DD6
:100E7000007520202020202020202020202020203D
:100E8000202020202020202020202020202D207500
:100E90007074696D650A0D007620202020202020C6
:100EA0002020202020202020202020202020202042
:100EB000202020202D2076657273696F6E0A0D0048
:100EC00068202020202020202020202020202020DA
:100ED0002020202020202020202020202D20686578
:100EE0006C700A0D00256300756E6B6E6F776E2057
:100EF000636D640A00484D4335383833002573006C
:100F0000257300202573002025362E32662000250B
:100F10003032780074656D705F65787465726E3D0F
:100F2000252D362E326600202573002025362E32E0
:100F300066204F6E2D426F6172640025303278005A
:100F400074656D705F626F6172643D252D362E325F
:100F500066000A00503A20256C642050612020254C
:100F60002D372E3266206D0A002563002563004967
:100F700032433A2000452025642E256420636C6F9F
:100F8000636B20256C752063707520256C75206C53
:100F9000706D20256C752069727120256C75206735
:100FA0006C656420256C7520796C656420256C75F2
:100FB00020726C656420256C7520747820256C7512
:100FC000206C697374656E20256C752073656E7373
:100FD0006F727320256C752073657269616C2025B2
:100FE0006C750A00532025642E256420636C6F63A2
:100FF0006B20256C7520747820256C752072782004
:10100000256C752072747820256C7520727278209A
:10101000256C75207265786D697420256C7520616A
:10102000636B747820256C75206E6F61636B7478C8
:1010300020256C752061636B727820256C75207497
:10104000696D65646F757420256C752062616461DB
:10105000636B727820256C7520746F6F6C6F6E6790
:1010600020256C7520746F6F73686F727420256C07
:10107000752062616473796E636820256C752062E7
:10108000616463726320256C7520636F6E74656E96
:1010900074696F6E64726F7020256C752073656E55
:1010A00064696E6764726F7020256C75206C6C7457
:1010B0007820256C75206C6C727820256C750A0080
:1010C000257325730A004F6E6C696E650A000A006D
:1010D0002C20636865636B20726174652025752020
:1010E000487A0025732025732C206368616E6E6535
:1010F0006C20257520706F776572202575000A00B9
:1011000025783A004D414320616464726573732011
:101110000052616E646F6D2045554936342061641C
:1011200064726573732067656E6572617465640AC5
:10113000000A2A2A2A2A2A2A2A426F6F74696E67AD
:101140002025732A2A2A2A2A2A2A0A00454550528B
:101150004F4D20697320636F72727570742C20720A
:101160006577726974696E67207769746820646551
:101170006661756C74732E0A006C6F63616C686FC6
:1011800073740041544D45474131323872666131C4
:1011900000020000FFFE0000016E616E00696E66D5
:1011A0000000407A10F35A00A0724E18090010A5F2
:1011B000D4E80000E87648170000E40B5402000071
:1011C000CA9A3B000000E1F50500008096980000F7
:1011D0000040420F000000A0860100000010270020
:1011E000000000E803000000006400000000000AA6
:1011F00000000000000100000000002C76D888DC10
:10120000674F0823DFC1DFAE59E1B1B796E5E3E4EC
:1012100053C63AE651997696E8E6C28426EB898C65
:101220009B62ED407C6FFCEFBC9C9F40F2BAA56FC7
:10123000A5F490055A2AF75C936B6CF9676DC11B96
:10124000FCE0E40D47FEF520E6B500D0ED902E035E
:1012500000943577050080841E080000204E0A00A7
:101260000000C80C333333330F986E12831141EFF3
:101270008D2114893BE65516CFFEE6DB18D1844B51
:10128000381BF77C1D901DA4BBE424203284725EC1
:10129000228100C9F124ECA1E53D274E414E494E83
:1012A000495459494E46CDCCCC3D0AD7233C17B7BB
:1012B000D13877CC2B329595E6241FB14F0A000028
:1012C00020410000C84200401C4620BCBE4CCA1B46
:1012D0000E5AAEC59D7411241FBECFEFD1E4DEBF00
:1012E000CDBF19E0A0E0B2E0E2E6FEE201E00BBF14
:1012F00002C007900D92AE3BB107D9F721E3AEEBE8
:10130000B9E001C01D92A33DB207E1F70E94198523
:101310000C942F970C9400008115910511F0019702
:10132000F1F7089589EB94E09F938F930E941494B2
:101330008091580290915902A0915A02B0915B029B
:101340000F900F9093FF03C083EB94E002C08DEAEF
:1013500094E09F938F930E9414940F900F900895A0
:10136000E091771BEF73F0E0E853F44E80838091B7
:10137000771B8F5F8093771B80910D298860809306
:101380000D294EE352E061E1CA010E949E5580E0C2
:1013900090E00895CF93DF93EC018091C50990917F
:1013A000C60986FF1DC08E811F928F938D811F926B
:1013B0008F938C811F928F938B811F928F938A8141
:1013C0001F928F9385E693E09F938F930E940294E0
:1013D0008DB79EB70C960FB6F8949EBF0FBE8DBF0B
:1013E000BE018CEF99E00E94D056BE0184E092E0ED
:1013F000DF91CF910C9445568823B9F052985A98B2
:101400001DBA80916900806280936900EA9A5398BE
:101410005B98EB9A80916900806880936900809165
:1014200068008160809368000895109269005A9A5C
:10143000EA985B9AEB9808951F920F920FB60F925D
:1014400011248F939F93AF93BF938091680080FF87
:1014500020C08091E8289091E928A091EA28B091D5
:10146000EB280196A11DB11D8093E8289093E928EF
:10147000A093EA28B093EB288091C5099091C60902
:1014800087FF07C0749882E090E090938502809374
:101490008402BF91AF919F918F910F900FBE0F90DB
:1014A0001F9018951F920F920FB60F9211248F93D1
:1014B0009F93AF93BF938091680080FF20C080917D
:1014C000EC289091ED28A091EE28B091EF2801969C
:1014D000A11DB11D8093EC289093ED28A093EE28D8
:1014E000B093EF288091C5099091C60990FF07C07D
:1014F000739882E090E09093850280938402BF917C
:10150000AF919F918F910F900FBE0F901F901895E4
:1015100080937C0080917B00877F80937B0080910B
:101520007C00806C80937C0085E080937A008091C1
:101530007A00806880937A0080917B0087FFFCCFDF
:1015400080917B0085FFFCCF80917A00806480933E
:101550007A0080917A0086FDFCCF1092790010927B
:10156000780084E090E060E070E020917A002064F0
:1015700020937A0020917A0026FDFCCF20917800FC
:1015800030917900620F731F0197009771F71092E5
:101590007C0080917A008F7780937A0076956795AA
:1015A0007695679580E090E00E946F8A089580E0CC
:1015B0000E94880A20917C0230917D0240917E0237
:1015C00050917F020E94538C21EE3AE744E95EE39A
:1015D0000E94088908950F931F93CF93DF93CFE163
:1015E000D0E00BE51EE0C093510187EC90E00E9433
:1015F0008C098091510185FD0DC0C031D10521F0CC
:101600002CF00B54110904C004EC19E00253110929
:101610002197E9CFB80180E090E00E946F8A20E036
:1016200030E04AE754E40E94D289DF91CF911F91C4
:101630000F910895CF93DF93EC01888199810097F2
:1016400099F0883B904121F01982188283E011C003
:10165000623171F40E94EB0A60933F24709340243E
:10166000809341249093422488EB90E1998388836E
:1016700081E0DF91CF91089580917B008860809315
:101680007B0089EC80937C0085E080937A008091D8
:101690007A00806880937A0080917B0087FFFCCF7E
:1016A00080917B0085FFFCCF80917A0080648093DD
:1016B0007A0080917A0086FDFCCF80917A00806468
:1016C00080937A0080917A0086FDFCCF609178004B
:1016D0007091790080917A008F7780937A0080E012
:1016E00090E00E946F8A27ED33EA40E95FE30E94B1
:1016F000538C26E636E648E853E40E9407890895AD
:10170000BF92CF92DF92EF92FF920F931F93CF93EE
:10171000DF93CDB7DEB729970FB6F894DEBF0FBEC3
:10172000CDBF6C011092BE098FEF898708E81BE1DD
:10173000B12C7E0189E0E80EF11C89858823E9F14E
:10174000E8E0BE16E1F1BE016F5F7F4FC7010E9466
:10175000395F89858F3F11F08E3F19F48093BE0960
:101760002CC0CE010196C114D10471F40E94525FC5
:1017700080930A29FE013196A2E0B9E281918D930E
:10178000EE15FF05D9F71DC00E94525FF801808356
:10179000FE01319620E030E0A801485051098191C6
:1017A000DA01A20FB31F8C932F5F3F4F2830310512
:1017B000B1F7B394075F1F4FC0CF8B2D03C088E0F4
:1017C00001C081E029960FB6F894DEBF0FBECDBFF1
:1017D000DF91CF911F910F91FF90EF90DF90CF900D
:1017E000BF90089582E59FE09F938F930E94149489
:1017F0000F900F9008952F923F924F925F926F92A9
:101800007F928F929F92AF92BF92CF92DF92EF9290
:10181000FF920F931F93CF93DF93EC014B0100973F
:1018200011F427E004C08130910549F426E04AE232
:1018300050E06BE270E089E290E00E94195ECE0118
:101840000E94800B9E012154364F5901D9018C937F
:10185000CD2B69F098E8C92E9BE1D92EC0E8DBE1D9
:10186000E12CF12C23E0222E2FE0322EA6C082E0C4
:1018700099E20E948760BC01882777FD8095982FA8
:101880000E94718A6B017C01892869F020E030E0B8
:1018900048EC52E40E94D2899F938F937F936F9379
:1018A00080E49FE0ACC0C2E0D9E20BE31FE0899185
:1018B0001F928F931F930F930E9414940F900F9079
:1018C0000F900F90B9E2CA30DB0789F720E030E0D3
:1018D00048EC52E4C701B6010E94D2899F938F93CE
:1018E0007F936F938BE29FE09F938F930E9414945A
:1018F0000F900F900F900F900F900F9080910A29EA
:10190000882319F084E993E002C088E094E09F9373
:101910008F9387E29FE09F938F930E9414940F9080
:101920000F900F900F9075C000E010E0FE01E00FE7
:10193000F11F80811F928F93AFE0BFE0BF93AF9301
:101940000E9414940F5F1F4F0F900F900F900F90F5
:101950000830110559F720E030E048EC52E4C301AB
:10196000B2010E94D2899F938F937F936F93A7E0D8
:10197000BFE0BF93AF930E9414940F900F900F900D
:101980000F900F900F90D6018C91882309F455C0C9
:1019900084E993E09F938F933F922F920E94149437
:1019A0000E94F20BBFEFEB1AFB0AE9E0CE0ED11C4E
:1019B00029960F900F900F900F90D5018C9190E089
:1019C000E816F906ECF5CE010E948760BC01882775
:1019D00077FD8095982F0E94718A2B013C0181141C
:1019E000910409F4A1CF20E030E048EC52E40E94D9
:1019F000D2899F938F937F936F9384E19FE09F930E
:101A00008F930E9414940F900F900F900F900F904F
:101A10000F90DF91CF911F910F91FF90EF90DF908A
:101A2000CF90BF90AF909F908F907F906F905F907E
:101A30004F903F902F900C94F20B88E094E0AACF47
:101A4000DF91CF911F910F91FF90EF90DF90CF909A
:101A5000BF90AF909F908F907F906F905F904F90CE
:101A60003F902F900895CF93DF9300D0CDB7DEB78E
:101A7000809103298983809109298A83CE01019667
:101A80000E9492530F900F90DF91CF910895CF93C2
:101A9000DF93EC0120910229309103294091042920
:101AA0005091052960910629709107298091082994
:101AB00090910929AFEF0E94838FE1F427E04AE279
:101AC00050E06BE270E089E290E00E94195E80E0F5
:101AD00090E00E94800BC154D64F888349E050E0CB
:101AE0006AE070E082E099E20E948695DF91CF91F2
:101AF0000C94330DDF91CF9108951F920F920FB682
:101B00000F9211240BB60F92DF92EF92FF920F9378
:101B10001F932F933F934F935F936F937F938F9375
:101B20009F93AF93BF93CF93DF93EF93FF938091F6
:101B30000D29826080930D298091580286FD2B9A91
:101B40008091580287FD2B9A8091840290918502A2
:101B50001816190614F4749A739A8091C509909115
:101B6000C60985FF02C07498739880910202909113
:101B7000030201979093030280930202892B09F0DC
:101B80003DC18091D3099091D40901969093D409D5
:101B90008093D3098091432490914424A0914524BB
:101BA000B09146240196A11DB11D809343249093CA
:101BB0004424A0934524B093462480E190E0909380
:101BC0000302809302028091580280FD02C01D9B97
:101BD00007C01092C3091092C20983B7817F09C060
:101BE00081E090E09093C3098093C20983B7817F1D
:101BF000866083BF8091C5099091C60997FF08C090
:101C00008091C2099091C309892B61F0749A7398ED
:101C100007E21BE1C4E5D4E234E0E32EF12CDD243D
:101C2000D3941FC0739A7498F3CF8091D309909185
:101C3000D40901960E94238D892BD1F0F80160858B
:101C400071856115710509F5F8016085718561156A
:101C5000710569F5065F1F4F2596FBE10F341F07DD
:101C6000D1F1F801608571856115710539F3DDCF1A
:101C700077988091C5099091C60992FFDFCF74983B
:101C8000F0928502E0928402D9CF8091D30990919D
:101C9000D40901960E94238D892BB1F61C821B82E8
:101CA000AE0162E186E192E00E949E55CDCF809127
:101CB000D3099091D4090E94238D892B59F6D8829B
:101CC0001A8309831C821B82AE0162E184E392E0E5
:101CD0000E949E55BFCF60915E0270915F026115B8
:101CE0007105A1F18091D3099091D4090E94238DAF
:101CF000892B61F58091E8289091E928A091EA2844
:101D0000B091EB284091351C5091361C6091371CE6
:101D10007091381C841B950BA60BB70B80934F1B3F
:101D20009093501BA093511BB093521B8091E828B5
:101D30009091E928A091EA28B091EB288093351C76
:101D40009093361CA093371CB093381C60915C02B2
:101D500070915D0261157105A1F18091D309909197
:101D6000D4090E94238D892B61F58091EC289091F4
:101D7000ED28A091EE28B091EF284091391C5091A8
:101D80003A1C60913B1C70913C1C841B950BA60B6C
:101D9000B70B8093531B9093541BA093551BB09388
:101DA000561B8091EC289091ED28A091EE28B091DF
:101DB000EF288093391C90933A1CA0933B1CB0935E
:101DC0003C1C8091580286FD2B988091580290917E
:101DD0005902A0915A02B0915B0291FF0FC00E947C
:101DE000386A8A3119F0C1E0C80F01C0CBE00E9407
:101DF000F4688C2F0E94506A0E943C6940E050E0D9
:101E000060E086E892E00E949E55FF91EF91DF919D
:101E1000CF91BF91AF919F918F917F916F915F9182
:101E20004F913F912F911F910F91FF90EF90DF9075
:101E30000F900BBE0F900FBE0F901F9018958091C2
:101E4000771B90915324891B08950E941F0F8823AC
:101E500071F0E0915324EF73F0E0E853F44E808189
:101E600090E0209153242F5F2093532408958FEF07
:101E70009FEF0895CF93DF93EC011092F009109239
:101E8000EF09888199810097C1F08838934021F04B
:101E90001982188283E0B8C0613109F0B4C0F894A7
:101EA00078940E94250F99279093EB098093EA0973
:101EB0008D3009F443C08F3F49F40E941F0F8111F8
:101EC000EECF88E893E0998388839DC082319105A5
:101ED00009F45AC08F37910509F052C08091E80982
:101EE0009091E909181619060CF56091CD317091A1
:101EF000CE3188E090E00E94D0936091CD31709116
:101F0000CE3180E290E00E94D0936091CD3170910B
:101F1000CE3188E090E00E94D0938091E8099091C2
:101F2000E90901979093E9098093E8098091E8090C
:101F30009091E9098F37910509F0BFCF1092532492
:101F40001092771B8091E8099091E909FC01E8590A
:101F5000FB4D10829093F0098093EF091092E909EC
:101F60001092E80980910B2990910C29009709F4AF
:101F7000A4CF40E050E06091FE110E949E559DCF9D
:101F80008830910571F5AACF6091CD317091CE3135
:101F90008DE090E00E94D0931092E7091092E6093C
:101FA0008091E6099091E7092091E8093091E909CB
:101FB000821793070CF0BACFFC01E859FB4D8081E2
:101FC0006091CD317091CE3190E00E94D09380919C
:101FD000E6099091E70901969093E7098093E60955
:101FE000DFCF6091CD317091CE310E94D09380913E
:101FF000E8099091E9092091EA09FC01E859FB4DB3
:10200000208301968FCF81E0DF91CF910895809159
:10201000C2099091C309892BD1F080915802909107
:102020005902A0915A02B0915B0293FD10C00E9428
:10203000F46883B7817F866083BFF89483B781603B
:1020400083BF7894889583B78E7F83BF78940895F3
:10205000CF93DF93EC0188819981009719F08B3E33
:10206000904199F40E94B1670E94071040E050E04F
:1020700065E880910212909103120E949E558BEEAA
:1020800090E19983888381E003C01982188283E0FC
:10209000DF91CF910895CF93DF9300D0CDB7DEB716
:1020A000892B81F05F934F9380E09FE09F938F9304
:1020B00069837A830E9414940F900F900F900F9071
:1020C0007A8169817F936F938DEF9EE09F938F93C9
:1020D0000E9414940F900F900F900F900F900F90FC
:1020E000DF91CF910895FF920F931F93CF93DF93CA
:1020F0000E94B16780EB0E94146181111CC00E9494
:10210000786180913D2090913E20816090933E20A7
:1021100080933D208DE993E09F938F938DEF9EE018
:102120009F938F930E9414940F900F900F900F9095
:10213000C1E0D0E002C0C0E0D0E0FEB08F2D8470DE
:10214000F82E729A0E94B1678EE40E941461811188
:1021500016C00E94786180913D2090913E2082605F
:1021600090933E2080933D208E010F5F1F4F43E2EE
:1021700059E065EA73E0CE010E944B10E801F110CE
:1021800001C072980E94B1678EEE0E9414618111A5
:1021900016C00E94786180913D2090913E2084601D
:1021A00090933E2080933D208E010F5F1F4F43E2AE
:1021B00059E06DEA73E0CE010E944B10E8010E94E5
:1021C000B16786EA0E941461811116C00E9478618D
:1021D00080913D2090913E20886090933E20809396
:1021E0003D208E010F5F1F4F43E259E064EB73E027
:1021F000CE010E944B10E8010E94B1678CE30E945F
:10220000146181111EC00E94786180913D209091DF
:102210003E20806190933E2080933D208E010F5F91
:102220001F4F43E259E06CEB73E0CE010E944B106C
:1022300085EF9EE09F938F930E9414940F900F90D0
:10224000E8010E94B16782ED0E941461811116C0FD
:102250000E94786180913D2090913E208062909311
:102260003E2080933D208E010F5F1F4F43E259E0D7
:1022700064EC73E0CE010E944B10E8010E94B1674C
:1022800080E80E941461811116C00E9478618091DB
:102290003D2090913E20916090933E2080933D2080
:1022A0008E010F5F1F4F43E259E06DEC73E0CE01EA
:1022B0000E944B10E8010E94B16780ED0E941461FA
:1022C000811116C00E94786180913D2090913E203E
:1022D000806890933E2080933D208E010F5F1F4FBA
:1022E00043E259E063ED73E0CE010E944B10E80138
:1022F0000E94B1678CEE0E941461811116C00E9489
:10230000786180913D2090913E20926090933E2094
:1023100080933D208E010F5F1F4F43E259E06BED2C
:1023200073E0CE010E944B10E80107E010E00E942C
:10233000B1678CE70E941461811113C00E9478611B
:1023400080913D2090913E20806490933E20809328
:102350003D2043E259E062EE73E0CE010E944B1053
:1023600005C0015011090115110509F70E94786196
:10237000DF91CF911F910F91FF900C94F20BCF93AF
:10238000DF9300D0CDB7DEB74A8369830E944F61E7
:102390006981862F0E9480614A81842F0E9480611A
:1023A0000F900F90DF91CF910C947861AF92BF9214
:1023B000DF92EF92FF920F931F93CF93DF9300D0A2
:1023C0001F92CDB7DEB7182FD22E4A835B83698365
:1023D0000E944F616981862F0E948061812F8160F8
:1023E0000E9476614A81A42E5B81B52E00E010E048
:1023F000ED2CF12C81E0E81AF1080D1580F40E1592
:102400001F0519F40E949B6102C00E949161F501B1
:1024100080830F5F1F4FFFEFAF1ABF0AEECF0F9001
:102420000F900F90DF91CF911F910F91FF90EF9040
:10243000DF90BF90AF900C947861AF92BF92CF9233
:10244000DF92EF92FF920F931F93CF93DF93CDB75D
:10245000DEB760970FB6F894DEBF0FBECDBFB82EC3
:10246000A42E6623E9F18E010F5F1F4F80E1F80172
:1024700011928A95E9F728E0A80168E980EB0E94AB
:10248000D611BB2041F02BEE33E03F932F930E94F7
:1024900002940F900F906E01F8E0CF0ED11C52EF16
:1024A000E52E53E0F52EF80181918F011F928F9355
:1024B000FF92EF920E9402940F900F900F900F9056
:1024C0000C151D0581F788851F928F9327E434E052
:1024D0003F932F930E9402940F900F900F900F90B4
:1024E000AA20E9F18E010F5F1F4F80E1F8011192E0
:1024F0008A95E9F728E0A80160E880EB0E94D611F0
:10250000BB2041F087EF93E09F938F930E9402944A
:102510000F900F906E01F0E1CF0ED11C42EFE42E30
:1025200043E0F42EF80181918F011F928F93FF9267
:10253000EF920E9402940F900F900F900F900C1545
:102540001D0581F788851F928F9387E494E09F9300
:102550008F930E9402940F900F900F900F906096AF
:102560000FB6F894DEBF0FBECDBFDF91CF911F91A4
:102570000F91FF90EF90DF90CF90BF90AF900895B4
:10258000CF93DF9300D0CDB7DEB71A82198222E055
:10259000AE014F5F5F4F6AEA8EEE0E94D6118981CD
:1025A00090E0982F88272A81822B9093091C809392
:1025B000081C22E0AE014F5F5F4F6CEA8EEE0E9476
:1025C000D611898190E0982F88272A81822B9093B9
:1025D0000B1C80930A1C22E0AE014F5F5F4F6EEA36
:1025E0008EEE0E94D611898190E0982F88272A814B
:1025F000822B90930D1C80930C1C22E0AE014F5F48
:102600005F4F60EB8EEE0E94D611898190E0982F8B
:1026100088272A81822B90931B1C80931A1C22E00E
:10262000AE014F5F5F4F62EB8EEE0E94D611898143
:1026300090E0982F88272A81822B90931D1C8093ED
:102640001C1C22E0AE014F5F5F4F64EB8EEE0E94D8
:10265000D611898190E0982F88272A81822B909328
:102660001F1C80931E1C22E0AE014F5F5F4F66EB84
:102670008EEE0E94D611898190E0982F88272A81BA
:10268000822B90930F1C80930E1C22E0AE014F5FB3
:102690005F4F68EB8EEE0E94D611898190E0982FF3
:1026A00088272A81822B9093111C8093101C22E092
:1026B000AE014F5F5F4F6AEB8EEE0E94D6118981AB
:1026C00090E0982F88272A81822B9093151C809365
:1026D000141C22E0AE014F5F5F4F6CEB8EEE0E9448
:1026E000D611898190E0982F88272A81822B909398
:1026F000171C8093161C22E0AE014F5F5F4F6EEBFC
:102700008EEE0E94D611898190E0982F88272A8129
:10271000822B9093191C8093181C0F900F90DF91BF
:10272000CF9108952F923F924F925F926F927F9236
:102730008F929F92AF92BF92CF92DF92EF92FF92D1
:102740000F931F93CF93DF93CDB7DEB76A970FB682
:10275000F894DEBF0FBECDBF182F488F298F198286
:102760001A821B8280912C1C811107C06A8F0E94E3
:10277000C01281E080932C1C6A8D662309F46CC022
:102780004EE264EF8EEE0E94BF1169E07AE180E0D4
:1027900090E00E94F26022E0AE014F5F5F4F66EF73
:1027A0008EEE0E94D6112981822F90E0A0E0B0E049
:1027B0002227382F492F5A2F8A81282B80911E1CBF
:1027C00090911F1C281B390B41095109A0911C1C19
:1027D000B0911D1C0E94B78D6B017C018FE0F594B8
:1027E000E794D794C7948A95D1F76091161C70919D
:1027F000171C882777FD8095982F2BE0660F771F91
:10280000881F991F2A95D1F72091181C3091191C07
:10281000442737FD4095542F2C0D3D1D4E1D5F1D47
:102820000E946D8DC20ED31ED092131CC092121C3A
:1028300088E0C80ED11C34E0D594C7943A95E1F7EE
:10284000EE24D7FCE094FE2CC092201CD092211CD8
:10285000E092221CF092231C012F0295000F000F22
:10286000007C0C5CA12FB0E0BD8BAC8BA3E0B0E092
:10287000012E02C0AA0FBB1F0A94E2F725E335E040
:102880000E94B08DDC01CB010296A11DB11D8C8789
:102890009D87AE87BF8780E593ECA0E0B0E004C0E1
:1028A000B595A795979587951A95D2F7888B998BAB
:1028B000AA8BBB8B10E0188619861A861B86A8E0A7
:1028C0002A2E312CAC89BD892A1A3B0A988D1917FA
:1028D00009F436C1402F64EF8EEE0E94BF116C8563
:1028E0007D858E859F850E94F26023E0AE014F5F5B
:1028F0005F4F66EF8EEE0E94D611E091121CF091B0
:10290000131CE05AFF409F01DF010E94998D6B016B
:102910007C0180910A1C90910B1C9F8B8E8BA09048
:10292000081CB090091C20910C1C30910D1C0E94B9
:10293000998D2B013C013DE0759467945794479421
:102940003A95D1F7A0910E1CB0910F1CA7019601EA
:102950006CE055954795379527956A95D1F70E9474
:10296000C28DBB2797FDB095AB2F480E591E6A1E2E
:102970007B1E92E0490E511C611C711CB2E07594E3
:10298000679457944794BA95D1F7A0E85A0E611C02
:10299000711CA0911A1CB0911B1CA30192010E94F2
:1029A000B78DDC01CB012FE0B695A795979587955C
:1029B0002A95D1F78C839D83AE83BF8329818A8139
:1029C00090E0A0E0B0E04424582E692E7A2E622ACE
:1029D0008B81482A022C04C07594679457944794BD
:1029E0000A94D2F74501AA2497FCA094BA2C42E09D
:1029F000880C991CAA1CBB1C4A95D1F7A091101CED
:102A0000B091111CA70196010E94C28D6B017C013F
:102A100057E1F594E794D794C7945A95D1F72E8946
:102A20003F89DF010E94998DEBE095958795779519
:102A30006795EA95D1F7C60ED71EE81EF91E8C0CD5
:102A40009D1CAE1CBF1C0C8804C0880C991CAA1CC1
:102A5000BB1C0A94D2F792E0890E911CA11CB11CF8
:102A6000F2E0B594A79497948794FA95D1F7481813
:102A700059086A087B08A3019201688979898A89C3
:102A80009B890E94138D97FD0DC0660F771F881FCD
:102A9000991F2C813D814E815F810E944B8D4901A0
:102AA0005A010CC02C813D814E815F810E944B8D6B
:102AB00049015A01880C991CAA1CBB1C9927B7FC18
:102AC0009A958B2D7A2D692D9B01AC010E94138D57
:102AD0009B01AC01AEEDBBE00E94B78D6C01FF2401
:102AE000D7FCF094EF2CA3E4B3EEA50194010E946F
:102AF000C58DBB2797FDB095AB2FC80ED91EEA1E1A
:102B0000FB1EAFECCA0EAEE0DA1EE11CF11CA4E025
:102B1000F594E794D794C794AA95D1F7C80CD91C1B
:102B2000EA1CFB1C88859985AA85BB858C0D9D1D9B
:102B3000AE1DBF1D88879987AA87BB871F5FC6CE3A
:102B4000112391F0212F30E040E050E06885798535
:102B50008A859B850E944B8D2093241C3093251CD5
:102B60004093261C5093271CA98DAA2389F16091BC
:102B7000241C7091251C8091261C9091271C6115A6
:102B800071058105910521F10E94718A20E836EED8
:102B900045EC57E40E94D28921E03EED42E45EE339
:102BA0000E94B68C9B01AC0160E070E080E89FE37E
:102BB0000E9407892BE43AE34DEB57E30E94D28948
:102BC0006093281C7093291C80932A1C90932B1CC3
:102BD0006A960FB6F894DEBF0FBECDBFDF91CF91DE
:102BE0001F910F91FF90EF90DF90CF90BF90AF902B
:102BF0009F908F907F906F905F904F903F902F901D
:102C000008950F931F93CF93DF9300D000D000D08F
:102C1000CDB7DEB78E010F5F1F4F86E0F80111922E
:102C20008A95E9F780911E1B811113C040E061E392
:102C300086EA0E94BF114AE06CE286EA0E94BF1158
:102C400081E080931E1B6CE77EE380E090E00E94B1
:102C5000F26048E06DE286EA0E94BF116CE77EE315
:102C600080E090E00E94F26026E0A80162E386EA3C
:102C70000E94D61147E06DE286EA0E94BF118A8168
:102C800090E0982F88272981822B9093191B80939D
:102C9000181B2C8130E0322F22274B81242B3093BC
:102CA0001B1B20931A1B4E8150E0542F44276D812B
:102CB000462B50931D1B40931C1B5F934F933F93D8
:102CC0002F939F938F938BEF93E09F938F930E940B
:102CD00002940FB6F894DEBF0FBECDBF26960FB696
:102CE000F894DEBF0FBECDBFDF91CF911F910F9142
:102CF0000895CF92DF92EF92FF920F931F93CF939D
:102D0000DF93CDB7DEB72A970FB6F894DEBF0FBEBC
:102D1000CDBF8E010F5F1F4F86E0F80111928A959B
:102D2000E9F741E062E08CE30E94BF1148E560E012
:102D30008CE30E94BF1162E174E380E090E00E94A6
:102D4000F26026E0A80163E08CE30E94D61143E024
:102D500062E08CE30E94BF11098110E0102F002770
:102D60008A81082B1093F91A0093F81AEB80F12C42
:102D7000FE2CEE248C81E82AF092FB1AE092FA1ADB
:102D8000CD80D12CDC2CCC248E81C82AD092FD1A87
:102D9000C092FC1AB801882777FD8095982F0E9471
:102DA000718A9B01AC01B701882777FD8095982F28
:102DB0002F83388749875A870E94718A2F813885E7
:102DC00049855A850E947B8920EE3EE245E652E421
:102DD0000E94538C20E030E044E353E40E940889D1
:102DE0009F938F937F936F93DF92CF92FF92EF9297
:102DF0001F930F9389E094E09F938F930E94029416
:102E00000FB6F894DEBF0FBECDBF2A960FB6F8946A
:102E1000DEBF0FBECDBFDF91CF911F910F91FF900D
:102E2000EF90DF90CF900895CF93DF93EC018881EE
:102E300099810097F9F0843D904121F01982188220
:102E400083E063C085ED99E00E944458892BE1F04E
:102E50008091C5099091C60993FD18C08091C5095C
:102E60009091C60994FD43C08091C5099091C6090F
:102E700095FD44C060E870E085ED99E00E941D5822
:102E800084ED90E19983888381E03FC080913D206B
:102E900082FFE4CF21E048E061E083E00E949213EA
:102EA00080912B1C8F9380912A1C8F938091291CD9
:102EB0008F938091281C8F938091271C8F938091F2
:102EC000261C8F938091251C8F938091241C8F93B7
:102ED00084E59FE09F938F930E9414948DB79EB7D3
:102EE0000A960FB6F8949EBF0FBE8DBFB7CF8091E4
:102EF0003D2083FFB9CF0E940116B6CF80913D20BF
:102F000084FFB8CF0E947916B5CFDF91CF91089595
:102F1000CF93C82F8CEE0E9476618C2F0E94806127
:102F200065E375E080E090E00E94F2608DEE0E9423
:102F300076610E949161C82F0E949B612C2F30E026
:102F4000322F2227A901482BCA01CF910895CF9390
:102F5000DF93C82F8CEE0E9476618C2F0E948061D7
:102F600062E174E380E090E00E94F2608CEE0E94E7
:102F7000766180E00E94806165E375E080E090E02A
:102F80000E94F2608DEE0E9476610E949161C82FCE
:102F90000E949161D82F0E949B614D2F50E060E00C
:102FA00070E0762F652F542F44276C2B482BCB01D4
:102FB000BA01DF91CF9108952F923F924F925F9285
:102FC0006F927F928F929F92AF92BF92CF92DF9239
:102FD000EF92FF920F931F93CF93DF93CDB7DEB79E
:102FE000CD54D1090FB6F894DEBF0FBECDBF80918E
:102FF000000290910102892BD1F1109201021092EE
:1030000000028CEE0E9476618EE10E9480616BE18D
:103010007EE480E090E00E94F26082EA0E948817DD
:103020009093D2098093D10984EA0E9488179093E3
:10303000D0098093CF0986EA0E9488179093CE0921
:103040008093CD0988EA0E9488179093CC098093D9
:10305000CB098AEA0E9488179093CA098093C9090C
:103060008CEA0E9488179093C8098093C70988E466
:103070000E94A7176FAB78AF89AF9AAF88E50E941F
:10308000A7174B015C018091C9099091CA0920E002
:1030900030E040E050E0BA0126962FAF2697279601
:1030A0003FAF279728964FAF289729965FAF29976C
:1030B0002A966FAF2A972B967FAF2B979C0140E003
:1030C00050E060E070E080E090E008E00E94258F32
:1030D0000E94DE8E3901B42FA52FF62FE72F8C0129
:1030E0009401A50160E070E080E090E05301CB2EF8
:1030F000DA2EEF2EFE2E0E945C8F29833A832A015E
:103100001B014C01B101C401315041095F4F6F4FA8
:103110007F4F8F4F9F4FA1E0B0E02596BFAFAEAF7E
:10312000259721153F4F4F4F51406105710581058E
:10313000910509F020F425961FAE1EAE2597259621
:103140006EAC7FAC25978091C7099091C8095C014E
:10315000C12CD12CE12CF12C00E010E029813A8126
:10316000A201B101C4010E94CA8DD22EE32EF42E19
:10317000052F162FB72FF82FE92FA0E00E94838F7D
:1031800084F42150310940485F4F6F4F7F4F8F4F7C
:103190009F4FD22EE32EF42E052F162FB72FF82F88
:1031A000E92F2D2D3E2D4F2D502F612F7B2F8F2F4F
:1031B0009E2F07E10E943E8F2B8F3C8F4D8F5E8F9D
:1031C0006F8F78A389A39AA32053384F4F4F5F4F37
:1031D0006F4F7F4F8F4F9F4F2B8B3C8B4D8B5E8B59
:1031E0006F8B788F898F9A8F2056304F4F4F5F4F5C
:1031F0006F4F7F4F8F4F9F4F243D30434105510507
:10320000610571058105910541F038F025966EAC98
:103210007FAC2597FFEF6F1A7F0A8091CF099091BD
:10322000D0099C0140E050E060E070E080E090E078
:1032300000E10E94258F2B833C834D835E836A8748
:1032400079878F8398874091CB095091CC09A980C9
:10325000BA806201710184019A0140E050E060E0AF
:1032600070E080E090E00E94CA8DD22EE32EF42E12
:10327000052F162FB72FF82FE92FA0E00E94838F7C
:103280005CF4AFE70E94658FD22EE32EF42E052F5B
:10329000162FB72FF82FE92F2D2D3E2D4F2D502F04
:1032A000612F7B2F8F2F9E2F07E00E943E8F5901A9
:1032B0006A017B018C012B813C814D815E816A8595
:1032C00079858F8198850E945C8F2B833C834D8309
:1032D0005E836F8378878F87988B2E5F3F4F434045
:1032E00051096E4F7F4F8F4F9F4F22303105494F0D
:1032F0005F4F644071058105910521F018F01FEFC3
:10330000611A710A8091D1099091D209BC0180E0C3
:1033100090E020E030E840E050E00E94238E2987D2
:103320003A874B875C876A8B798B8D879E87409124
:10333000CD095091CE09A980BA8062017101840142
:103340009A0140E050E060E070E080E090E00E9490
:10335000CA8DD22EE32EF42E052F162FB72FF82F5D
:10336000E92FA0E00E94838F84F421503F4F4F4FFC
:103370005F4F6F4F7F4F8F4F9F4FD22EE32EF42E14
:10338000052F162FB72FF82FE92F2D2D3E2D4F2D5E
:10339000502F612F7B2F8F2F9E2F08E00E943E8F92
:1033A00059016A017B018C0129853A854B855C8531
:1033B0006A8979898D859E850E945C8F29873A87E5
:1033C0004B875C876D877E87898B9A8B2F5F3F4FFA
:1033D0004140510961097109810991092130304841
:1033E0004C4F5F47614071058105910521F018F050
:1033F000BFEF6B1A7B0A2B893C894D895E896F89E7
:10340000788D898D9A8D2F3C374041055105610596
:1034100071058105910511F00CF0A5C1A980BA8054
:103420006201710184019501A201B101C4010E94F0
:10343000CA8DA12CB12CC12C10E8D12EE12CF12C7D
:1034400000E010E00E94508E2BAF3CAF4DAF5EAF5E
:103450006FAF21967FAF219722968FAF2297239649
:103460009FAF2397AB8CBC8CCD8CDE8CEF8CF8A0FF
:1034700009A11AA19501A601B701C8010E94CA8D30
:1034800059016A017B01E82F192F02E00E94258F64
:103490000E2F0E945C8F69017A01162F272EF82FBC
:1034A000E92F322E8D2C942EAF2CB62E072F582EAE
:1034B000B92FA0E00E94838F5CF4A1E00E94658F89
:1034C000322E832E942EA52EB62E072F582EB92FCE
:1034D000232D382D492D5A2D6B2D702F852D9B2F87
:1034E00001E00E943E8F2E962FAF2E972D963FAF74
:1034F0002D9749A75AA76BA77CA78DA79EA7522EE9
:10350000432E4BA35CA36DA37EA38FA398A7B22DDC
:103510009601A701612F722D8F2F9E2FA0E00E9490
:10352000838F4CF4A3E00E94658F69017A01162F06
:10353000B72FF82FE92F9601A701612F7B2F8F2F2F
:103540009E2F02E00E943E8F2FA738AB49AB5AABAB
:103550006BAB7CAB8DAB9EAB19014A01B62FA72F8D
:1035600024968FAF2497F92F2B893C894D895E894A
:103570006F89788D898D9A8D24323A4F4F4F5F4FE6
:103580006F4F7F4F8F4F9F4F0CF08CC02B8D3C8D1A
:103590004D8D5E8D6F8D78A189A19AA12455324FF2
:1035A0004F4F5F4F6F4F7F4F8F4F9F4F59016A01B2
:1035B0007B018C010E94CA8D19014A01B62FA72FE9
:1035C000FC0103E00E94258F51016401EB2EFA2ECD
:1035D0008F010E94718F59016A017B018C012E9627
:1035E0002FAD2E972D963FAD2D9749A55AA56BA5CA
:1035F0007CA58DA59EA50E945C8F522E432E4BA3C9
:103600005CA36DA37EA38FA398A79101A4016B2F48
:103610007A2FCF0102E00E94258F51016401EB2E29
:10362000FA2E8F010E94718F02E00E94258F0E2FCB
:103630000E94718FF22E032F142FD52EE62EB72F56
:10364000F82FE92FA0E00E94838F5CF4A1E00E9494
:10365000658FF22E032F142FD52EE62EB72FF82FBD
:10366000E92F2F2D302F412F5D2D6E2D7B2F8F2F8A
:103670009E2F01E00E943E8F59016A017B018C015F
:103680002FA538A949A95AA96BA97CA98DA99EA9DA
:103690000E945C8F19014A01B62FA72F24968FAF85
:1036A0002497F92F2B813C814D815E816F81788534
:1036B0008F859889A52CB42CCBA0DCA0EDA0FEA012
:1036C0000FA118A50E94718F2B833C834D835E83CD
:1036D0006F8378878F87988B29853A854B855C85A2
:1036E0006D857E8589899A8951016401EB2EFA2EB8
:1036F00024960FAD24971F2F0E94718F29873A8738
:103700004B875C876D877E87898B9A8B2B893C8959
:103710004D895E896F89788D898D9A8DABACBCACF3
:10372000CDACDEACEFAC2196FFAC219722960FAD6D
:10373000229723961FAD23970E94718F2056304FFA
:103740004F4F5F4F6F4F7F4F8F4F9F4F243D304301
:1037500041055105610571058105910521F018F0BC
:103760002FEF621A720A6FA978AD89AD9AADAB01DD
:10377000BC0180E090E0DC0124964FAF24972596B1
:103780005FAF259726966FAF269727967FAF27972F
:1037900028968FAF289729969FAF29972A96AFAF83
:1037A0002A972B96BFAF2B97A984BA84CB84DC844D
:1037B000ED84FE8409891A899A01AB0160E070E00A
:1037C00080E090E00E94CA8DF22E032F142FD52E98
:1037D000E62EB72FF82FE92FA0E00E94838F84F404
:1037E00021503109404E5F4F6F4F7F4F8F4F9F4F9A
:1037F000F22E032F142FD52EE62EB72FF82FE92FF8
:103800002F2D302F412F5D2D6E2D7B2F8F2F9E2F33
:1038100005E10E943E8FAB80BC80CD80DE80EF80D2
:10382000F8840F8518890E94718FF22E032F142FB0
:10383000D52EE62EB72FF82FE92FA0E00E94838F18
:1038400084F4215030484F4F5F4F6F4F7F4F8F4F61
:103850009F4FF22E032F142FD52EE62EB72FF82FC1
:10386000E92F2F2D302F412F5D2D6E2D7B2F8F2F88
:103870009E2F0FE00E943E8F69017A018B018A839F
:10388000998329011A014B015C01285E33404109EB
:1038900051096109710981099109283D304D414063
:1038A0005105610571058105910521F018F0BFEF03
:1038B0006B1A7B0A0E947861672859F09601A7016C
:1038C000B8018A8199810E94DE8E29011A014B017B
:1038D0005C019201A101B401C5010E946B8A20E044
:1038E00030E048EC52E40E94D289C35BDF4F0FB650
:1038F000F894DEBF0FBECDBFDF91CF911F910F9126
:10390000FF90EF90DF90CF90BF90AF909F908F90FF
:103910007F906F905F904F903F902F9008954F92BF
:103920005F926F927F928F929F92AF92BF92CF924F
:10393000DF92EF92FF922B013C0169017A0123ECA7
:1039400035EF4CE851E4C701B6010E94538C4B019E
:103950005C0128EB3EE143E753E4C701B6010E9456
:1039600008899B01AC01C501B4010E94D2890E9463
:103970003F8A4B015C0120E030E048EC52E4C30197
:10398000B2010E94D28921E835E943EC50E40E945B
:10399000538CA50194010E94538C4B015C0123E3DD
:1039A00033E948E853E4C701B6010E9408899B0146
:1039B000AC01C501B4010E94D28923E333EB48E591
:1039C00053E40E94538CFF90EF90DF90CF90BF9014
:1039D000AF909F908F907F906F905F904F900895E1
:1039E0004F925F926F927F928F929F92AF92BF920F
:1039F000CF92DF92EF92FF9269017A010E94D58BFC
:103A000020E030E040E050E40E94078922E93CE5F4
:103A10004EED5EE30E94D2894B015C0123EC35EF51
:103A20004CE851E4C701B6010E94538C2B013C01C4
:103A300028EB3EE143E753E4C701B6010E94088941
:103A40009B01AC01C301B2010E94D2899B01AC0170
:103A5000C501B4010E9408896B017C0128EB3EE19D
:103A600043E753E40E94538C4B015C01A70196018C
:103A700063EC75EF8CE891E40E9407899B01AC012F
:103A8000C501B4010E94D289FF90EF90DF90CF90E2
:103A9000BF90AF909F908F907F906F905F904F906E
:103AA00008954F925F926F927F928F929F92AF9202
:103AB000BF92CF92DF92EF92FF922B013C016901FE
:103AC0007A0123EC35EF4CE851E4C701B6010E94BE
:103AD000538C4B015C0128EB3EE143E753E4C70103
:103AE000B6010E9408899B01AC01C501B4010E9486
:103AF000D2890E943F8A4B015C0120E030E048EC13
:103B000052E4C301B2010E94D289A50194010E942E
:103B1000538C20E030E040E251E40E94078924EE1B
:103B200038E34EE05FE30E94538C9B01AC01C70178
:103B3000B6010E940889FF90EF90DF90CF90BF9070
:103B4000AF909F908F907F906F905F904F9008956F
:103B500080E80E94766181110DC08EEF0E94806125
:103B6000811108C06BE17EE480E090E00E94F26089
:103B70000C9478610E94786180914F249091502438
:103B8000A0915124B09152240196A11DB11D8093A2
:103B90004F2490935024A0935124B093522408951D
:103BA000FC01DC0182E020E041E39D91292798E0BF
:103BB000322F330F27FF03C0232F242701C0232FC9
:103BC0009150B1F7815089F781E090E0328123175D
:103BD00011F080E090E00895DF92EF92FF920F9352
:103BE0001F93CF93DF930E94A81D80E80E94766107
:103BF00081116DC08AEF0E948061811168C08FE0E1
:103C00000E948061811163C065E375E080E090E00F
:103C10000E94F26081E80E947661811158C00E9482
:103C20009161C82F0E9491610E949161D82F0E94DA
:103C300091610E949161182F0E9491610E949B6185
:103C4000082F80E80E947661811141C08CEF0E94AC
:103C5000806181113CC089EC0E948061811137C074
:103C600065E375E080E090E00E94F26081E80E94E8
:103C700076610E949161E82E0E949161D82E0E9487
:103C800091610E949161F82E0E949B611F92DF92C8
:103C90001F92EF921F920F931F921F931F92DF9319
:103CA0001F92CF931F928F931F92FF928EE194E009
:103CB0009F938F930E9402940E9478618DB79EB764
:103CC00042960FB6F8949EBF0FBE8DBF17C00E94DC
:103CD000786180914F2490915024A0915124B0910B
:103CE00052240196A11DB11D80934F24909350241E
:103CF000A0935124B09352240E94A81D20E030E0EC
:103D000040E050E060E070E080E090E0DF91CF9133
:103D10001F910F91FF90EF90DF900895EF92FF9227
:103D20000F931F93CF93DF9300D01F92CDB7DEB7D1
:103D30008C0180E80E947661811154C00115110543
:103D400051F085EE0E94806181114CC061E077E9FD
:103D500080E090E009C083EE0E948061811142C042
:103D600069E97AEB81E090E00E94F26081E80E94CC
:103D70007661811137C00E949161F82E89830E947B
:103D80009161E82E8A830E949B618B830E947861F7
:103D9000CE0101960E94D01D892B21F16E2D70E07D
:103DA0007F296C7F80E090E0012B69F00E946F8A90
:103DB00020E030E04AEF5AE30E94538C20E030E0EC
:103DC00040EC50E40CC00E946F8A22E538EB4FE2D1
:103DD0005BE30E94538C26E636E64BE352E40E94F6
:103DE00007891BC00E94786180914F2490915024D4
:103DF000A0915124B09152240196A11DB11D809330
:103E00004F2490935024A0935124B09352240E94A5
:103E1000A81D60EF7FEF89E794E40F900F900F905B
:103E2000DF91CF911F910F91FF90EF9008950F9325
:103E30001F93CF93DF93729A8091580283FF08C03B
:103E40008EE40E941461811167C0C0E5D0E00AC011
:103E5000C0E5D0E087EE93E00E948C09219720977F
:103E6000C9F7EECF87EE93E00E948C092197209747
:103E7000C9F78FE40E9414610E949161082F0F73AB
:103E80000E949161182F0E949161D82F0E949B611E
:103E9000C82F0E9478618091580283FF7298602F2A
:103EA00070E0762F6627610F711D80E090E00E9420
:103EB0006F8A20E134E048EC5BE30E94538C60930E
:103EC000311C7093321C8093331C9093341C6D2FE3
:103ED00070E0762F66276C0F711D76956795769545
:103EE000679580E090E00E946F8A24EA3CEF44E20C
:103EF0005CE30E94538C20E030E040E252E40E94F8
:103F0000078960930E2970930F298093102990934D
:103F1000112980E090E002C081E090E0DF91CF9134
:103F20001F910F9108957298729A8EE40E94146105
:103F300080EA0E94806180E00E94806180E00E94AF
:103F400080618FE40E9414610E9491618EE40E945E
:103F5000146180E80E94806180E00E94806180E0BE
:103F60000E9480610E94786180E090E0089588EE70
:103F70009EE09F938F930E941494809173020F9000
:103F80000F90882361F01F928F9385EE9EE09F93A0
:103F90008F930E9414940F900F900F900F9008959C
:103FA00080EC9EE09F938F930E94149488E99EE09A
:103FB0009F938F930E94149481E79EE09F938F9329
:103FC0000E94149486E39EE09F938F930E94149422
:103FD00084E09EE09F938F930E94149488EC9DE070
:103FE0009F938F930E94149482EA9DE09F938F93F6
:103FF0000E9414948CE69DE09F938F930E941494EA
:1040000080913D2090913E20827091702DB73EB7F7
:10401000205F3F4F0FB6F8943EBF0FBE2DBF892BD8
:1040200041F08CE39DE09F938F930E9414940F9036
:104030000F9080E19DE09F938F930E94149484EDF4
:104040009CE09F938F930E9414948BEA9CE09F9333
:104050008F930E9414948FE79CE09F938F930E940C
:10406000149480E59CE09F938F930E9414948EE1BA
:104070009CE09F938F930E9414948DEE9BE09F93FE
:104080008F930E94149483EB9BE09F938F930E94E5
:1040900014948DE79BE09F938F930E9414948DE47A
:1040A0009BE09F938F930E94149481E29BE09F93E7
:1040B0008F930E94149482EF9AE09F938F930E94B3
:1040C000149489EB9AE09F938F930E94149480E854
:1040D0009AE09F938F930E94149489E49AE09F93AF
:1040E0008F930E94149485E19AE09F938F930E948E
:1040F00014948DB79EB780960FB6F8949EBF0FBEEE
:104100008DBF84EE99E09F938F930E94149485EB6A
:1041100099E09F938F930E94149486E899E09F936F
:104120008F930E9414948FE599E09F938F930E9440
:10413000149489E299E09F938F930E94149483EFE3
:1041400098E09F938F930E9414948DEB98E09F9337
:104150008F930E94149484E998E09F938F930E9418
:1041600014948CE598E09F938F930E94149481E3BC
:1041700098E09F938F930E9414942DB73EB72C5EC6
:104180003F4F0FB6F8943EBF0FBE2DBF08958DE48C
:1041900094E00C9438944F925F926F927F928F923A
:1041A0009F92AF92BF92CF92DF92EF92FF92CF9306
:1041B000DF93CDB7DEB728970FB6F894DEBF0FBEFA
:1041C000CDBF8091432490914424A0914524B09187
:1041D000462489839A83AB83BC83409043245090C8
:1041E000442460904524709046248091432490910B
:1041F0004424A0914524B09146248D839E83AF83AF
:10420000B887609143247091442480914524909113
:1042100046242CE3822E912CA12CB12CA5019401D3
:104220000E944B8D7F936F9330E1C32E3EE0D32EDF
:10423000E12CF12C6D817E818F819885A7019601FB
:104240000E944B8DA50194010E944B8D3F932F93AB
:1042500040E8842E41E5942EAA24A394B12CC301F6
:10426000B201A50194010E944B8DA70196010E9405
:104270004B8D3F932F9369817A818B819C81A5011E
:1042800094010E944B8D3F932F938BE098E09F9376
:104290008F930E9414940FB6F894DEBF0FBECDBF6B
:1042A00028960FB6F894DEBF0FBECDBFDF91CF9139
:1042B000FF90EF90DF90CF90BF90AF909F908F9046
:1042C0007F906F905F904F900895E3EDF1E38081D0
:1042D00091818234924479F0E35DF143FF93EF934F
:1042E0008DEE97E09F938F930E9414940F900F9000
:1042F0000F900F9008953A96E53F81E4F80738F360
:104300000895CF93DF93EC018C9A0E94D70A9F9374
:104310008F937F936F9381EE97E09F938F930E948B
:1043200014940F900F900F900F900F900F90209774
:1043300019F00E94F20B08C08FED97E09F938F93C6
:104340000E9414940F900F9081E00E94880A20919F
:1043500078023091790240917A0250917B020E945A
:10436000538C9F938F937F936F9383ED97E09F93ED
:104370008F930E9414940F900F900F900F900F90B6
:104380000F90209719F00E94F20B08C081ED97E082
:104390009F938F930E9414940F900F9082E00E943D
:1043A000880A2091740230917502409176025091F2
:1043B00077020E94538C9F938F937F936F9385EC2A
:1043C00097E09F938F930E9414940F900F900F90FB
:1043D0000F900F900F90209719F00E94F20B08C0D9
:1043E00083EC97E09F938F930E9414940F900F900B
:1043F00083E00E94880A9F938F937F936F9384EB4F
:1044000097E09F938F930E9414948C980F900F9035
:104410000F900F900F900F90209719F00E94F20BC1
:1044200008C082EB97E09F938F930E9414940F90A3
:104430000F9080913D2087FF83C021E042E161E041
:1044400080ED0E94D8629F938F937F936F9385EA4C
:1044500097E09F938F930E9414940F900F900F906A
:104460000F900F900F90209719F00E94F20B08C048
:1044700083EA97E09F938F930E9414940F900F907C
:1044800021E042E162E080ED0E94D8629F938F9329
:104490007F936F9386E997E09F938F930E94149484
:1044A0000F900F900F900F900F900F90209719F092
:1044B0000E94F20B08C084E997E09F938F930E94BB
:1044C00014940F900F9021E042E163E080ED0E9490
:1044D000D8629F938F937F936F9387E897E09F9322
:1044E0008F930E9414940F900F900F900F900F9045
:1044F0000F90CD2B19F00E94F20B08C085E897E0D1
:104500009F938F930E9414940F900F9021E042E1AB
:1045100064E080ED0E94D8629F938F937F936F93A6
:1045200088E797E09F938F930E9414940F900F90C9
:104530000F900F900F900F90DF91CF910C94F20B92
:10454000CD2BD1F3DF91CF9108950F931F93CF938C
:10455000DF93882389F049E050E06FEF70E082E05C
:1045600099E20E94569349E050E06AE070E082E0F0
:1045700099E20E94869513C0C2E0D9E203E717E0F2
:1045800089911F928F931F930F930E9414940F9001
:104590000F900F900F9089E2CA30D80789F7DF910A
:1045A000CF911F910F910C94F20B882311F02A9A4E
:1045B00008952A980895882311F02B9A08952B982E
:1045C0000895CF92DF92EF92FF92CF93DF936B012A
:1045D0007C0160FF11C08AE894E09F938F938DEF78
:1045E0009EE09F938F930E9414940F900F900F90D2
:1045F0000F9081E090E002C080E090E0C1FE09C031
:10460000EC01219643E259E06FE874E00E944B1000
:10461000CE01C2FE09C0EC01219643E259E067E9F0
:1046200074E00E944B10CE01C3FE09C0EC0121963C
:1046300043E259E06FE974E00E944B10CE01C4FEE2
:1046400009C0EC01219643E259E063EA74E00E945C
:104650004B10CE01C5FE09C0EC01219643E259E0A2
:1046600066EA74E00E944B10CE01C6FE09C0EC0160
:10467000219643E259E06AEA74E00E944B10CE01B1
:10468000C7FE09C0EC01219643E259E060EB74E0FB
:104690000E944B10CE01D0FE09C0EC01219643E2EE
:1046A00059E068EB74E00E944B10CE01D1FE09C0C6
:1046B000EC01219643E259E060EC74E00E944B105B
:1046C000CE01D2FE09C0EC01219643E259E064EC30
:1046D00074E00E944B10CE0120913D2030913E208D
:1046E00024703270232B59F0D3FE09C0EC012196BF
:1046F00043E259E06AEC74E00E944B10CE01209135
:104700003D2023FF0BC0D4FE09C0EC01219643E2FB
:1047100059E06FEC74E00E944B10CE0120913D20D7
:1047200024FF0BC0D5FE09C0EC01219643E259E0FD
:1047300065ED74E00E944B10CE01D6FE09C0EC017D
:10474000219643E259E06DED74E00E944B10CE01DA
:10475000B701A60144275078452B462B472B61F023
:1047600043E259E068EE74E0DF91CF91FF90EF9063
:10477000DF90CF900C944B10CD28CE28CF2841F459
:104780008EE697E09F938F930E9414940F900F9062
:10479000DF91CF91FF90EF90DF90CF9008950F932E
:1047A0001F93CF93DF938C01C0E0D0E0011511057A
:1047B00009F48AC069E677E0C8010E943593892B25
:1047C00009F4C16061E677E0C8010E943593892B46
:1047D00009F4C26069E577E0C8010E943593892B2E
:1047E00009F4C46065E577E0C8010E943593892B20
:1047F00009F4C86062E577E0C8010E943593892B0F
:1048000009F4C0616EE477E0C8010E943593892BFA
:1048100009F4C06268E477E0C8010E943593892BEF
:1048200009F4C06460E477E0C8010E943593892BE5
:1048300009F4C06868E377E0C8010E943593892BCA
:1048400009F4D16064E377E0C8010E943593892BB5
:1048500009F4D2606EE277E0C8010E943593892B9B
:1048600009F4D46069E277E0C8010E943593892B8E
:1048700009F4D86063E277E0C8010E943593892B80
:1048800009F4D0616BE177E0C8010E943593892B70
:1048900009F4D06260E177E0C8010E943593892B6A
:1048A00009F4D0646FEF76E0C8010E943593892B3C
:1048B00009F4D068609171027091720280E090E01A
:1048C0000E9449938C0172CFCE01DF91CF911F914D
:1048D0000F910895AF92BF92CF92DF92EF92FF9225
:1048E0000F931F93CF93DF93F22E032F142FE52EF8
:1048F000D62EA72EB82EC92E217030E040E050E011
:1049000060E070E080E090E0A0E00E94838F89F09A
:10491000E9EFF4E0FF93EF93EDEFFEE0FF93EF9309
:104920000E9414940F900F900F900F90E1E0F0E030
:1049300002C0E0E0F0E080913D2080FF17C02F2D05
:10494000247030E040E050E060E070E080E090E013
:10495000A0E00E94838F51F0EF01219643E259E0DD
:104960006DEF74E0CF010E944B10FE012F2D2270DD
:1049700030E040E050E060E070E080E090E0A0E0F7
:104980000E94838F51F0EF01219643E259E061E0EC
:1049900075E0CF010E944B10FE012F2D287030E0F2
:1049A00040E050E060E070E080E090E0A0E00E9435
:1049B000838F51F0EF01219643E259E069E175E000
:1049C000CF010E944B10FE012F2D207130E040E0FE
:1049D00050E060E070E080E090E0A0E00E94838F13
:1049E00051F0EF01219643E259E064E075E0CF0118
:1049F0000E944B10FE012F2D207230E040E050E06D
:104A000060E070E080E090E0A0E00E94838F51F0D1
:104A1000EF01219643E259E067E075E0CF010E9483
:104A20004B10FE012F2D207430E040E050E060E09C
:104A300070E080E090E0A0E00E94838F51F0EF01F1
:104A4000219643E259E06DE075E0CF010E944B10E2
:104A5000FE012F2D207830E040E050E060E070E073
:104A600080E090E0A0E00E94838F51F0EF0121965A
:104A700043E259E063E175E0CF010E944B10FE0173
:104A800020E0302F317040E050E060E070E080E0E6
:104A900090E0A0E00E94838F51F0EF01219643E265
:104AA00059E066E175E0CF010E944B10FE0120E065
:104AB000302F327040E050E060E070E080E090E045
:104AC000A0E00E94838F51F0EF01219643E259E06C
:104AD0006BE175E0CF010E944B10FE0120E0302F0A
:104AE000347040E050E060E070E080E090E0A0E0F2
:104AF0000E94838F51F0EF01219643E259E062E278
:104B000075E0CF010E944B10FE0120E0302F38707D
:104B100040E050E060E070E080E090E0A0E00E94C3
:104B2000838F51F0EF01219643E259E065E275E091
:104B3000CF010E944B10FE0120E0302F307140E089
:104B400050E060E070E080E090E0A0E00E94838FA1
:104B500051F0EF01219643E259E06AE275E0CF019E
:104B60000E944B10FE0120E0302F307240E050E0F8
:104B700060E070E080E090E0A0E00E94838F51F060
:104B8000EF01219643E259E061E375E0CF010E9415
:104B90004B10FE0120E030E040E050E06D2D6470ED
:104BA00070E080E090E0A0E00E94838F51F0EF0180
:104BB000219643E259E068E375E0CF010E944B1073
:104BC000FE0180913D2081FF17C020E0302F30741E
:104BD00040E050E060E070E080E090E0A0E00E9403
:104BE000838F51F0EF01219643E259E06CE375E0C9
:104BF000CF010E944B10FE0180913D2090913E20FC
:104C000090FF17C020E030E040E05E2D507160E082
:104C100070E080E090E0A0E00E94838F51F0EF010F
:104C2000219643E259E06FE375E0CF010E944B10FB
:104C3000FE0180913D2090913E2090FF17C020E022
:104C400030E040E05E2D507260E070E080E090E087
:104C5000A0E00E94838F51F0EF01219643E259E0DA
:104C600062E475E0CF010E944B10FE0180913D206F
:104C700090913E2090FF17C020E030E040E05E2D94
:104C8000507460E070E080E090E0A0E00E94838FCC
:104C900051F0EF01219643E259E068E475E0CF015D
:104CA0000E944B10FE0120E0302F307840E050E0B1
:104CB00060E070E080E090E0A0E00E94838F51F01F
:104CC000EF01219643E259E063E575E0CF010E94D0
:104CD0004B10FE0120E030E0412F417050E060E0D9
:104CE00070E080E090E0A0E00E94838F51F0EF013F
:104CF000219643E259E068E575E0CF010E944B1030
:104D0000FE0120E030E0412F427050E060E070E0B2
:104D100080E090E0A0E00E94838F51F0EF012196A7
:104D200043E259E06BE575E0CF010E944B10FE01B4
:104D300020E030E0412F447050E060E070E080E01F
:104D400090E0A0E00E94838F51F0EF01219643E2B2
:104D500059E06EE575E0CF010E944B10FE01809195
:104D60003D2087FF17C020E030E0412F487050E021
:104D700060E070E080E090E0A0E00E94838F51F05E
:104D8000EF01219643E259E061E675E0CF010E9410
:104D90004B10FE0180913D2087FF17C020E030E0DE
:104DA000412F407150E060E070E080E090E0A0E0D2
:104DB0000E94838F51F0EF01219643E259E065E6AE
:104DC00075E0CF010E944B10FE0180913D2087FFCE
:104DD00017C020E030E0412F407250E060E070E00A
:104DE00080E090E0A0E00E94838F51F0EF012196D7
:104DF00043E259E069E675E0CF010E944B10FE01E5
:104E000080913D2087FF17C020E030E0412F4074A3
:104E100050E060E070E080E090E0A0E00E94838FCE
:104E200051F0EF01219643E259E06DE675E0CF01C4
:104E30000E944B10FE0180913D2082FF17C020E0B0
:104E400030E0412F407850E060E070E080E090E09A
:104E5000A0E00E94838F51F0EF01219643E259E0D8
:104E60006DE376E0CF010E944B10FE0180913D2062
:104E700082FF17C020E030E040E05E2D517060E01E
:104E800070E080E090E0A0E00E94838F51F0EF019D
:104E9000219643E259E061E775E0CF010E944B1093
:104EA000FE0180913D2090913E2090FF17C020E0B0
:104EB00030E040E05E2D527060E070E080E090E015
:104EC000A0E00E94838F51F0EF01219643E259E068
:104ED00064E775E0CF010E944B10FE0180913D20F8
:104EE00090913E2090FF17C020E030E040E05E2D22
:104EF000547060E070E080E090E0A0E00E94838F5A
:104F000051F0EF01219643E259E06CE775E0CF01E3
:104F10000E944B10FE0180913D2090913E2091FF18
:104F20001EC020E030E040E05E2D587060E070E090
:104F300080E090E0A0E00E94838F89F043E259E096
:104F400065E875E0CF01DF91CF911F910F91FF9040
:104F5000EF90DF90CF90BF90AF900C944B102F2D1F
:104F6000302F412F5E2D6D2D7A2D8B2D9C2DA0E0A5
:104F70000E94838F41F48AEF96E09F938F930E9463
:104F800014940F900F90DF91CF911F910F91FF908C
:104F9000EF90DF90CF90BF90AF9008958F929F9247
:104FA000BF92DF92EF920F931F93CF93DF93EC01A9
:104FB0004B01FB01108265EF76E00E943593892B4F
:104FC00061F580913D207DE4D72EE0E8EE2E82FD54
:104FD00002C004E001C004E810E0B12C81FF02C06F
:104FE00060ECE62E26E04AE250E06BE270E089E2F7
:104FF00090E00E94195E81E090E00E94800B88237F
:1050000011F05DE5D52E80913D2090913E2090FDE0
:1050100016E091FF07C0186005C0D12CE12C00E01C
:1050200010E0B12C63EF76E0CE010E943593892B1E
:1050300061F481E0F40180836091710270917202E9
:1050400080E090E00E944993EC0161EF76E0CE01B0
:105050000E943593892B61F48FEFF4018083609176
:1050600071027091720280E090E00E944993EC011D
:10507000209709F424C16DEE76E0CE010E943593AD
:10508000892B19F4FD2DF160DF2E69EE76E0CE015B
:105090000E943593892B19F48D2D8460D82E66EEED
:1050A00076E0CE010E943593892B19F4ED2DE26054
:1050B000DE2E64EE76E0CE010E943593892B19F442
:1050C000FD2DF860DF2E61EE76E0CE010E94359373
:1050D000892B19F48D2D8061D82E6BED76E0CE01F1
:1050E0000E943593892B19F4ED2DE062DE2E65EDDB
:1050F00076E0CE010E943593892B19F4FD2DF064E2
:10510000DF2E62ED76E0CE010E943593892B19F4F3
:105110008D2D8068D82E6DEC76E0CE010E943593FF
:10512000892B19F4EE2DE160EE2E66EC76E0CE01CF
:105130000E943593892B19F4FE2DF260EF2E63EC5B
:1051400076E0CE010E943593892B19F48E2D846070
:10515000E82E6EEB76E0CE010E943593892B19F490
:10516000EE2DE860EE2E67EB76E0CE010E943593DF
:10517000892B19F4FE2DF061EF2E60EB76E0CE0165
:105180000E943593892B19F48E2D8062E82E6CEAEB
:1051900076E0CE010E943593892B19F4EB2DE46063
:1051A000BE2E69EA76E0CE010E943593892B19F470
:1051B000FE2DF064EF2E64EA76E0CE010E94359376
:1051C000892B19F48E2D8068E82E61EA76E0CE01F5
:1051D0000E943593892B09F401606EE976E0CE01D7
:1051E0000E943593892B09F402606BE976E0CE01C9
:1051F0000E943593892B09F4046067E976E0CE01BB
:105200000E943593892B09F4086063E976E0CE01AA
:105210000E943593892B09F400616FE876E0CE0196
:105220000E943593892B09F400626BE876E0CE0189
:105230000E943593892B09F4006469E876E0CE0179
:105240000E943593892B09F4006866E876E0CE0168
:105250000E943593892B09F411606EE776E0CE0148
:105260000E943593892B09F4126065E776E0CE0140
:105270000E943593892B09F414606CE676E0CE0128
:105280000E943593892B09F4186069E676E0CE0117
:105290000E943593892B09F4106163E676E0CE0114
:1052A0000E943593892B09F4106268E576E0CE01FF
:1052B0000E943593892B09F0D2CE1064D0CE2D2DCB
:1052C0003E2DA8016B2D70E080E090E0DF91CF9142
:1052D0001F910F91EF90DF90BF909F908F90089556
:1052E0005F926F927F928F929F92AF92BF92CF9276
:1052F000DF92EF92FF920F931F93CF93DF93782E5D
:10530000C7E2DBE100E010E0F2E5EF2EF6E0FF2E71
:105310008170582E872D8270682EADE3CA2EA6E0CC
:10532000DA2EB5E4AB2EB6E0BB2E83E4882E86E001
:10533000982E772051F01F930F93FF92EF920E94C7
:1053400014940F900F900F900F905520A1F0898525
:105350008F9388858F93BF92AF920E9414940F9081
:105360000F900F900F906620C1F09F928F920E9435
:1053700014940F900F90662081F0DF92CF920E94DC
:105380001494288139814A815B816C817D818E8171
:105390009F810E946A240F900F900E94F20B0F5F72
:1053A0001F4F2A960430110521F6DF91CF911F91EE
:1053B0000F91FF90EF90DF90CF90BF90AF909F90B4
:1053C0008F907F906F905F90089588E396E09F9311
:1053D0008F930E94149480912D1C90912E1CA0916B
:1053E0002F1CB091301C0F900F90813027EA92074C
:1053F0002EE1A207B10519F48AE296E01DC08230C1
:1054000026EA92072EE1A207B10519F48DE196E094
:1054100013C0823027EA92072EE1A207B10519F4E2
:105420008FE096E009C0823028EA92072EE1A207B9
:10543000B10549F481E096E09F938F930E94149404
:105440000F900F900895BF93AF939F938F938BEF1F
:1054500095E09F938F930E9414940F900F900F905C
:105460000F900F900F9008958BEE95E09F938F9380
:105470000E9414940E94C7200E94E5290E94F20B0A
:105480008EE09BE19F938F9383EE95E09F938F93A4
:105490000E941494609152027091530280915402C0
:1054A0009091550228EE33E040E050E00E944B8D91
:1054B0005F934F933F932F9383ED95E09F938F934B
:1054C0000E9414948AEC95E09F938F930E94149409
:1054D0000E94731080913D202DB73EB7225F3F4F51
:1054E0000FB6F8943EBF0FBE2DBF80FF05C041E050
:1054F00061E081E00E941D1286EC95E09F938F93FE
:105500000E94149480E00E94A5220E94CB208091EA
:1055100057021F928F938DEB95E09F938F930E947C
:1055200014948091C1091F928F9384EB95E09F930F
:105530008F930E941494809183028F9380918202B2
:105540008F93809181028F93809180028F9386EA5E
:1055500095E09F938F930E9414941F9280E48F9301
:105560008EE895E09F938F930E9414948091132965
:105570001F928F93809112291F928F938BE795E052
:105580009F938F930E941494809156021F928F9341
:1055900082E795E09F938F930E9414948091580224
:1055A00090915902A0915A02B0915B022DB73EB77B
:1055B000225E3F4F0FB6F8943EBF0FBE2DBF96FF41
:1055C00003C08EE895E002C081E995E09F938F9338
:1055D00088E695E09F938F930E94149483E00E9445
:1055E00070290F900F900F900F901D9B03C08EE8B5
:1055F00095E002C081E995E09F938F938CE595E05B
:105600009F938F930E94149482E595E09F938F93CC
:105610000E941494809158020F900F900F900F9059
:105620000F900F9081FF09C08CE495E09F938F93BA
:105630000E9414940F900F9013C080FF03C08EE857
:1056400095E002C081E995E09F938F9388E495E00F
:105650009F938F930E9414940F900F900F900F9030
:105660008091580290915902A0915A02B0915B0228
:1056700097FF03C08EE895E002C081E995E09F9313
:105680008F938FE395E09F938F930E94149488E308
:1056900095E09F938F930E9414946091C509709137
:1056A000C60980E090E00E94E1220E94F20B0F9078
:1056B0000F900F900F900F900F90779903C08EE886
:1056C00095E002C081E995E09F938F938FE295E08A
:1056D0009F938F930E9414940E9492090E943C0B06
:1056E0009F938F937F936F9381E295E09F938F9326
:1056F0000E9414940E94EB0A9F938F937F936F9361
:1057000083E195E09F938F930E94149481E090E051
:105710000E9481218091E8289091E928A091EA28AF
:10572000B091EB28BF93AF939F938F9385E095E063
:105730009F938F930E9414948091FD288F93809162
:10574000FC288F938091FB288F938091FA288F9368
:1057500081EF94E09F938F930E9414948091EC28A2
:105760009091ED28A091EE28B091EF28BF93AF93D0
:105770009F938F9383EE94E09F938F930E94149452
:105780008DB79EB782960FB6F8949EBF0FBE8DBFA1
:10579000809101298F93809100298F938091FF2818
:1057A0008F938091FE288F938FEC94E09F938F933B
:1057B0000E94149461E070E080E090E00E94FB0B96
:1057C00061E070E081E090E00E94FB0B0F900F9091
:1057D0000F900F900F900F90299B03C08EE895E0DB
:1057E00002C081E995E09F938F9387EC94E09F93AB
:1057F0008F930E9414940F900F900F900F902A9BFC
:1058000003C08EE895E002C081E995E09F938F93F5
:105810008FEB94E09F938F930E9414940F900F90BE
:105820000F900F900895F894E0E0F0E081E280930B
:1058300057008491E2E0F0E041E240935700449148
:10584000E4E0F0E091E290935700E49190E0A0E072
:10585000B0E0DC019927882750E060E070E0762F07
:10586000652F542F4427840F951FA61FB71F8E0F37
:10587000911DA11DB11D80932D1C90932E1CA093F2
:105880002F1CB093301C78940895CF93DF93CDB73D
:10589000DEB761970FB6F894DEBF0FBECDBF48E20A
:1058A00050E06EE170E087E29BE10E9468952091F4
:1058B000271B3091281B4091291B50912A1B609176
:1058C0002B1B70912C1B80912D1B90912E1BAFEFE9
:1058D0000E94838F09F05DC08DE48093271B80E8D0
:1058E0008093281B84E08093291B10922A1B10921E
:1058F0002B1B10922C1B10922D1B10922E1B8CE335
:1059000090E09093301B80932F1B1092311B1092CC
:10591000321B1092331B1092341B1092351B1092C5
:10592000361B1092371B1092381B10923A1B1092A4
:10593000391B10923B1B10923C1B10923D1B109286
:105940003E1B10923F1B1092401B1092411B109265
:10595000421B1092441B1092431B1092451B109245
:10596000461B1092471B1092481B1092491B109225
:105970004A1B10924B1B10924C1B10924E1B109204
:105980004D1B48E250E06EE170E087E29BE10E942F
:10599000869544E050E06AE170E0CE010B960E94EB
:1059A00068958B859C85AD85BE858F3F2FEF9207CF
:1059B000A207B207A9F48AE090E4A0E0B0E08093E7
:1059C000580290935902A0935A02B0935B0244E0AC
:1059D00050E06AE170E088E592E00E94869508C098
:1059E0008093580290935902A0935A02B0935B029D
:1059F0008091580290915902A0915A02B0915B0295
:105A0000A2FF02C02A9A03C080E00E94D52242E091
:105A100050E066E570E0CE010F960E9468958F8594
:105A200098898F3F2FEF920769F41092C609109260
:105A3000C50942E050E066E570E085EC99E00E941F
:105A4000869504C09093C6098093C50949E050E04B
:105A50006AE070E082E099E20E9468950E94330D4E
:105A600044E050E06AE470E0CE010B960E94689535
:105A70008B859C85AD85BE8544E050E06AE470E08E
:105A80008F3F9F4FAF4FBF4F29F488E792E00E94AE
:105A9000869504C088E792E00E94689544E050E053
:105AA00066E470E0CE010B960E9468958B859C851C
:105AB000AD85BE8544E050E066E470E08F3F9F4FC7
:105AC000AF4FBF4F29F484E792E00E94869504C04F
:105AD00084E792E00E94689544E050E06EE470E054
:105AE000CE010B960E9468958B859C85AD85BE8501
:105AF00044E050E06EE470E08F3F9F4FAF4FBF4FE8
:105B000029F48CE792E00E94869504C08CE792E02D
:105B10000E94689541E050E069E170E0CE01419655
:105B20000E946895898941E050E069E170E08F3F0B
:105B300029F481EC99E00E94869504C081EC99E0FB
:105B40000E94689541E050E068E170E0CE01419626
:105B50000E946895898941E050E068E170E08F3FDC
:105B600029F487E592E00E94869504C087E592E0DB
:105B70000E94689541E050E067E170E0CE014196F7
:105B80000E946895898941E050E067E170E08F3FAD
:105B900029F486E592E00E94869504C086E592E0AD
:105BA0000E9468954AE050E060E070E0CE01019606
:105BB0000E94689589814AE050E060E070E08F3F84
:105BC00029F48EE09BE10E94869504C08EE09BE163
:105BD0000E94689544E050E062E570E0CE010B96CB
:105BE0000E9468958B859C85AD85BE8544E050E01C
:105BF00062E570E08F3F9F4FAF4FBF4F29F480E8C1
:105C000092E00E94869504C080E892E00E94689528
:105C100044E050E063E170E0CE010B960E9468958D
:105C20008B859C85AD85BE8544E050E063E170E0E6
:105C30008F3F9F4FAF4FBF4F29F482E592E00E9404
:105C4000869504C082E592E00E94689561960FB641
:105C5000F894DEBF0FBECDBFDF91CF910895CF92F4
:105C6000DF92EF92FF92609171027091720280E078
:105C700090E00E94499365E975E00E945D93892B4D
:105C800009F01FC18DE48093271B80E88093281BB7
:105C900084E08093291B10922A1B10922B1B1092D8
:105CA0002C1B10922D1B10922E1B8CE390E09093D6
:105CB000301B80932F1B1092311B1092321B1092BD
:105CC000331B1092341B1092351B1092361B10920E
:105CD000371B1092381B10923A1B1092391B1092EE
:105CE0003B1B10923C1B10923D1B10923E1B1092CE
:105CF0003F1B1092401B1092411B1092421B1092AE
:105D0000441B1092431B1092451B1092461B10928D
:105D1000471B1092481B1092491B10924A1B10926D
:105D20004B1B10924C1B10924E1B10924D1B48E2C5
:105D300050E06EE170E087E29BE10E9486958AE088
:105D400090E4A0E0B0E08093580290935902A093B1
:105D50005A02B0935B0244E050E06AE170E088E5EB
:105D600092E00E9486951092C6091092C50942E001
:105D700050E066E570E085EC99E00E94869542E28D
:105D8000C42EDD24DA944CECE42E4BE3F42EC092C6
:105D90007802D0927902E0927A02F0927B0244E09B
:105DA00050E06AE470E088E792E00E948695C09235
:105DB0007402D0927502E0927602F092770244E08B
:105DC00050E066E470E084E792E00E94869587EDFB
:105DD00094E3AFEEBCE380937C0290937D02A093AA
:105DE0007E02B0937F0244E050E06EE470E08CE706
:105DF00092E00E9486958AE999E9A9E1B0E480934E
:105E0000800290938102A0938202B093830244E0C7
:105E100050E062E570E080E892E00E948695109282
:105E2000C10980E00E94946B41E050E069E170E0BC
:105E300081EC99E00E9486958AE1809357020E9446
:105E40003B6A41E050E068E170E087E592E00E9443
:105E500086958FE08093560241E050E067E170E064
:105E600086E592E00E9486958AE0EEE0FBE1DF01A4
:105E70001D928A95E9F74AE050E060E070E0CF01BA
:105E80000E94869580EA96E8A1E0B0E080935202F5
:105E900090935302A0935402B093550244E050E013
:105EA00063E170E082E592E00E94869581E00E94C5
:105EB000A52280E090E0FF90EF90DF90CF900C94CF
:105EC000470DFF90EF90DF90CF9008952F923F9273
:105ED0004F925F926F927F928F929F92AF92BF92FA
:105EE000CF92DF92EF92FF920F931F93CF93DF93A6
:105EF000CDB7DEB72B970FB6F894DEBF0FBECDBF80
:105F00009B878A874A01FC0180819181892B11F04E
:105F10000C9475426091710270917202CA010E94E4
:105F2000499360E870E0C4010E947C93009759F4A3
:105F30006091CD317091CE318AE090E00E94D09393
:105F400081E00C947A428130910561F4F401B080D3
:105F50001B2D110F110B012F412E512E612E712E71
:105F6000A12EBCC082309105B9F4F401808199273B
:105F700087FD9095982F88272181820F911D27FDFD
:105F80009A95B82E192F092F000F000B402E502E76
:105F9000602E702EA02EA2C083309105B1F5F401C1
:105FA0002081922F990F990B392F492F592F692F43
:105FB000792F892F00E10E94258F19012A013B01C9
:105FC000B82FA92F2181922F990F990B392F492F83
:105FD000592F692F792F892F08E00E94258F5901A9
:105FE0006A017B018C019101A201B3018B2F9A2FD1
:105FF0000E945C8FA2801A2D110F110BB12EC12EA1
:10600000D12EE12EF12E012F55C004970CF45DC066
:10601000F4012081922F990F990B392F492F592F75
:10602000692F792F892F08E10E94258F19012A01F4
:106030003B01B82FA92F2181922F990F990B392F4E
:10604000492F592F692F792F892F00E10E94258F21
:1060500059016A017B018C019101A201B3018B2FCF
:106060009A2F0E945C8FA3801A2D110F110BB12E55
:10607000C12ED12EE12EF12E012F0E945C8F19012D
:106080002A013B01B82FA92F2281922F990F990B3A
:10609000392F492F592F692F792F892F08E00E9416
:1060A000258F59016A017B018C019101A201B30185
:1060B0008B2F9A2F0E945C8FB22E132F042F452E08
:1060C000562E672E782EA92E09C07AE0B72E10E042
:1060D00000E0412C512C612C712CA12C0E94F20B60
:1060E0002B2D312F402F542D652D762D872D9A2D58
:1060F0002537F3E63F07FDE64F07510561057105BA
:106100008105910511F40C945D3D2537E3E63E07CA
:10611000EDE64E075105610571058105910511F008
:1061200008F0AAC12337F2E73F0741055105610591
:1061300071058105910511F40C94F03F2337E2E7D6
:106140003E0741055105610571058105910511F075
:1061500008F0B2C02536F4E63F0741055105610558
:1061600071058105910509F4C8C62536E4E63E07A8
:1061700041055105610571058105910509F0B8F5E5
:10618000A6E70E94838F11F40C94F4390E94838F48
:1061900009F068F4A8E60E94838F09F4F4C6A5E725
:1061A0000E94838F11F40C94DE390C9473422B2DD2
:1061B000312F402F542D652D762D872D9A2D2A3382
:1061C000F6E23F074105510561057105810591051D
:1061D00009F433C324363146410551056105710583
:1061E0008105910511F40C9418400C9473422B2DE9
:1061F000312F402F542D652D762D872D9A2D273741
:10620000FFE63F07410551056105710581059105CF
:1062100011F40C94C33D2737EFE63E0741055105C5
:10622000610571058105910509F0C8F42436F9E688
:106230003F0741055105610571058105910511F47F
:106240000C94B73925363E46410551056105710567
:106250008105910511F40C94F73D0C9473422B2D9C
:10626000312F402F542D652D762D872D9A2D2536D3
:10627000F2E73F074105510561057105810591056B
:1062800011F40C94C13E2936E2E73E074105510561
:10629000610571058105910511F40C949F3F23332D
:1062A000314741055105610571058105910511F0E1
:1062B0000C9473420C9418402B2D312F402F542DE9
:1062C000652D762D872D9A2D2236E5E63E07E4E6EC
:1062D0004E075105610571058105910509F40DC64B
:1062E0002236F5E63F07F4E64F07510561057105D3
:1062F0008105910511F008F054C02133E4E63E0712
:10630000E1E64E075105610571058105910509F426
:10631000A4C22133F4E63F07F1E64F0751056105BA
:1063200071058105910509F0C0F42337E3E73E07C5
:1063300041055105610571058105910511F40C9424
:106340000440283734474105510561057105810531
:10635000910509F472C20C9473422B2D312F402FFA
:10636000542D652D762D872D9A2D2336E4E63E0794
:10637000E1E64E075105610571058105910511F4AE
:106380000C94184028373446414651056105710583
:106390008105910511F00C9473420E9401160C9432
:1063A00075422B2D312F402F542D652D762D872DA5
:1063B0009A2D2D36E5E73E07E8E64E0751056105C3
:1063C00071058105910511F40C942E402D36F5E7E9
:1063D0003F07F8E64F0751056105710581059105F5
:1063E00009F0E0F42237E2E73E07E5E64E07510503
:1063F000610571058105910511F40C941C3D23364E
:106400003D4648465105610571058105910511F02C
:106410000C9473420E9479160C9475422B2D312FE7
:10642000402F542D652D762D872D9A2D2436E3E6A9
:106430003E07ECE64E0751056105710581059105A2
:1064400011F40C947F3C2736FFE63F07FCE64F072C
:106450005105610571058105910511F40C94823C8B
:106460002336324349465105610571058105910581
:1064700011F00C94734211C22B2D312F402F542D4B
:10648000652D762D872D9A2D2136FDE63F07F5E700
:106490004F07F8E65F07610571058105910511F465
:1064A0000C94E13D2136EDE63E07E5E74E07E8E6D0
:1064B0005E07610571058105910511F008F0D9C0ED
:1064C0002437F8E73F07F4E74F07510561057105E9
:1064D0008105910509F4F4C72437E8E73E07E4E7AE
:1064E0004E075105610571058105910511F008F010
:1064F00054C02133F1E33F07F1E74F075105610530
:1065000071058105910511F40C945D3D2133E1E3A2
:106510003E07E1E74E0751056105710581059105CB
:1065200009F0C8F42233F2E63F07F0E74F075105C0
:10653000610571058105910509F487C22033314356
:1065400041475105610571058105910511F40C94D0
:106550001C3D0C9473422B2D312F402F542D652D53
:10656000762D872D9A2D2037F5E63F07F2E74F0766
:106570005105610571058105910511F40C94C13E29
:106580002C36344744475105610571058105910555
:1065900011F40C949C410C9473422B2D312F402FFD
:1065A000542D652D762D872D9A2D2936FCE63F0733
:1065B000F1E64F07F3E65F07610571058105910577
:1065C00009F4D9C22936ECE63E07E1E64E07E3E6D8
:1065D0005E07610571058105910509F0E0F4243736
:1065E000F4E63F07F7E74F0751056105710581059F
:1065F000910511F40C94EA4124373F464F46524628
:10660000610571058105910511F00C9473420C949C
:1066100000000C9475422B2D312F402F542D652DE9
:10662000762D872D9A2D2633F9E63F07F5E74F079C
:10663000F5E65F07610571058105910509F4A7C4B9
:106640002037ECE63E07E5E64E07E8E65E07610523
:1066500071058105910509F496C42E3631464846E8
:106660005346610571058105910509F4FDC60C9439
:1066700073422B2D312F402F542D652D762D872DD4
:106680009A2D2437E3E73E07E5E64E07E2E75E078B
:10669000610571058105910511F40C94713E243753
:1066A000F3E73F07F5E64F07F2E75F07610571057E
:1066B0008105910511F008F055C02337E2E73E0748
:1066C000E7E74E07E0E75E07610571058105910583
:1066D00011F40C94743E2337F2E73F07F7E74F07B6
:1066E000F0E75F07610571058105910509F0C8F4C0
:1066F0002237E7E73E07E0E74E075E0761057105D1
:106700008105910509F406C22337354642475047B3
:10671000610571058105910511F40C94DE400C941E
:1067200073422B2D312F402F542D652D762D872D23
:106730009A2D2436EDE63E07E3E64E07E2E75E07D4
:10674000610571058105910509F42CC521363C468A
:1067500045465247610571058105910509F434C428
:106760000C9473422B2D312F402F542D652D762DF7
:10677000872D9A2D2437E2E73E07E1E64E07E5E74D
:106780005E07610571058105910509F466C5243729
:10679000F2E73F07F1E64F07F5E75F07610571058F
:1067A0008105910509F0C8F42437E3E73E07E5E6E3
:1067B0004E07E4E75E07610571058105910509F45F
:1067C000AAC62737304748475447610571058105F8
:1067D000910509F41FC60C9473422B2D312F402FC5
:1067E000542D652D762D872D9A2D2F36ECE63E07FC
:1067F000EFE54E07E6E75E07610571058105910546
:1068000009F47BC42C36F1E63F07F4E74F07F8E7BD
:106810005F07610571058105910511F40C946641CE
:106820002237374640475547610571058105910577
:1068300011F00C9473420C945A3C83E08093F0283E
:106840001092F2281092F12840EF58E262E184E3BE
:1068500092E00E949E550C94754221E042E161E075
:1068600080ED0E94D86221E042E161E080ED0E946B
:10687000D86221E042E161E080ED0E94D86221E02F
:1068800042E161E080ED0E94D86221E042E161E0F6
:1068900080ED0E94D8620C947542609171027091F3
:1068A000720280E090E00E9449936CE975E00E94DA
:1068B0005D93892B09F0C5C06091710270917202DD
:1068C00080E090E00E9449935C01009709F497C032
:1068D00060EE73E00E945D93892BE1F488EE93E013
:1068E000A0E0B0E08093520290935302A093540230
:1068F000B093550268EE73E080E090E00E94FF6084
:1069000044E050E063E170E082E592E00E94869509
:106910000C94754262EA75E0C5010E945D93892B73
:10692000E1F480E197E2A0E0B0E08093520290931E
:106930005302A0935402B093550260E177E280E0E5
:1069400090E00E94FF6044E050E063E170E082E587
:1069500092E00E9486950C94754265EA75E0C50147
:106960000E945D93892BE1F480EA96E8A1E0B0E013
:106970008093520290935302A0935402B093550215
:1069800060EA76E881E090E00E94FF6044E050E039
:1069900063E170E082E592E00E9486950C94754276
:1069A00069EA75E0C5010E945D93892BE1F480E8F6
:1069B0009AE1A6E0B0E08093520290935302A09334
:1069C0005402B093550260E87AE186E090E00E94BC
:1069D000FF6044E050E063E170E082E592E00E94F5
:1069E00086950C94754280E093E09F938F930E946C
:1069F00014940E94F20B0F900F900C9475426091CA
:106A0000520270915302809154029091550228EEE7
:106A100033E040E050E00E944B8D5F934F933F93F3
:106A20002F938CEF92E09F938F930E9414940E9477
:106A3000F20B0F900F900F900F900F900F900C94FF
:106A400075420E9473100C947542609171027091AE
:106A5000720280E090E00E9449938C016EE875E03C
:106A60000E945D93892BE1F4809158029091590224
:106A7000A0915A02B0915B02A46080935802909357
:106A80005902A0935A02B0935B022A9A44E050E064
:106A90006AE170E088E592E00E9486950C94754268
:106AA00061E975E0C8010E945D93892BF1F4809142
:106AB000580290915902A0915A02B0915B02AB7FAB
:106AC0008093580290935902A0935A02B0935B02AC
:106AD00080E00E94D52244E050E06AE170E088E561
:106AE00092E00E9486950C9475422A9B03C08EE822
:106AF00095E002C081E995E09F938F9384EF92E047
:106B00009F938F930E9414940F900F900F900F906B
:106B10000C947542609171027091720280E090E075
:106B20000E9449938C016EE875E00E945D93892B69
:106B300019F477980C94754261E975E0C8010E94D8
:106B40005D93892B19F4779A0C947542779903C059
:106B50008EE895E002C081E995E09F938F9389EAE2
:106B600094E09F938F930E9414940F900F900F9036
:106B70000F900C947542609171027091720280E0E6
:106B800090E00E9449938C0168E575E00E945D9356
:106B9000892B09F077C0609171027091720280E0D8
:106BA00090E00E9449938C01009711F40C94754277
:106BB0006DEA75E00E945D93892BB1F482E29FEF4C
:106BC000ACECBBE38093780290937902A0937A02B5
:106BD000B0937B0244E050E06AE470E088E792E022
:106BE0000E9486950C94754263EB75E0C8010E9483
:106BF0005D93892BB1F482E29FEFACECBAE3809312
:106C0000780290937902A0937A02B0937B0244E0D9
:106C100050E06AE470E088E792E00E9486950C9468
:106C20007542C8010E9433922B013C0120E030E004
:106C3000A9010E94CE898823D9F081E00E94880AA8
:106C40009B01AC01C301B2010E94D289609378021A
:106C50007093790280937A0290937B0244E050E033
:106C60006AE470E088E792E00E9486950C94754291
:106C700087EE92E09F938F930E9414940F900F9051
:106C80000C9475426BE575E0C8010E945D93892BF9
:106C900009F077C0609171027091720280E090E01B
:106CA0000E9449938C01009711F40C9475426DEA8F
:106CB00075E00E945D93892BB1F482E29FEFACEC0A
:106CC000BBE38093740290937502A0937602B09315
:106CD000770244E050E066E470E084E792E00E94CE
:106CE00086950C94754263EB75E0C8010E945D9334
:106CF000892BB1F482E29FEFACECBAE3809374028B
:106D000090937502A0937602B093770244E050E02E
:106D100066E470E084E792E00E9486950C947542E8
:106D2000C8010E9433922B013C0120E030E0A90110
:106D30000E94CE898823D9F082E00E94880A9B01B4
:106D4000AC01C301B2010E94D289609374027093B6
:106D50007502809376029093770244E050E066E4F7
:106D600070E084E792E00E9486950C9475428AED6B
:106D700092E09F938F930E9414940F900F900C9425
:106D8000754263E575E0C8010E945D93892B09F0A7
:106D900073C0609171027091720280E090E00E9475
:106DA00049938C01009711F40C9475426DEA75E0DB
:106DB0000E945D93892BB1F487ED94E3AFEEBCE3C1
:106DC00080937C0290937D02A0937E02B0937F0219
:106DD00044E050E06EE470E08CE792E00E9486951B
:106DE0000C94754263EB75E0C8010E945D93892B9A
:106DF00051F48BEC92E09F938F930E9414940F9028
:106E00000F900C947542C8010E9433922B013C01F3
:106E100020E030E0A9010E94CE89882319F180E0AA
:106E20000E94880A4B015C0121EE3AE744E95EE3E7
:106E3000C301B2010E940789A50194010E94D28971
:106E400060937C0270937D0280937E0290937F0218
:106E500044E050E06EE470E08CE792E00E9486959A
:106E60000C9475428EEB92E09F938F930E94149442
:106E70000F900F900C9475420E94D70A9F938F93A6
:106E80007F936F9387EB92E09F938F930E9414946C
:106E900082E00E94880A209174023091750240912C
:106EA0007602509177020E94538C162F072FF82EEE
:106EB000E92E81E00E94880AEF92FF920F931F93C0
:106EC000209178023091790240917A0250917B02B0
:106ED0000E94538C9F938F937F936F938BEA92E0E2
:106EE0009F938F930E9414940E94F20B0FB6F89414
:106EF000DEBF0FBECDBF0C947542609171027091E0
:106F0000720280E090E00E9449930097C1F00E94D5
:106F1000CF232091C5093091C6098217930709F143
:106F20009093C6098093C50942E050E066E570E0A1
:106F300085EC99E00E94869582EA94E002C08BE994
:106F400094E09F938F930E9414946091C50970916F
:106F5000C60980E090E00E94E1220E94F20B0F90AF
:106F60000F9080E994E09F938F930E9414946FEFA9
:106F70007FEF80E090E00E94E1220E94F20B0F90F0
:106F80000F900C9475420E94D01F0C947542F4012E
:106F90008481843329F440E061E080E00E941D1286
:106FA00080917302882311F40C9475421F928F9381
:106FB0008DE894E09F938F930E9414940F900F900C
:106FC0000F900F900C947542F4018481893709F079
:106FD00080C0609171027091720280E090E00E9426
:106FE00049938C016EE875E00E945D93892B51F402
:106FF0008091580290915902A0915A02B0915B027F
:10700000906410C061E975E0C8010E945D93892B0E
:10701000D1F48091580290915902A0915A02B091F6
:107020005B029F7B8093580290935902A0935A026F
:10703000B0935B0244E050E06AE170E088E592E0E2
:107040000E94869546C068EB75E0C8010E945D937A
:10705000892B21F58091261B8F938091251B8F937F
:107060008091241B8F938091231B8F938091221BEF
:107070008F938091211B8F938091201B8F93809100
:107080001F1B8F9380E892E09F938F930E9414942C
:107090000FB6F894DEBF0FBECDBF1BC08091580263
:1070A00090915902A0915A02B0915B0296FF03C0E1
:1070B0008EE895E002C081E995E09F938F938CE77D
:1070C00092E09F938F930E9414940F900F900F90D3
:1070D0000F9080917302882311F40C9475421F92D3
:1070E0008F938AE894E09F938F930E9414940F905B
:1070F0000F900F900F900C947542F40184818737A4
:10710000E9F5609171027091720280E090E00E9456
:1071100049930097D9F00E9433922B013C0120E063
:1071200030E0A9010E94CE89882381F0409280023C
:1071300050928102609282027092830244E050E099
:1071400062E570E080E892E00E948695809183027B
:107150008F93809182028F93809181028F9380918F
:1071600080028F938EE692E09F938F930E941494F7
:107170000F900F900F900F900F900F9080917302CF
:10718000882311F40C9475421F928F9387E894E042
:107190009F938F930E9414940F900F900F900F90D5
:1071A0000C947542609171027091720280E090E0DF
:1071B0000E9449938C016EE875E00E945D934090B7
:1071C00058025090590260905A0270905B02892BCD
:1071D00019F4689457F809C061E975E0C8010E9484
:1071E0005D93892B99F4E89457F840925802509295
:1071F000590260925A0270925B0244E050E06AE1E8
:1072000070E088E592E00E94869513C057FE03C0A7
:107210008EE895E002C081E995E09F938F938AE61E
:1072200092E09F938F930E9414940F900F900F9071
:107230000F9080917302882311F40C9475421F9271
:107240008F9384E894E09F938F930E9414940F90FF
:107250000F900F900F900C94754260917102709195
:10726000720280E090E00E9449935C016EEB75E051
:107270000E945D93892B11F489E108C062EC75E0EE
:10728000C5010E945D93892B49F480E18093C4007D
:107290001092C50082E08093C00055C066EC75E096
:1072A000C5010E945D93892B11F488E0EFCF6BEC50
:1072B00075E0C5010E945D93892B39F060ED75E0A2
:1072C000C5010E945D93892B11F483E0DFCF80918B
:1072D000C400893141F485E692E09F938F930E9428
:1072E00014940F900F908091C400803141F480E697
:1072F00092E09F938F930E9414940F900F9080912F
:10730000C400883041F48AE592E09F938F930E94F5
:1073100014940F900F908091C400833041F484E561
:1073200092E09F938F930E9414940F900F908091FE
:10733000C400883041F48EE492E09F938F930E94C2
:1073400014940F900F9080917302882311F40C9481
:1073500075421F928F9381E894E09F938F930E94D0
:1073600014940F900F900F900F900C9475426091B1
:1073700071027091720280E090E00E9449936DEA80
:1073800075E00E945D93892B11F481E001C080E0DB
:107390000E94A52280917302882311F40C947542F7
:1073A0001F928F938EE794E09F938F930E94149483
:1073B0000F900F900F900F900C9475420E94CB206D
:1073C00080917302882311F40C9475421F928F935D
:1073D0008BE794E09F938F930E9414940F900F90EB
:1073E0000F900F900C9475420E94C72080917302F9
:1073F000882311F40C9475421F928F9388E794E0D0
:107400009F938F930E9414940F900F900F900F9062
:107410000C947542609171027091720280E090E06C
:107420000E9449930E943792803170F48093C10981
:107430000E94946B41E050E069E170E081EC99E0DA
:107440000E9486950C9475428091C1091F928F937A
:1074500084E492E09F938F930E9414940F900F9076
:107460000F900F900C9475426091710270917202AE
:1074700080E090E00E9449930E94379295EF980F28
:10748000903170F4809357020E943B6A41E050E0D3
:1074900068E170E087E592E00E9486950C94754261
:1074A000809157021F928F938BE392E09F938F936B
:1074B0000E9414940F900F900F900F900C947542AF
:1074C000609171027091720280E090E00E94499395
:1074D000009789F04AE050E0BC018EE09BE10E94F9
:1074E0006D934AE050E060E070E08EE09BE10E9426
:1074F00086950C9475428EE09BE19F938F9385ED6A
:1075000095E09F938F930E9402940F900F900F909D
:107510000F900C947542609171027091720280E03C
:1075200090E00E9449935C0160EE73E00E945D93DD
:10753000892BD9F4219A8091580290915902A091F7
:107540005A02B0915B028061809358029093590275
:10755000A0935A02B0935B0244E050E06AE170E00D
:1075600088E592E00E948695C0C76CE575E0C5018C
:107570000E945D93892BD9F4229A809158029091B0
:107580005902A0915A02B0915B0280628093580226
:1075900090935902A0935A02B0935B0244E050E0EA
:1075A0006AE170E088E592E00E9486959EC762ECF1
:1075B00073E0C5010E945D93892BD9F4239A8091D1
:1075C000580290915902A0915A02B0915B028064D6
:1075D0008093580290935902A0935A02B0935B0291
:1075E00044E050E06AE170E088E592E00E94869510
:1075F0007CC76FEF74E0C5010E945D93892BD9F4BD
:10760000239A8091580290915902A0915A02B09108
:107610005B0280688093580290935902A0935A02AB
:10762000B0935B0244E050E06AE170E088E592E0EC
:107630000E9486955AC76CE679E0C5010E945D9369
:10764000892B71F581E08093542487E29BE190932C
:1076500056248093552410925824109257248091D8
:10766000580290915902A0915A02B0915B02916028
:107670008093580290935902A0935A02B0935B02F0
:1076800044E050E06AE170E088E592E00E9486956F
:1076900044E554E262E184E392E00E949E5525C7EE
:1076A00069EE73E0C5010E945D93892B11F5E7E552
:1076B000FBE1119211922BE1E737F207D1F78091AC
:1076C000580290915902A0915A02B0915B029260C7
:1076D0008093580290935902A0935A02B0935B0290
:1076E00044E050E06AE170E088E592E00E9486950F
:1076F000FCC661E975E0C5010E945D9340915802A6
:107700005091590260915A0270915B02892BC1F429
:107710004F705C7F409358025093590260935A0215
:1077200070935B022B9A44E050E06AE170E088E5D8
:1077300092E00E9486958091F9280E94506AD5C6F1
:1077400044FF03C08EE895E002C081E995E09F9375
:107750008F9380E392E09F938F930E941494809183
:1077600058020F900F900F900F9085FF03C08EE886
:1077700095E002C081E995E09F938F9385E292E0C6
:107780009F938F930E941494809158020F900F90B2
:107790000F900F9086FF03C08EE895E002C081E94C
:1077A00095E09F938F938AE192E09F938F930E943D
:1077B0001494809158020F900F900F900F9087FFB4
:1077C00003C08EE895E002C081E995E09F938F9316
:1077D0008FE092E09F938F930E94149480915802BF
:1077E00090915902A0915A02B0915B020F900F90B4
:1077F0000F900F9090FF03C08EE895E002C081E9E2
:1078000095E09F938F9384E092E09F938F930E94E3
:1078100014948091580290915902A0915A02B0910B
:107820005B020F900F900F900F9091FF03C08EE8B6
:1078300095E002C081E995E09F938F9389EF91E0F5
:107840009F938F930E9414948091580290915902B3
:10785000A0915A02B0915B020F900F900F900F9081
:1078600091FF43C68DED95E00E94389457E5A52E13
:107870005BE1B52E0BE010E065EE862E65E0962EFE
:10788000F50180819181F2E0AF0EB11C9F938F933F
:107890001F930F939F928F920E9402940F5F1F4F2E
:1078A0000F900F900F900F900F900F900B311105CC
:1078B00039F71BC684E794E09F938F930E9414943A
:1078C000809173020F900F90882361F01F928F9325
:1078D00081E794E09F938F930E9414940F900F90F0
:1078E0000F900F90F89428E088E190E00FB6F8949C
:1078F000A895809360000FBE20936000FFCF0E9488
:107900008962F3C5609171027091720280E090E02B
:107910000E9449938C016EE875E00E945D93892B6B
:10792000E9F40E943C698091580290915902A0911B
:107930005A02B0915B028D7F8160809358029093D0
:107940005902A0935A02B0935B0244E050E06AE10E
:1079500070E088E592E00E948695C7C561E975E010
:10796000C8010E945D93892BE1F40E94F468809124
:10797000580290915902A0915A02B0915B028C7FFB
:107980008093580290935902A0935A02B0935B02DD
:1079900044E050E06AE170E088E592E00E9486955C
:1079A000A4C560EF75E0C8010E945D93892BE9F4DE
:1079B0000E94F4688091580290915902A0915A0255
:1079C000B0915B028E7F826080935802909359023F
:1079D000A0935A02B0935B0244E050E06AE170E089
:1079E00088E592E00E94869580C58091580281FFCB
:1079F0000FC080EF95E09F938F9385EF91E09F9369
:107A00008F930E9414940F900F900F900F906DC55C
:107A100080FF03C08EE895E002C081E995E09F9366
:107A20008F9381EF91E09F938F930E9414940F9016
:107A30000F900F900F9059C5809152248F93809191
:107A400051248F93809150248F9380914F248F9352
:107A500080914E248F9380914D248F9380914C245C
:107A60008F9380914B248F9380914A248F938091A0
:107A700049248F93809148248F93809147248F933A
:107A80008EE494E09F938F930E94149480917302EC
:107A90000FB6F894DEBF0FBECDBF882309F425C50D
:107AA0001F928F938BE494E09F938F930E94149482
:107AB0000F900F900F900F9018C5F89481E090E010
:107AC00029E0FC0120935700C895E02C80E090E06D
:107AD000FC0120935700C895F02C7894F89483E02B
:107AE00090E0FC0120935700C895002D82E090E0C3
:107AF000FC0120935700C895102D78948091301C7C
:107B00008F9380912F1C8F9380912E1C8F93809147
:107B10002D1C8F9321E434E03F932F930E94149403
:107B20001F92EF921F92FF921F920F931F921F932B
:107B30008AE194E09F938F930E9414940E946521A0
:107B4000809166001F928F938EE094E09F938F93B5
:107B50000E9414940E94F20B809173020FB6F89465
:107B6000DEBF0FBECDBF882309F4BFC41F928F9321
:107B70008BE094E09F938F930E9414940F900F904A
:107B80000F900F90B2C460E070E080E090E00E943F
:107B9000FB0B60E070E081E090E00E94FB0B8091C5
:107BA0007302882309F4A1C41F928F9388E094E0A4
:107BB0009F938F930E9414940F900F900F900F90AB
:107BC00094C40E94931F0E94F20B80917302882339
:107BD00009F48BC41F928F9385E094E09F938F9359
:107BE0000E9414940F900F900F900F907EC460919C
:107BF00071027091720280E090E00E94499365EFFB
:107C000075E00E945D93892B31F5F8948CEF99E033
:107C10000E948B565C01009769F0C5010F960E9487
:107C20008F59B50184E092E00E944556C5010E943B
:107C30003357F0CF8CEF99E00E941857892B29F029
:107C40008CEF99E00E94C456F5CF8CEF99E00E942A
:107C50008756789434C08CEF99E00E948B565C0173
:107C60000BEF15E0A114B10451F1F50186811F92CB
:107C70008F9380851F928F9385811F928F9381852B
:107C80001F928F9387811F928F9384811F928F936E
:107C900083811F928F9382811F928F9382851F927F
:107CA0008F931F930F930E940294C5010E94335734
:107CB0005C010FB6F894DEBF0FBECDBFD3CF80916D
:107CC0007302882309F411C41F928F9382E094E019
:107CD0009F938F930E9414940F900F900F900F908A
:107CE00004C40E942F2E01C460917102709172022F
:107CF00080E090E00E9449938C016AE376E00E9464
:107D00005D93892BD1F48091580290915902A091F2
:107D10005A02B0915B02977F809358029093590268
:107D2000A0935A02B0935B0244E050E06AE170E035
:107D300088E592E00E948695D8C363EB75E0C801A0
:107D40000E945D93892BD1F4809158029091590241
:107D5000A0915A02B0915B02986080935802909370
:107D60005902A0935A02B0935B0244E050E06AE1EA
:107D700070E088E592E00E948695B7C30E94920960
:107D8000B4C3609171027091720280E090E00E9431
:107D90004993FC0120812332B1F44AE050E060E0D5
:107DA00070E001960E94EB8F1B016091710270914F
:107DB000720280E090E00E944993F4E02F163104B3
:107DC0000CF094C002C0212C312C009709F48EC015
:107DD0001982BE016F5F7F4F0E94CE2729013A01B1
:107DE0004B01B82FA92F8AE0829DF001839DF00DF1
:107DF0001124E95DF44E20812A8331813B83828105
:107E00008C8393819D8324812E8335813F8386815A
:107E10008887978199879201A301B4018B2F9A2FAC
:107E2000AA80BB80CC80DD80EE80FF80088519852C
:107E30000E947A8F09F45DC08981882351F18CF00A
:107E40002A81422A3B81532A8C81682A9D81792A82
:107E50002E81822A3F81932A8885B82B9985A92B68
:107E600018C0409450946094709480949094B0950D
:107E7000A0952A8142223B8153228C8168229D81D8
:107E800079222E8182223F8193228885B823998589
:107E9000A923408251826282738284829582B68352
:107EA000A78348E250E06EE170E087E29BE10E9428
:107EB00086958AEF93E09F938F930E9414948AE0B3
:107EC000829DF001839DF00D1124E95DF44E208127
:107ED00031814281538164817581868197810E94BD
:107EE0006A240E94F20B0F900F9003C082E00E9460
:107EF00070298EEE93E09F938F930E9414942FEF3E
:107F00003FEF4FEF5FEF6FEF7FEF8FEF9FEF0E943D
:107F10006A240E94F20B809173020F900F908823C5
:107F200009F4E3C21F928F938BEE93E09F938F939C
:107F30000E9414940F900F900F900F90D6C26091F2
:107F400071027091720280E090E00E944993FC01FE
:107F500020812332A1F44AE050E060E070E0019615
:107F60000E94EB8F8B01609171027091720280E030
:107F700090E00E94499304301105ECF402C000E047
:107F800010E00097C1F04AE050E060E070E00E942D
:107F90001F912AE0209FF001219FF00D1124E95D3F
:107FA000F44E7187608748E250E06EE170E087E24E
:107FB0009BE10E94869581E00E9470298091730266
:107FC000882309F492C21F928F9388EE93E09F93C7
:107FD0008F930E9414940F900F900F900F9085C272
:107FE0000E94C85980917302882309F47EC21F92AF
:107FF0008F9385EE93E09F938F930E9414940F903C
:108000000F900F900F9071C20E94342A80917302DA
:10801000882309F46AC21F928F9382EE93E09F93A4
:108020008F930E9414940F900F900F900F905DC249
:1080300080E090E00E94812180917302882309F4FE
:1080400054C21F928F938FED93E09F938F930E9462
:1080500014940F900F900F900F9047C280913D2085
:1080600081FF2DC00E94171F892B49F58091341C78
:108070008F938091331C8F938091321C8F938091CA
:10808000311C8F9384ED93E09F938F930E941494FF
:10809000809111298F93809110298F9380910F29BE
:1080A0008F9380910E298F9387EC93E09F938F930A
:1080B0000E9414940FB6F894DEBF0FBECDBF0E948D
:1080C000F20B80913D2090913E2090FF63C081E0B3
:1080D00090E00E948E1E3B014C0180E090E00E94E7
:1080E0008E1E1B012C010E94EC1D9F928F927F928D
:1080F0006F9286EB93E09F938F930E9414945F920C
:108100004F923F922F9286EA93E09F938F930E9423
:108110001494222D332D442D552D662D772D882D29
:10812000992D0E948F1C9F938F937F936F938BE960
:1081300093E09F938F930E941494222D332D442D0E
:10814000552D662D772D882D992D0E94F01C9F931B
:108150008F937F936F938DE893E09F938F930E940B
:108160001494222D332D442D552D662D772D882DD9
:10817000992D0E94511D9F938F937F936F938AE750
:1081800093E09F938F930E9414940FB6F894DEBFF0
:108190000FBECDBF0E94F20B80917302882309F4B9
:1081A000A4C11F928F9387E793E09F938F930E94C0
:1081B00014940F900F900F900F9097C180913D20D5
:1081C00082FF2BC021E048E061E083E00E9492132F
:1081D00080912B1C8F9380912A1C8F938091291C56
:1081E0008F938091281C8F938091271C8F9380916F
:1081F000261C8F938091251C8F938091241C8F9334
:1082000080E693E09F938F930E9414940E94F20B58
:108210000FB6F894DEBF0FBECDBF80913D20909188
:108220003E2091FF41C00E94DC17B62EA72E982E4B
:10823000892E20E030E048EC52E4D501F4016B2FA8
:108240007A2F8F2F9E2F0E94538C20E836EE45EC1C
:1082500057E40E94D28921E03EED42E45EE30E94B1
:10826000B68C9B01AC0160E070E080E89FE30E9467
:1082700007892BE43AE34DEB57E30E94D2899F93A1
:108280008F937F936F938F929F92AF92BF9287E469
:1082900093E09F938F930E9414940E94F20B0FB669
:1082A000F894DEBF0FBECDBF80917302882309F41E
:1082B0001CC11F928F9384E493E09F938F930E943D
:1082C00014940F900F900F900F900FC16091710256
:1082D0007091720280E090E00E9449936FE376E033
:1082E0000E945D93892BB1F46091710270917202CA
:1082F00080E090E00E944993009709F4F6C00E9444
:108300003792803108F0F1C090915201982B9093F0
:108310005201EBC0809152018F701F928F9384EEB7
:1083200091E09F938F930E9414940E94F20B0F9000
:108330000F900F900F90D9C06091710270917202EE
:1083400080E090E00E944993009711F14AE050E0EC
:1083500060E070E00E94EB8F603198F46093560209
:108360001F926F9387E393E09F938F930E941494DF
:1083700041E050E067E170E086E592E00E9486957A
:1083800011C0809156021F928F938EE293E006C037
:10839000809156021F928F9385E293E09F938F9373
:1083A0000E9414940F900F900F900F900E94F20B68
:1083B00080917302882309F498C01F928F9382E200
:1083C00093E09F938F930E9414940F900F900F90BF
:1083D0000F908BC0609171027091720280E090E00A
:1083E0000E9449938C016EE875E00E945D93892B91
:1083F000E1F40E94A5678091580290915902A091E2
:108400005A02B0915B029061809358029093590296
:10841000A0935A02B0935B0244E050E06AE170E03E
:1084200088E592E00E94869560C061E975E0C80128
:108430000E945D93892B81F5F8940E94B36788E1CF
:108440000FB6F89480936000109260000FBE84B75E
:10845000877F84BF80916000886180936000109264
:10846000600078948091580290915902A0915A022C
:10847000B0915B029F7E8093580290935902A09323
:108480005A02B0935B0244E050E06AE170E088E594
:1084900092E00E94869529C064E476E0C8010E94BB
:1084A0005D93409158025091590260915A02709127
:1084B0005B02892B21F454FF18C0F894FFCF54FFBE
:1084C00003C08EE895E002C081E995E09F938F9309
:1084D00080EE91E09F938F930E9414940F900F90E1
:1084E0000F900F9002C00E94B71FEA85FB85118292
:1084F000108283E02B960FB6F894DEBF0FBECDBF7F
:10850000DF91CF911F910F91FF90EF90DF90CF906F
:10851000BF90AF909F908F907F906F905F904F90A3
:108520003F902F9008950F931F93CF93DF93EC010B
:108530008A0188819981009711F1823C904121F054
:108540001982188283E020C06231E9F4A80162E157
:1085500070E08DEE99E00E94662F84E08093F02811
:108560001092F2281092F1281093F4280093F32827
:1085700040EF58E262E184E392E00E949E5582EC73
:1085800090E19983888381E0DF91CF911F910F91D2
:1085900008950E9499676C9A6B9A6A9A6F9A729A78
:1085A000749A739A779A809880B3897F80BB8398F6
:1085B000849887E080937E00549A0E94132C0E9436
:1085C000452C81E00E94FC0980E090E00E94470D6C
:1085D0006091520270915302809154029091550221
:1085E0000E94FF600E94EB0A60933F247093402436
:1085F00080934124909342248091580286FD239ACF
:10860000219A229A239A0895CF93DF93EC018881CF
:108610009981009741F08D3A904109F48CC01982FC
:10862000188283E093C00E94C9428091580280FD65
:1086300005C081FF01C01D9B0E94F46880917000FD
:108640008C7F809370008091B60080628093B6002A
:108650001092B20082E08093B1008091B6008770E2
:10866000E1F78091700081608093700060EB79E0A9
:1086700080E090E00E9483670E94C72080E00E9413
:10868000A5228FE69FE09F938F930E9414940E94EF
:10869000731080913D200F900F9086FD0E943562EF
:1086A00080913D2090913E2090FD0E94A81D8091D8
:1086B0003D2087FF06C021E04CE061E080ED0E9494
:1086C000D8628091C1090E94946B809157020E94E8
:1086D0003B6A0E94386A8093EC09809157020E949D
:1086E0003B6A8091C1091F928F938091EC091F9280
:1086F0008F9389E496E09F938F930E940294109247
:10870000EE091092ED090F900F900F900F900F90BF
:108710000F9088E492E090930C2980930B2983E2D8
:1087200090E09093FF118093FE118DEA90E1998380
:10873000888381E00BC06332E1F748E654E260E0F1
:1087400070E08DEE99E00E94662FE3CFDF91CF912C
:1087500008958436910514F19F938F938BE596E0ED
:108760009F938F930E940294809147249091482474
:10877000A0914924B0914A240196A11DB11D809376
:10878000472490934824A0934924B0934A240F90FF
:108790000F900F900F9081E090E0089580E090E0BE
:1087A00008952F923F924F925F926F927F928F9295
:1087B0009F92AF92BF92CF92DF92EF92FF920F9370
:1087C0001F93CF93DF93CDB7DEB7C859D1090FB64A
:1087D000F894DEBF0FBECDBFCF56DF4F998388839D
:1087E000C159D0408A01633871F481EF99E0C856CD
:1087F000DF4F6883C859D0400E94E153C856DF4F0D
:108800006881C859D040CF56DF4FA881B981C1597E
:10881000D0402D913C912A35B0E13B0709F4C9C302
:1088200040F42115310581F028393E4009F407C490
:10883000FBC32C3640E1340709F4D7C3233730415A
:1088400011F40C94E950F0C34AEE52E061E870E094
:1088500081EF99E00E94C75388E99EE0A1C3E3E05D
:10886000F0E0EC0FFD1FE20FF31F1082C9010E9420
:10887000A943892B89F720E030E040E050E0C3575E
:10888000DF4F6881CD58D040627070E080E090E0AA
:10889000A0E00E94838F09F084C6C557DF4F28816E
:1088A000CB58D040287030E040E050E060E070E00D
:1088B00080E090E0A0E00E94838FA1F127E04AE2EF
:1088C00050E06BE270E089E290E00E94195E82E085
:1088D00099E20E948760BC01882777FD8095982FD8
:1088E0000E94718A20E030E048EC52E40E94D28974
:1088F0009F938F937F936F938FE896E09F938F93CF
:108900001F9287E78F93CE018E0D9F1D03969F9335
:108910008F930E946594E80EF91E0FB6F894DEBF9F
:108920000FBECDBFC557DF4F2881CB58D040207137
:1089300030E040E050E060E070E080E090E0A0E0F7
:108940000E94838FF1F126E04AE250E06BE270E092
:1089500089E290E00E94195E81E090E00E94800B25
:108960008093C00980E89BE10E948760BC01882752
:1089700077FD8095982F0E94718A20E030E048ECC6
:1089800052E40E94D2899F938F937F936F9389E9DA
:1089900096E09F938F931F9287E78F93C70102966C
:1089A000E1E0F0E0EC0FFD1F8E0F9F1F9F938F9370
:1089B0000E946594E80EF91E0FB6F894DEBF0FBE54
:1089C000CDBF272D30E040E050E060E070E080E077
:1089D00090E0A0E00E94838F01F10E943C0B9F93E6
:1089E0008F937F936F9384EA96E09F938F931F9268
:1089F00087E78F93C701029641E050E04C0F5D1F5F
:108A0000840F951F9F938F930E946594E80EF91E23
:108A10000FB6F894DEBF0FBECDBFC557DF4F28811C
:108A2000CB58D040207430E040E050E060E070E08F
:108A300080E090E0A0E00E94838F31F18091422499
:108A40008F93809141248F93809140248F938091C4
:108A50003F248F9382EB96E09F938F931F9287E73B
:108A60008F93C7010296A1E0B0E0AC0FBD1F8A0F43
:108A70009B1F9F938F930E946594E80EF91E0FB67B
:108A8000F894DEBF0FBECDBFC557DF4F2881CB584E
:108A9000D040207830E040E050E060E070E080E0DE
:108AA00090E0A0E00E94838F41F1F8948091E82843
:108AB0009091E928A091EA28B091EB287894BF938F
:108AC000AF939F938F9380EC96E09F938F931F9229
:108AD00087E78F93C701029621E030E02C0F3D1FFE
:108AE000820F931F9F938F930E946594E80EF91E47
:108AF0000FB6F894DEBF0FBECDBF20E0C457DF4FE6
:108B00003881CC58D040317040E050E060E070E0F7
:108B100080E090E0A0E00E94838F09F054C520E03F
:108B2000C457DF4F3881CC58D040327040E050E01D
:108B300060E070E080E090E0A0E00E94838F09F0A8
:108B4000B5C520E0C457DF4F3881CC58D0403470D1
:108B500040E050E060E070E080E090E0A0E00E9443
:108B6000838F09F0D4C520E0C457DF4F3881CC583B
:108B7000D040387040E050E060E070E080E090E08D
:108B8000A0E00E94838F09F0F1C520E0C457DF4FB9
:108B90003881CC58D040307140E050E060E070E067
:108BA00080E090E0A0E00E94838F09F052C620E0B0
:108BB000C457DF4F3881CC58D040307240E050E08D
:108BC00060E070E080E090E0A0E00E94838F09F018
:108BD00070C620E030E040E050E0C357DF4F6881CE
:108BE000CD58D040647070E080E090E0A0E00E943A
:108BF000838F09F08CC620E0C057DF4F3881C05901
:108C0000D04040E050E060E070E080E090E0A0E024
:108C10000E94838F09F0E8C620E0CA56DF4F3881F2
:108C2000C659D04040E050E060E070E080E090E065
:108C3000A0E00E94838F09F005C720E030E0402FBC
:108C4000417050E060E070E080E090E0A0E00E94C1
:108C5000838F09F025C720E030E0402F427050E0BC
:108C600060E070E080E090E0A0E00E94838F09F077
:108C70004AC720E030E0C657DF4F4881CA58D0408D
:108C800050E060E070E080E090E0A0E00E94838F20
:108C900009F06CC720E030E0402F487050E060E001
:108CA00070E080E090E0A0E00E94838F09F088C728
:108CB00020E030E0402F407150E060E070E080E064
:108CC00090E0A0E00E94838F09F0AAC720E030E086
:108CD000402F407250E060E070E080E090E0A0E063
:108CE0000E94838F09F0CCC720E030E0402F407411
:108CF00050E060E070E080E090E0A0E00E94838FB0
:108D000009F0EFC7F02FF078BF2E20E030E04F2FB2
:108D100050E060E070E080E090E0A0E00E94838F8F
:108D200011F00C94A24E212F2170C22E20E030E0D1
:108D300040E05C2D60E070E080E090E0A0E00E9408
:108D4000838F11F00C94AF4E20E030E04B2D50E0BB
:108D500060E070E080E090E0A0E00E94838F11F07E
:108D60000C94BD4E20E030E040E05C2D60E070E00F
:108D700080E090E0A0E00E94838F11F00C94F24E0E
:108D800020E030E040E0512F527060E070E080E081
:108D900090E0A0E00E94838F11F00C94274F20E018
:108DA00030E040E0512F547060E070E080E090E0EF
:108DB000A0E00E94838F11F00C945A4F20E030E025
:108DC00040E0512F507160E070E080E090E0A0E062
:108DD0000E94838F11F00C948D4F20E030E040E032
:108DE000512F507260E070E080E090E0A0E00E94BF
:108DF000838F11F00C94CC4F20E030E040E0512FF5
:108E0000507460E070E080E090E0A0E00E94838F0A
:108E100011F00C940B5020E030E040E0512F5870DE
:108E200060E070E080E090E0A0E00E94838F11F0AD
:108E30000C944A5020E030E040E05D2D60E070E0AE
:108E400080E090E0A0E00E94838F11F00C947B50B2
:108E5000779A8091C5099091C60992FD749AC55779
:108E6000DF4F2881CB58D040C457DF4F3881CC58D2
:108E7000D040A801C357DF4F6881CD58D040CD56B0
:108E8000DF4F7881C359D040CC56DF4F8881C45919
:108E9000D040CB56DF4F9881C559D040A0E08E011D
:108EA0000D5F1F4F0E94838F11F00C94B75080917B
:108EB0005602806189838091E5098A83F801EE0D6D
:108EC000FF1D10828091C5099091C60987010D5F31
:108ED0001F4F80FF0CC01F930F9387E598E09F936F
:108EE0008F930E9402940F900F900F900F90B801F3
:108EF000CE0101960E94105D8091580282FF0AC047
:108F000028EE34E2A801BE016F5F7F4F81E692E058
:108F10000E94A5618091C5099091C60982FD739850
:108F20000E943C6981EF99E00E94E35380915802CE
:108F300090915902A0915A02B0915B0290FF40C0FB
:108F40003FEFE31AF30A0E94386AD82E89E10E94A3
:108F5000506A409158025091590260915A027091A2
:108F60005B0250FF29C073988091E5098F5F809361
:108F7000E5098A83B7016F5F7F4FCE0101960E949A
:108F8000105D81EF99E00E94E35340E050E065E816
:108F900080910212909103120E949E558AE590E101
:108FA000CF56DF4FA881B981C159D0408D939C9392
:108FB00038C0E12CF12CCDCF8D2D0E94506A739AD0
:108FC0008091C2099091C309892B11F00E94F46825
:108FD0008091E5098F5F8093E5098091C5099091A3
:108FE000C60982FF39CC739A37CC8DED99E00E9487
:108FF0004458892BB1F00E943C698091580287FD4A
:109000002B9860E470E08DED99E00E941D5883E795
:1090100090E1CF56DF4FE881F981C159D04091836B
:10902000808381E00C94FC50CF56DF4FA881B9813A
:10903000C159D0401D921C9283E00C94FC506231C7
:1090400081F7C0905802D0905902E0905A02F090F7
:109050005B02D1FC01CCF8018081813091F5018067
:10906000F281E02D2081C557DF4F2883CB58D040B7
:109070003181C457DF4F3883CC58D04002811381EF
:109080004481C357DF4F4883CD58D0405581CD56DA
:10909000DF4F5883C359D0408681CC56DF4F888339
:1090A000C459D0409781CB56DF4F9883C559D040E3
:1090B00020843184C257DF4F19821882CE58D040A5
:1090C0006AC08230E9F4A381B481C257DF4FB9830B
:1090D000A883CE58D040212C312CB1E0C557DF4FAA
:1090E000B883CB58D040C457DF4F1882CC58D040FB
:1090F00000E010E8C357DF4F1882CD58D0403CC085
:109100008330F9F0843009F0A7CB212C312CC257E1
:10911000DF4F19821882CE58D040E5E0C557DF4FA7
:10912000E883CB58D040C457DF4F1882CC58D0408A
:1091300000E010E0F2E0C357DF4FF883CD58D04095
:109140001BC0212C312CC257DF4F19821882CE58F8
:10915000D04025E0C557DF4F2883CB58D040C457B7
:10916000DF4F1882CC58D04000E010E031E0C35708
:10917000DF4F3883CD58D040CD56DF4F1882C359CA
:10918000D040CC56DF4F1882C459D040CB56DF4F69
:109190001882C559D04080903F2490904024A090E0
:1091A0004124B0904224409080025090810260900F
:1091B0008202709083022DEC3CEC4CE45EE3C30130
:1091C000B2010E9408899B01AC01C501B4010E9453
:1091D000948B87FD0BC0E894E0F8C0925802D092BF
:1091E0005902E0925A02F0925B024AC0A301920136
:1091F000C501B4010E94CE8987FF42C080914B24F3
:1092000090914C24A0914D24B0914E240196A11D23
:10921000B11D80934B2490934C24A0934D24B09384
:109220004E24E0FC19CB6894E0F8C0925802D0922A
:109230005902E0925A02F0925B0245E4C557DF4FB3
:109240004883CB58D04050E2C457DF4F5883CC58A6
:10925000D04000E010E084E0C357DF4F8883CD5852
:10926000D040CD56DF4F1882C359D040CC56DF4F87
:109270001882C459D040CB56DF4F1882C559D04010
:10928000902F9470C657DF4F9883CA58D04020E083
:1092900030E0492F50E060E070E080E090E0A0E036
:1092A0000E94838F09F08C9AC557DF4FA881CB5855
:1092B000D040A0727A2E2A2F30E040E050E060E0EB
:1092C00070E080E090E0A0E00E94838F11F00E94A7
:1092D0003C0BC457DF4FB881CC58D040B074C05756
:1092E000DF4FB883C059D04020E03B2F40E050E032
:1092F00060E070E080E090E0A0E00E94838F11F0D9
:109300000E94171FC457DF4FE881CC58D040E07847
:10931000CA56DF4FE883C659D04020E03E2F40E0D8
:1093200050E060E070E080E090E0A0E00E94838F79
:1093300051F00E94D70A6093F5287093F628809325
:10934000F7289093F828C557DF4F2881CB58D04095
:10935000217030E040E050E060E070E080E090E0BC
:10936000A0E00E94838FF1F08EE09BE19F938F93AA
:109370008FE696E09F938F931F9287E78F93CE019E
:1093800003969F938F930E9465946C010E94A9435A
:109390000FB6F894DEBF0FBECDBF892B09F05CCAB3
:1093A000760102C0E12CF12CC557DF4F2881CB5844
:1093B000D040227030E040E050E060E070E080E0BB
:1093C00090E0A0E00E94838FD1F1C701029667E789
:1093D00076E041E050E04C0F5D1F840F951F0E9426
:1093E000669353E0E50EF11C22E0A22E29E2B22E94
:1093F00032EFC32E33E0D32E47E7942ED5018D9163
:109400005D011F928F93DF92CF921F929F92C701AF
:109410000296E1E0F0E0EC0FFD1F8E0F9F1F9F937F
:109420008F930E946594E80EF91E0FB6F894DEBF84
:109430000FBECDBF3AE0A31639E2B306F9F6C55721
:10944000DF4F2881CB58D040247030E040E050E01E
:1094500060E070E080E090E0A0E00E94838F09F47B
:1094600047C0C70102966BE776E041E050E04C0F41
:109470005D1F840F951F0E94669354E0E50EF11C5A
:109480004E018AE7880E911C80E1D4011D928A95D5
:10949000E9F728E0A40168E980EB0E94D6115401A5
:1094A000B8E0AB0EB11C82EFC82E83E0D82E97E750
:1094B000692EF40181914F011F928F93DF92CF9219
:1094C0001F926F92C701029621E030E02C0F3D1FE2
:1094D000820F931F9F938F930E946594E80EF91E4D
:1094E0000FB6F894DEBF0FBECDBF8A149B0409F7F8
:1094F000512F5078D52E20E030E040E060E070E061
:1095000080E090E0A0E00E94838FE1F48091C209A6
:109510009091C3099F938F9380E896E09F938F93D8
:109520001F9287E78F93CE018E0D9F1D03969F9309
:109530008F930E946594E80EF91E0FB6F894DEBF73
:109540000FBECDBF20E030E040E050E0C357DF4F1A
:109550006881CD58D040617070E080E090E0A0E07C
:109560000E94838F09F487C9E3E0F0E0EC0FFD1F50
:10957000EE0DFF1D80E28083EBE6F4E2808197012F
:109580002F5F3F4F7901882309F469C98081A1E0E9
:10959000B0E0AC0FBD1FAE0DBF1D12968C9331967F
:1095A000EDCFCE018E0D9F1D67E876E003960E94F9
:1095B000669397E0E90EF11CC7010E94A943892B2D
:1095C00009F04AC96AC92114310409F4A8CAF894F7
:1095D0004090E8285090E9286090EA287090EB28A5
:1095E00078948091781B9091791BA0917A1BB0910F
:1095F0007B1BA3019201281B390B4A0B5B0BCA0191
:10960000B9010E946F8A4B015C01B10180E090E0DA
:109610000E946F8A9B01AC01C501B4010E94D289EE
:10962000B82EC92E9F938F937F936F938BEC96E008
:109630009F938F931F9287E78F939E012E0D3F1D5F
:109640002D5F3F4F3F932F93C856DF4F6883C85914
:10965000D040C956DF4F7883C759D0400E946594E7
:10966000E80EF91EC856DF4F6881C859D040C95668
:10967000DF4F7881C759D040862F972FAB2DBC2D57
:109680008093FA289093FB28A093FC28B093FD28A0
:109690004092781B5092791B60927A1B70927B1BD0
:1096A0000FB6F894DEBF0FBECDBF39CA2114310406
:1096B00009F447CAF89480914F1B9091501BA091D8
:1096C000511BB091521B78949F938F9380915F02AE
:1096D0008F9380915E028F9388ED96E09F938F9396
:1096E0001F9287E78F93C7010296A1E0B0E0AC0F0D
:1096F000BD1F8A0F9B1F9F938F930E946594E80E56
:10970000F91E0FB6F894DEBF0FBECDBF1ACAF8948B
:109710008091EC289091ED28A091EE28B091EF284F
:109720007894BF93AF939F938F9388EE96E09F9327
:109730008F931F9287E78F93C701029621E030E055
:109740002C0F3D1F820F931F9F938F930E94659450
:10975000E80EF91EC7010E94A9430FB6F894DEBFB8
:109760000FBECDBF892B09F077C8FDC92114310484
:1097700009F40BCAF8944090EC285090ED286090C2
:10978000EE287090EF28789480917C1B90917D1B3F
:10979000A0917E1BB0917F1BA3019201281B390B66
:1097A0004A0B5B0BCA01B9010E946F8A4B015C0135
:1097B000B10180E090E00E946F8A9B01AC01C5017D
:1097C000B4010E94D289B82EC92E9F938F937F93A4
:1097D0006F9383EF96E09F938F931F9287E78F930A
:1097E0009E012E0D3F1D2D5F3F4F3F932F93C85677
:1097F000DF4F6883C859D040C956DF4F7883C759B7
:10980000D0400E946594E80EF91EC856DF4F68816B
:10981000C859D040C956DF4F7881C759D040862FEC
:10982000972FAB2DBC2D8093FE289093FF28A093FB
:109830000029B093012940927C1B50927D1B6092BD
:109840007E1B70927F1B0FB6F894DEBF0FBECDBF9C
:109850009CC9232809F4ABC9F8948091531B9091BB
:10986000541BA091551BB091561B78949F938F93D6
:1098700080915D028F9380915C028F9380E097E0EE
:109880009F938F931F9287E78F93C7010296A1E062
:10989000B0E0AC0FBD1F8A0F9B1F9F938F930E9458
:1098A0006594E80EF91E0FB6F894DEBF0FBECDBF6B
:1098B0007EC98091432490914424A0914524B09185
:1098C0004624BF93AF939F938F9380E197E09F933C
:1098D0008F931F9287E78F93C701029621E030E0B4
:1098E0002C0F3D1F820F931F9F938F930E946594AF
:1098F000E80EF91EC7010E94A9430FB6F894DEBF17
:109900000FBECDBF892B11F00C942C4462C98091FD
:109910004E248F9380914D248F9380914C248F936C
:1099200080914B248F9380914A248F938091492476
:109930008F93809148248F93809147248F938BE15C
:1099400097E09F938F931F92B7E7CB2ECF92C701DB
:109950000296A1E0B0E0AC0FBD1F8A0F9B1F9F9342
:109960008F930E946594E80EF91EC7010E94A943D7
:109970000FB6F894DEBF0FBECDBF892B11F00C944B
:109980002C4480913D2090913E2090FF34C98091DD
:1099900052248F93809151248F93809150248F93E0
:1099A00080914F248F938FE397E09F938F931F9223
:1099B000CF92C701029621E030E02C0F3D1F820FAD
:1099C000931F9F938F930E946594E80EF91EC70121
:1099D0000E94A9430FB6F894DEBF0FBECDBF892BFE
:1099E00011F00C942C4407C98091341C8F93809102
:1099F000331C8F938091321C8F938091311C8F93F5
:109A000081E597E09F938F931F9287E78F93C7011C
:109A10000296A1E0B0E0AC0FBD1F8A0F9B1F9F9381
:109A20008F930E946594E80EF91EC7010E94A94316
:109A30000FB6F894DEBF0FBECDBF892B11F00C948A
:109A40002C44EAC88091F8288F938091F7288F934F
:109A50008091F6288F938091F5288F938CE597E07D
:109A60009F938F931F9287E78F93C701029621E000
:109A700030E02C0F3D1F820F931F9F938F930E9406
:109A80006594E80EF91EC7010E94A9430FB6F89429
:109A9000DEBF0FBECDBF892B11F00C942C44CDC876
:109AA00081E00E94880A20917802309179024091E9
:109AB0007A0250917B020E94538C9F938F937F93E5
:109AC0006F9389E697E09F938F931F9287E78F9319
:109AD000C7010296A1E0B0E0AC0FBD1F8A0F9B1F2B
:109AE0009F938F930E946594E80EF91EC7010E9410
:109AF000A9430FB6F894DEBF0FBECDBF892B11F07E
:109B00000C942C44A8C882E00E94880A2091740218
:109B10003091750240917602509177020E94538CE9
:109B20009F938F937F936F9386E797E09F938F9395
:109B30001F9287E78F93C701029621E030E02C0F38
:109B40003D1F820F931F9F938F930E946594E80E91
:109B5000F91EC7010E94A9430FB6F894DEBF0FBEDD
:109B6000CDBF892B11F00C942C4483C883E00E9454
:109B7000880A9F938F937F936F9383E897E09F93D7
:109B80008F931F9287E78F93C7010296A1E0B0E001
:109B9000AC0FBD1F8A0F9B1F9F938F930E946594EC
:109BA000E80EF91E8C98C7010E94A9430FB6F894DD
:109BB000DEBF0FBECDBF892B11F00C942C446AC8B8
:109BC00080913D2087FF74C821E042E161E080ED93
:109BD0000E94D8629F938F937F936F9380E997E061
:109BE0009F938F931F9287E78F93C701029621E07F
:109BF00030E02C0F3D1F820F931F9F938F930E9485
:109C00006594E80EF91EC7010E94A9430FB6F894A7
:109C1000DEBF0FBECDBF892B11F00C942C4448C879
:109C200080913D2087FF52C821E042E162E080ED53
:109C30000E94D8629F938F937F936F938EE997E0F2
:109C40009F938F931F9287E78F93C7010296A1E09E
:109C5000B0E0AC0FBD1F8A0F9B1F9F938F930E9494
:109C60006594E80EF91EC7010E94A9430FB6F89447
:109C7000DEBF0FBECDBF892B11F00C942C4426C83B
:109C800080913D2087FF30C821E042E163E080ED14
:109C90000E94D8629F938F937F936F938CEA97E093
:109CA0009F938F931F9287E78F93C701029621E0BE
:109CB00030E02C0F3D1F820F931F9F938F930E94C4
:109CC0006594E80EF91EC7010E94A9430FB6F894E7
:109CD000DEBF0FBECDBF892B11F00C942C440C9429
:109CE000744680913D2087FF0DC821E042E164E089
:109CF00080ED0E94D8629F938F937F936F938AEB3E
:109D000097E09F938F931F9287E78F93C7010296E7
:109D1000A1E0B0E0AC0FBD1F8A0F9B1F9F938F93F4
:109D20000E946594E80EF91EC7010E94A9430FB670
:109D3000F894DEBF0FBECDBF892B11F00C942C44DC
:109D40000C94824680913D2082FD02C00C94934683
:109D500046E061E083E00E9492130C949346809168
:109D60003D2082FD02C00C94A44621E046E061E063
:109D700083E00E9492130C94A44680913D2082FDC2
:109D800002C00C94B2468091271C8F938091261CB0
:109D90008F938091251C8F938091241C8F9388EC46
:109DA00097E09F938F931F9287E78F93C701029647
:109DB00041E050E04C0F5D1F840F951F9F938F93E0
:109DC0000E946594E80EF91EC7010E94A9430FB6D0
:109DD000F894DEBF0FBECDBF892B11F00C942C443C
:109DE0000C94B24680913D2082FD02C00C94C04686
:109DF00080912B1C8F9380912A1C8F938091291C1A
:109E00008F938091281C8F9380ED97E09F938F9381
:109E10001F9287E78F93C7010296E1E0F0E0EC0F15
:109E2000FD1F8E0F9F1F9F938F930E946594E80ED6
:109E3000F91EC7010E94A9430FB6F894DEBF0FBEFA
:109E4000CDBF892B11F00C942C440C94C04680910A
:109E50003D2090913E2090FD02C00C94CF4680E0C2
:109E600090E00E948E1E9F938F937F936F938BED54
:109E700097E09F938F931F9287E78F93C701029676
:109E800041E050E04C0F5D1F840F951F9F938F930F
:109E90000E946594E80EF91EC7010E94A9430FB6FF
:109EA000F894DEBF0FBECDBF892B11F00C942C446B
:109EB0000C94CF4680913D2090913E2090FD02C0B1
:109EC0000C94DE4681E090E00E948E1E9F938F935B
:109ED0007F936F938BEE97E09F938F931F9287E70B
:109EE0008F93C7010296E1E0F0E0EC0FFD1F8E0FAB
:109EF0009F1F9F938F930E946594E80EF91EC701E0
:109F00000E94A9430FB6F894DEBF0FBECDBF892BC8
:109F100011F00C942C440C94DE4680913D209091DD
:109F20003E2090FD02C00C94ED4681E090E00E943E
:109F30008E1E4B015C0180E090E00E948E1E9B0112
:109F4000AC01C501B4010E948F1C9F938F937F9336
:109F50006F938CEF97E09F938F931F9287E78F9378
:109F6000C701029641E050E04C0F5D1F840F951F22
:109F70009F938F930E946594E80EF91EC7010E947B
:109F8000A9430FB6F894DEBF0FBECDBF892B11F0E9
:109F90000C942C440C94ED4680913D2090913E20F1
:109FA00090FD02C00C94FC4681E090E00E948E1E61
:109FB0004B015C0180E090E00E948E1E9B01AC0191
:109FC000C501B4010E94F01C9F938F937F936F9300
:109FD00087E098E09F938F931F9287E78F93C70145
:109FE0000296E1E0F0E0EC0FFD1F8E0F9F1F9F93A4
:109FF0008F930E946594E80EF91EC7010E94A94341
:10A000000FB6F894DEBF0FBECDBF892B11F00C94B4
:10A010002C440C94FC4680913D2090913E2090FD74
:10A0200002C00C940B4781E090E00E948E1E4B0111
:10A030005C0180E090E00E948E1E9B01AC01C50196
:10A04000B4010E94511D9F938F937F936F9385E17D
:10A0500098E09F938F931F9287E78F93C701029693
:10A0600041E050E04C0F5D1F840F951F9F938F932D
:10A070000E946594E80EF91EC7010E94A9430FB61D
:10A08000F894DEBF0FBECDBF892B11F00C942C4489
:10A090000C940B4780913D2090913E2091FD02C091
:10A0A0000C941A470E94DC179F938F937F936F93B2
:10A0B00088E298E09F938F931F9287E78F93C70161
:10A0C0000296E1E0F0E0EC0FFD1F8E0F9F1F9F93C3
:10A0D0008F930E946594E80EF91EC7010E94A94360
:10A0E0000FB6F894DEBF0FBECDBF892B11F00C94D4
:10A0F0002C440C941A47C257DF4FA881B981CE581F
:10A10000D04016968C9116971F928F9315968C912E
:10A1100015971F928F9313968C9113971F928F937D
:10A1200012968C911F928F9389E398E09F938F935F
:10A130001F9287E78F93C7010296E1E0F0E0EC0FF2
:10A14000FD1F8E0F9F1F9F938F930E946594E80EB3
:10A15000F91EC7010E94A9430FB6F894DEBF0FBED7
:10A16000CDBF892B11F00C942C440C94284780917E
:10A17000C5099091C60982FD0CC08091580280FDEE
:10A1800008C081FD02C00C9457471D9902C00C9471
:10A1900057471F930F9380E598E09F938F930E94FA
:10A1A0000294809173020F900F900F900F9088236C
:10A1B00011F40C9457471F928F938CE69FE09F9366
:10A1C0008F930E9414940F900F900F900F900C9407
:10A1D00057478DED99E00E944458892B11F40C9457
:10A1E00011480E94F4688091580287FD02C00C94C7
:10A1F0002C442B9A0C942C44C856DF4F0FB6F8947D
:10A20000DEBF0FBECDBFDF91CF911F910F91FF90A9
:10A21000EF90DF90CF90BF90AF909F908F907F9006
:10A220006F905F904F903F902F9008950C940A5438
:10A230004F925F926F927F928F929F92AF92BF9256
:10A24000CF92DF92EF92FF920F931F93CF93DF9302
:10A25000CDB7DEB760970FB6F894DEBF0FBECDBFA7
:10A260006B010E94386AE82FF0E0EE0FFF1FEF5BF2
:10A27000F44E808191810196918380838091C509FC
:10A280009091C60981FD749880905802909059026F
:10A29000A0905A02B0905B020E94645C7C01FC01B9
:10A2A0008081982F92959F70913099F48F7051F41E
:10A2B0008091251B9091261B01969093261B8093DD
:10A2C000251B07C1B60182E199E20E948053892BC8
:10A2D00051F08091231B9091241B01969093241B95
:10A2E0008093231BF6C0D501C4011EE0B695A79547
:10A2F000979587951A95D1F7F82FF1708F2E8CEFDF
:10A3000099E00E948B568C01009709F448C0B60171
:10A31000C80102960E948053892BE9F198014AEC0A
:10A3200059E060E074E6C8010F960E940B59F701EE
:10A330009181F8018481981321C082858F5F828783
:10A340008091211B9091221B01969093221B809358
:10A35000211B84E00E94815DF801208530E02817F0
:10A36000390708F0A9C184E00E94815DF801808767
:10A37000F70180818F70F8018187ABC0F8011286E8
:10A3800084E00E94815DF8018087F70180818F70F1
:10A39000F801818792C1C8010E943357B4CF84E08D
:10A3A00092E00E9420568C01009709F492C0B601F9
:10A3B000C80102960E947753F70181818150F8010C
:10A3C000848380E091E0A0E0B0E083879487A58754
:10A3D000B687128684E00E94815DF8018087F701CC
:10A3E00080818F70F8018187B8018CEF99E00E941D
:10A3F000EB5698014AEC59E060E074E6C8010F960C
:10A400000E940B5999249394F7018181F801848368
:10A41000F70180818F70F801878384E00E94815D5D
:10A42000F801858383E00E94815D5C01F8018683E9
:10A4300087818F3009F0912CF7014180F8018481E8
:10A44000481A512C612C712C76E0440C551C661C6A
:10A45000771C7A95D1F72385348545855685A0EC00
:10A46000B0E00E94B78DBB27A92F982F872F480EE9
:10A47000591E6A1E7B1E43865486658676868091A9
:10A48000C5099091C60981FD2EC08091580280FDBA
:10A490002AC081FD26C08091580290915902A09156
:10A4A0005A02B0915B0297FDD2C0992091F082E0F0
:10A4B00080935424109256241092552410935824BB
:10A4C0000093572444E554E262E184E392E00E9461
:10A4D0009E558091C5099091C60981FFF0C0749A7C
:10A4E000EEC01D9BD8CFA4E6B0E0A30192010E946C
:10A4F000B78D672F782F892F992724E630E040E029
:10A5000050E00E944B8D7F936F93452C562C672C07
:10A5100077245F924F92BB24BF92AF92F80185815E
:10A520001F928F93F70180818F701F928F9381818B
:10A530001F928F93F60181811F928F9380811F92CA
:10A540008F93C70102969F938F9388E698E09F931D
:10A550008F930E940294809173020FB6F894DEBF2D
:10A560000FBECDBF882361F01F928F9389E69FE0D5
:10A570009F938F930E9414940F900F900F900F90C1
:10A580008091580290915902A0915A02B0915B02B9
:10A5900096FF2DC0882059F1F7012081322F3F709E
:10A5A000832F90E00297D4F08FEF830F207F822BD0
:10A5B000808381EF99E00E94165180911F1B90913A
:10A5C000201B01969093201B80931F1B8091C5092F
:10A5D0009091C60996FF0BC0739809C08091251B06
:10A5E0009091261B01969093261B8093251B8091AA
:10A5F0003D2086FF50CF0E942762C70105960E942A
:10A60000F361F70181811F928F93F80186811F9278
:10A610008F9385811F928F938CEA98E09F938F93FD
:10A620001F9280E18F939E012F5F3F4F6901DF9260
:10A630002F930E94659482E00E940D62C6010E94E1
:10A64000F3610FB6F894DEBF0FBECDBF24CF8EE00E
:10A650009BE120910E1B222309F427CF9F938F9318
:10A660008FEB98E09F938F93FE0131966F01DF92FD
:10A67000EF930E94A2945C01B601C70102960E946A
:10A6800087930F900F900F900F900F900F9000975F
:10A6900009F40BCF95012F5F3F4F280F391FA901F8
:10A6A0002F5F3F4FFA0180818032C9F362E18CE075
:10A6B00092E00E949E55F9CE812C912CA5CE6096F9
:10A6C0000FB6F894DEBF0FBECDBFDF91CF911F91C3
:10A6D0000F91FF90EF90DF90CF90BF90AF909F9041
:10A6E0008F907F906F905F904F9008950895FB0139
:10A6F0002081FC012083FB012181FC01218308953D
:10A70000FC019081DB018C91981309C081E090E0FD
:10A71000318111962C91321721F080E0089580E06C
:10A7200090E00895BC0182E199E20C947753DC013A
:10A730001996ED91FC911A970280F381E02D3097E4
:10A7400009F0099408950F931F93CF93DF9300D0DE
:10A75000CDB7DEB78C0188E10E94945DBC01CE01CB
:10A7600001960E947753D8011996ED91FC911A97A2
:10A770000190F081E02DBE016F5F7F4FC801099508
:10A780000F900F90DF91CF911F910F910895EF924D
:10A79000FF920F931F93CF93DF93EC018B017A010C
:10A7A00042E053E00E94F053FA86E98666E073E0E7
:10A7B000C801DF91CF911F910F91FF90EF900C9402
:10A7C00049540C940854CF93DF93EC0162E179E291
:10A7D00088E10E948A5DCE01DF91CF910C940A54EA
:10A7E000EF92FF920F931F93CF93DF93EC018B01B6
:10A7F0007A010E942554F886EF826AE073E0C8016E
:10A80000DF91CF911F910F91FF90EF900C944954DD
:10A810000C942D540C94B26EDC011796ED91FC91C2
:10A8200018970190F081E02D0994DC011796ED91C5
:10A83000FC9118970280F381E02D309709F009947C
:10A84000089580E092E10C948756FC017383628343
:10A85000BC0180E092E10C94EB56BC0180E092E1F7
:10A860000C94D056CF93DF93EC0180E092E10E94EC
:10A870008B56009749F0FC01228133812C173D074C
:10A8800029F00E943357F5CF80E090E0DF91CF911F
:10A8900008950F931F93CF93DF938B010E9432543F
:10A8A000EC01009731F01D830C83C8010E94E37016
:10A8B0008E83DF91CF911F910F9108951F93CF93B6
:10A8C000DF93EC01162FEC81FD813097D1F090934E
:10A8D00003128093021282E08887CE0106960995C2
:10A8E000992787FD90950297029710F0133839F455
:10A8F000BE01CE01DF91CF911F910C948B5481E06A
:10A900008887DF91CF911F910895FC01208520FD5C
:10A910000C945E540895CF92DF92EF92FF920F93C2
:10A920001F93CF93DF93EC016B01E0900212F09044
:10A9300003120091041210910512F801EC17FD07A3
:10A9400039F0309709F44AC00190F081E02DF6CF3C
:10A95000209709F443C08885882309F118860115DA
:10A96000110561F0C017D10729F0AE0167E8C801F1
:10A970000E948554F80100811181F1CFEC81FD81A5
:10A98000309769F0CC15DD0551F0D0930312C093D8
:10A99000021240E050E063E8CE0106960995E0918E
:10A9A0000412F0910512CE17DF0769F488819981AE
:10A9B00090930512809304120DC0808191818C17B1
:10A9C0009D0721F0FC013097C1F704C0888199816F
:10A9D00091838083F0920312E0920212DF91CF9173
:10A9E0001F910F91FF90EF90DF90CF9008951F93EC
:10A9F000CF93DF9310920E12C0910412D0910512E2
:10AA000011E0209779F08985882341F0188719860D
:10AA100040E050E062E8CE010E945E540990D88187
:10AA2000C02DEFCFDF91CF911F9108958091B1128A
:10AA300091E0980F9093B112089560910212709175
:10AA400003120C948B548AE88093B1121092AF12C7
:10AA50001092B0121092051210920412109203126A
:10AA600010920212089580910E1281110E94F754E3
:10AA70007091B012772309F451C0E091AF122E2FDC
:10AA800030E085E0E89FF0011124E15FFD4E608138
:10AA900060930D124181528150930C1240930B121E
:10AAA0008381948190930A12809309122F5F3F4F04
:10AAB0002F7133272093AF1271507093B01200970B
:10AAC00031F58091041290910512909308128093B1
:10AAD00007128091071290910812892BF9F080914A
:10AAE0000E1281110E94F75440910B1250910C12DA
:10AAF00060910D1280910712909108120E94855466
:10AB0000E0910712F091081280819181DECF6138C7
:10AB100019F421E0FC0120870E94855480910E12D7
:10AB20002091B01290E0820F911D089580910E1235
:10AB30002091B01290E0820F911D08952091B012E3
:10AB40002032B9F0E091AF12E20FEF71E0930612FC
:10AB500035E0E39FF0011124E15FFD4E60835283F5
:10AB60004183948383832F5F2093B01280E090E031
:10AB7000089581E090E00895CF93DF93C091021291
:10AB8000D09103120E948554D0930312C0930212F5
:10AB9000DF91CF910895AB013091041220910512FD
:10ABA000E32FF22FE817F907B1F0309721F0019069
:10ABB000F081E02DF7CF009771F0FC013083218305
:10ABC000909305128093041221E020871782168249
:10ABD00061E80C94BC550895009749F0FC0120856C
:10ABE0002150223020F421E0218720930E12089575
:10ABF00021E030E0FC018085811102C020E030E0DE
:10AC0000C9010895CF93DF93EC014A815B8160E035
:10AC100070E08C819D810E9456932A813B818881BE
:10AC20009981289FA001299F500D389F500D112414
:10AC300060E070E08E819F81DF91CF910C945693FC
:10AC4000FC018281938120E030E028173907D1F0A0
:10AC5000A481B581A20FB31F4C91411110C081E0B6
:10AC60008C9380819181289FA001299F500D389F4E
:10AC7000500D112486819781840F951F08952F5FB1
:10AC80003F4FE3CF80E090E00895FC0126813781BB
:10AC90004281538180E090E084179507C9F0261720
:10ACA000370781F4A481B581A80FB91F2C91121622
:10ACB00014F421502C930480F581E02DE80FF91F46
:10ACC00080810895A081B1812A0F3B1F0196E4CFB6
:10ACD0008FEF0895FC018681978168177907A0F0AE
:10ACE000A081B18142815381A49F9001A59F300D25
:10ACF000B49F300D1124280F391F81E090E06217B6
:10AD0000730720F080E0089580E090E00895FC0152
:10AD1000118210820895FC01808191810895FB01C8
:10AD200020813181FC01318320830895DC01ED9184
:10AD3000FC91309731F080819181009729F0FC01DE
:10AD4000FACF80E090E00895CF010895DC01ED9105
:10AD5000FC9111973097A9F020813181232B21F4A8
:10AD60001D921C92CF010895A081B1818D919C917B
:10AD70001197892B11F0FD01F7CF11821082CD01BF
:10AD8000089580E090E00895DC01ED91FC91119729
:10AD9000309721F0208131812D933C93CF0108958C
:10ADA000DC01ED91FC913097A9F0A0E0B0E02081AA
:10ADB0003181E617F70741F4109709F4DC012D9370
:10ADC0003C931182108208952115310519F0DF019D
:10ADD000F901EDCF08950F931F93CF93DF938C016B
:10ADE000EB010E94D05619821882C8010E94965623
:10ADF000009711F4F80101C0FC01D183C083DF91F9
:10AE0000CF911F910F9108950F931F93CF93DF93CD
:10AE1000EC018B010E94D05688819981F8019183C1
:10AE2000808319830883DF91CF911F910F9108953B
:10AE3000DC01ED91FC9180E090E0309729F00196E3
:10AE40000190F081E02DF9CF0895FB01309719F4BE
:10AE5000BA010C94045780819181DA018D939C93FF
:10AE6000518340830895009721F0FC0180819181F6
:10AE7000089580E090E008958091B4129091B51209
:10AE8000892B29F41092B3121092B21208950E94E5
:10AE90003F66E091B412F091B51222813381408176
:10AEA0005181240F351F281B390B0480F581E02DBB
:10AEB000309769F04281538160817181460F571F3D
:10AEC000481B590B4217530780F79A01EECF280F02
:10AED000391F3093B3122093B212089586E892E09E
:10AEE0000C94EC55EF92FF920F931F93CF93DF9347
:10AEF0008C01FC0180819181009799F08A35910540
:10AF0000D9F0F8011182108283E068C086819781B0
:10AF10008417950709F049C00480F581E02D30972A
:10AF2000A9F71092B5121092B4128AE590E0F801D8
:10AF30009183808381E052C0673891F16238A9F72C
:10AF4000C091B412D091B512E12CF12C209769F385
:10AF5000CE010E94B474892BF1F0AE0168E88E81B5
:10AF60009F810E949E55892BA1F41F821E828C8195
:10AF70009D81E114F10421F0F7019583848304C0DD
:10AF80009093B5128093B4121D821C820E943C578C
:10AF9000D7CF0E946E577E010C80DD81C02DD6CFA9
:10AFA000E091B412F091B512BACFF093B512E093DC
:10AFB000B412A481B581109709F4B7CF16968D917C
:10AFC0009C9117978417950711F0FD01F2CF149605
:10AFD0008D919C91159795838483EBCFDF91CF91D1
:10AFE0001F910F91FF90EF900895CF93DF93EC01A5
:10AFF0000E946E578E819F813091B4122091B512BC
:10B00000892B59F0E32FF22F309739F0EC17FD0719
:10B0100081F00480F581E02DF7CF809102129091AC
:10B0200003129F838E833C832D83D093B512C093EC
:10B03000B412DF91CF910C943C57CF93DF93EC0186
:10B040000E949474CE01DF91CF910C94F557CF9369
:10B05000DF93EC010E94A074CE01DF91CF910C949C
:10B06000F557CF93DF93EC010E94AA74CE01DF91D4
:10B07000CF910C94F557FC0120813181260F371FA9
:10B08000318320830C943C5721E030E0FC01868121
:10B090009781892B11F020E030E0C9010895FC016F
:10B0A0002281338180819181820F931F0895FC0159
:10B0B00080819181089581E090E02091B4123091D7
:10B0C000B512232B11F480E090E008958091B41222
:10B0D0009091B512892B29F08091B2129091B31200
:10B0E000089580E090E00895CF93DF93EC01E09124
:10B0F000B412F091B5128E179F0769F48C819D816F
:10B100009093B5128093B4120DC0848195818C17F1
:10B110009D0721F0FC013097C1F706C08C819D810D
:10B12000958384830E943C571D821C821F821E824D
:10B13000DF91CF910895EF92FF920F931F93CF93DA
:10B14000DF938C017A01FC0180819181009741F0AD
:10B150008B34910501F1F8011182108283E048C01F
:10B1600087EB92E10E948B56EC01209751F06C81A5
:10B170007D81CE0102960E941D580990D881C02D74
:10B18000F4CF81E08093B6128BE490E0F8019183D4
:10B19000808381E02DC06838E1F787EB92E10E945F
:10B1A0008B56EC01209781F3CE010296E816F90642
:10B1B000D9F4BE0187EB92E10E94D056E0900212D2
:10B1C000F09003128A859B8590930312809302125C
:10B1D000EC85FD85309719F08E859F850995F09255
:10B1E0000312E0920212D0CF0990D881C02DDACF9D
:10B1F000DF91CF911F910F91FF90EF9008951092E2
:10B20000B61287EB92E10E94875660E070E080E919
:10B2100092E00C94CB550F931F93CF93DF93EC01E7
:10B2200000910212109103121B870A875D874C87D9
:10B230003F872E878091B612882379F080E992E0CB
:10B240009093031280930212CE0102960E941D5821
:10B25000109303120093021202C07D836C83BE011F
:10B2600087EB92E10E94D056BE0187EB92E1DF911D
:10B27000CF911F910F910C94EB560F931F93CF9387
:10B28000DF93EC018091B612882391F000910212B5
:10B290001091031280E992E09093031280930212BE
:10B2A000CE0102960E9427581093031200930212B7
:10B2B000BE0187EB92E10E94D056BE0187EB92E17E
:10B2C000DF91CF911F910F910C94EB560F931F9329
:10B2D000CF93DF93EC018091B612882391F0009117
:10B2E00002121091031280E992E09093031280936E
:10B2F0000212CE0102960E9431581093031200935D
:10B300000212BE0187EB92E10E94D056BE0187EB8C
:10B3100092E1DF91CF911F910F910C94EB56CF9357
:10B32000DF93EC018091B612882329F0CE010296BA
:10B330000E94745804C01F821E8219861886BE019E
:10B3400087EB92E1DF91CF910C94D056CF93DF93AE
:10B35000EC018091B612882331F0CE010296DF9184
:10B36000CF910C94445887EB92E10E948B56009742
:10B3700039F08C179D0739F0FC0180819181F7CF5E
:10B3800081E090E002C080E090E0DF91CF910895ED
:10B390002F923F924F925F926F927F928F929F92E5
:10B3A000AF92BF92CF92DF92EF92FF920F931F93D3
:10B3B000CF93DF93CDB7DEB7E8970FB6F894DEBF33
:10B3C0000FBECDBFE9E4FBE2208131814281538190
:10B3D000E5E4FBE25080418032802380E1E4FBE23F
:10B3E0008081898391819A83A281AB836380EDE31D
:10B3F000FBE2B081BC8381818D8392819E83A38196
:10B40000AF83E9E3FBE2B081B887818189879281CC
:10B410009A87A381AB87E5E3FBE2B081BC8781819A
:10B420008D8792819E87A381AF87E1E3FBE2B081A4
:10B43000B88B8181898B92819A8BA381AB8BEDE252
:10B44000FBE2B081BC8B81818D8B92819E8BA3812D
:10B45000AF8BE9E2FBE2B081B88F8181898F928165
:10B460009A8FA381AB8FE5E2FBE2B081BC8F818133
:10B470008D8F92819E8FA381AF8FE1E2FBE2B0813D
:10B48000B8A3818189A392819AA3A381ABA3EDE1A3
:10B49000FBE2B081BCA381818DA392819EA3A38195
:10B4A000AFA3E9E1FBE2B081B8A7818189A79281CE
:10B4B0009AA7A381ABA7E5E1FBE2B081BCA781819C
:10B4C0008DA792819EA7A381AFA7E1E1FBE2B081A6
:10B4D000B8AB818189AB92819AAB7380EDE0FBE2DE
:10B4E000B080A18092808380E9E0FBE2F080E1807F
:10B4F000D280C380E5E0FBE2A081AFABB181B8AF01
:10B50000128103812BAB3CAB4DAB5EAB0E946D66F1
:10B510005EA95F934DA94F933CA93F932BA92F930D
:10B520002F923F924F925F926F922B812F932A819D
:10B530002F9329812F932F812F932E812F932D814C
:10B540002F932C812F932B852F932A852F93298539
:10B550002F9328852F932F852F932E852F932D851D
:10B560002F932C852F932B892F932A892F93298909
:10B570002F9328892F932F892F932E892F932D89ED
:10B580002F932C892F932B8D2F932A8D2F93298DD9
:10B590002F93288D2F932F8D2F932E8D2F932D8DBD
:10B5A0002F932C8D2F932BA12F932AA12F9329A179
:10B5B0002F9328A12F932FA12F932EA12F932DA14D
:10B5C0002F932CA12F932BA52F932AA52F9329A539
:10B5D0002F9328A52F932FA52F932EA52F932DA51D
:10B5E0002F932CA52F937F922AA92F9329A92F93CC
:10B5F00028A92F938F929F92AF92BF92CF92DF9202
:10B60000EF92FF920F931F9328AD2F932FA92F93A3
:10B610009F938F937F936F93A3E1B9E28C911F92D5
:10B620008F93E2E1F9E280811F928F9384EE9FE095
:10B630009F938F930E941494E9E7FBE2208131816C
:10B6400042815381E5E7FBE25080418032802380D4
:10B65000E9E6FBE29080818072806380E5E6FBE2B0
:10B660008081898391819A83A281AB83B381BC83DA
:10B67000E1E6FBE280818D8391819E83A281AF838D
:10B68000B381B887EDE5FBE28081898791819A8754
:10B69000A281AB87B381BC87E9E5FBE280818D871E
:10B6A00091819E87A281AF87B381B88BE5E5FBE2EC
:10B6B0008081898B91819A8BB280A380E1E5FBE246
:10B6C000F080E180D280C380EDE4FBE2A081AB8B0F
:10B6D000B181BC8B128103810FB6F894DEBF0FBE1F
:10B6E000CDBF2BAB3CAB4DAB5EAB0E946D665EA994
:10B6F0005F934DA94F933CA93F932BA92F932F9272
:10B700003F924F925F926F927F928F929F922C8185
:10B710002F932B812F932A812F9329812F93288573
:10B720002F932F812F932E812F932D812F932C8553
:10B730002F932B852F932A852F9329852F93288943
:10B740002F932F852F932E852F932D852F93AF9297
:10B75000BF922A892F9329892F93CF92DF92EF925C
:10B76000FF920F931F932C892F932B892F939F93D5
:10B770008F937F936F93A3E1B9E28C911F928F9384
:10B78000E2E1F9E280811F928F9385E79FE09F932A
:10B790008F930E9414940FB6F894DEBF0FBECDBFF6
:10B7A000E8960FB6F894DEBF0FBECDBFDF91CF9104
:10B7B0001F910F91FF90EF90DF90CF90BF90AF90CF
:10B7C0009F908F907F906F905F904F903F902F90C1
:10B7D000089580E380936D130895CF93DF93609174
:10B7E0006D1370E0C0E3D0E0C61BD70B65547D4EEF
:10B7F000AE010E944D93CE01DF91CF910895CF927B
:10B80000DF92EF92FF920F931F93CF93DF937C0110
:10B81000C0907013D090711360916D1370E0E601C9
:10B82000E096C61BD70BC138D105D8F400E310E071
:10B83000061B170B65547D4EA8010E944D93609125
:10B84000B9127091BA1280916E1390916F13680FB4
:10B85000791FA601C701800F911F0E944D93CE0151
:10B8600002C080E090E0DF91CF911F910F91FF9097
:10B87000EF90DF90CF90089590916D13980F909373
:10B880006D13089540917013509171134817590723
:10B8900098F020916E1330916F13280F391F309359
:10B8A0006F1320936E13481B590B509371134093E1
:10B8B000701381E090E0089580E090E00895909307
:10B8C000711380937013089580916E1390916F138C
:10B8D00085519D4E089580916D1390E085549D4E45
:10B8E000089581E090E02091B9123091BA122B5E58
:10B8F000324111F480E090E008950E94715C892B40
:10B9000061F06091B9127091BA1240917013509128
:10B9100071138BEE92E10C944D9320916E13309144
:10B920006F1321153105B9F0809170139091711347
:10B93000C096EBEEF2E1AF014B5B5241481759075D
:10B9400034F4DF01A20FB31F4C914193F4CF109256
:10B950006F1310926E1308958091B9129091BA12DC
:10B9600008958091701390917113089590916D13C3
:10B9700080E3891B089520E380916D13281B80913B
:10B98000701390917113820F911D08951F93CF939F
:10B99000DF93EC0110916D13812F90E08C179D07C0
:10B9A0006CF00E94BB5C8C0F9D1F8138910530F4B8
:10B9B0001C1B10936D1381E090E002C080E090E0CA
:10B9C000DF91CF911F910895CF93DF93ECE1F9E2DE
:10B9D0001192119289E2EC34F807D1F7C4E1D9E26F
:10B9E00060E073E0CE010E947753229689E2CC3169
:10B9F000D807B1F7DF91CF91089510926F1310928D
:10BA00006E13109271131092701380E380936D1374
:10BA10008BEE92E19093BA128093B9120C94E45C8D
:10BA2000EF92FF920F931F93CF93DF9300D0CDB788
:10BA3000DEB78C0169837A830E94FD5C6981E62E02
:10BA40007A81F72E81E8E816F10418F080E8E82EF4
:10BA5000F12CA701B8018091B9129091BA120E94FD
:10BA60004D93F0927113E0927013C7010F900F90F5
:10BA7000DF91CF911F910F91FF90EF9008950F9359
:10BA80001F93CF93DF938C01EB010E94FD5C109319
:10BA9000BA120093B912D0937113C0937013DF914F
:10BAA000CF911F910F91089520E3ECE1F9E2DC01C1
:10BAB00001900D922A95E1F788E0E4E1F9E2DB01DB
:10BAC00001900D928A95E1F7089520E3FC01ACE125
:10BAD000B9E201900D922A95E1F788E0FB01A4E11B
:10BAE000B9E201900D928A95E1F70895E82FF0E010
:10BAF000EE0FFF1FE45EF64D7183608381E090E0FE
:10BB00000895E82FF0E0EE0FFF1FE45EF64D808110
:10BB10009181089590E0880F991F8C51974D0E9454
:10BB2000775381E090E0089590E0880F991F8C5141
:10BB3000974D08958115910511F00197F1F708953A
:10BB4000E0914F29F0915029908180914E298923CD
:10BB50000895E0914C29F0914D29808190914E29D2
:10BB6000892B8083E0915129F09152298081909115
:10BB70004E29892B80830895E0914C29F0914D291D
:10BB8000908180914E29809589238083E09151296D
:10BB9000F0915229908180914E298095892380834C
:10BBA00008951F93CF93DF93E0914C29F0914D2995
:10BBB000908180914E29809589238083E09151293D
:10BBC000F0915229808190914E29892B80838FEBAF
:10BBD00093E00E949A5D1FB7F894E0915129F0918B
:10BBE0005229908180914E2980958923808383E812
:10BBF00090E00E949A5DE0914F29F0915029D08108
:10BC0000C0914E291FBF78948BE393E00E949A5D08
:10BC1000E0914F29F0915029908180914E299823ED
:10BC200019F08D2F8C2301C081E0DF91CF911F91FE
:10BC30000895509352294093512970934D29609350
:10BC40004C299093502980934F2981E001C0880F9F
:10BC50002A95EAF780934E290C94D15DCF93DF9318
:10BC6000C82FDFB7F894E0915129F09152298081D3
:10BC700090914E29892B808383E090E00E949A5D09
:10BC8000CC2351F0E0915129F0915229808190917B
:10BC90004E2990959823908387E190E00E949A5DC9
:10BCA000E0914F29F0915029808190914E2989236C
:10BCB00009F4C0E089E590E00E949A5DE091512985
:10BCC000F0915229808190914E29909598239083EC
:10BCD000DFBF8BE390E00E949A5D8C2FDF91CF91C4
:10BCE0000895CF93DF93C82FD8E08C2F81700E94E6
:10BCF0002E5EC6958111C068D150B9F78C2FDF91A7
:10BD0000CF9108958FEF0C94715EDF92EF92FF92C6
:10BD10000F931F93CF93DF93E82EEB010E94D15D29
:10BD200081112FC080EF0E94715EF12C10E488EF2A
:10BD3000D82ED10E81E00E942E5E082F81E00E9455
:10BD40002E5E882319F0002361F01DC0011109C087
:10BD50001E1528F0888180FF04C0E11611F0F12E35
:10BD600001E0802F0E942E5E9881969501119068C7
:10BD7000988311501D11DECF21961111D8CF8F2D30
:10BD800003C08FEF01C08EEFDF91CF911F910F9114
:10BD9000FF90EF90DF900895FF920F931F93CF9342
:10BDA000DF93F82EEB010E94D15D209769F085E5C5
:10BDB0000E94715E8E01085F1F4F89910E94715E23
:10BDC000C017D107D1F703C08CEC0E94715E8F2D94
:10BDD000DF91CF911F910F91FF900C94715E0F93A3
:10BDE0001F93CF93DF93DB01EC9111969C911197F8
:10BDF000F0E0F92B803181F4BF016E7FE3E0660F44
:10BE0000771FEA95E1F716969C911697ECE0F0E023
:10BE1000E91BF109E60FF71FF7FF07C091E0EA0100
:10BE20009883F195E195F10902C0EA011882883200
:10BE300079F414968C91982F9076903649F086FF7D
:10BE400002C0EE7F05C085FF02C0EC7F01C0E87F25
:10BE5000CF0144E0969587954A95E1F7D9018C93F7
:10BE6000EF70E801E88380E0DF91CF911F910F919F
:10BE700008950F931F93CF93DF93EC018B01B801CB
:10BE800088810E94855E888381508D3F30F4F8015F
:10BE90008081883211F0803191F7DF91CF911F912D
:10BEA0000F910895CF93DF93EC010E94D15DBE0105
:10BEB00084EB0E94CC5E81E00E942E5EC82F0E941F
:10BEC000D15D81E0C11101C080E0DF91CF91089583
:10BED0001F93CF93DF9300D0CDB7DEB7182F6983C0
:10BEE0007A830E94D15D0E94A05D69817A81882356
:10BEF00041F084E40E94CC5E113029F00E94A95DDB
:10BF000002C082E001C080E00F900F90DF91CF91DE
:10BF10001F9108954F925F926F927F928F929F929E
:10BF2000AF92BF92CF92DF92EF92FF920F931F9347
:10BF3000CF93DF93CDB7DEB729970FB6F894DEBF66
:10BF40000FBECDBF6C015B014A0189010E94D15D2A
:10BF5000B6018EEB0E94CC5ECE0101967C013E01C3
:10BF60009AE0690E711C27010E94825EF70181939D
:10BF70007F01E615F705C1F769E070E0C2010E9494
:10BF80002579811109C09401A501B201F6018081D2
:10BF90000E94EF5E80E001C083E029960FB6F8941E
:10BFA000DEBF0FBECDBFDF91CF911F910F91FF90EC
:10BFB000EF90DF90CF90BF90AF909F908F907F9049
:10BFC0006F905F904F9008955F926F927F928F92E3
:10BFD0009F92AF92BF92CF92DF92EF92FF920F9318
:10BFE0001F93CF93DF93CDB7DEB729970FB6F894A1
:10BFF000DEBF0FBECDBF582E6B015A01890160E034
:10C0000070E08EEB0E94CC5ECE0101967C014E0169
:10C010009AE0890E911C37010E94825EF70181939C
:10C020007F01E815F905C1F769E070E0C3010E94DE
:10C030002579811108C09501A601B301852D0E94C3
:10C04000EF5E80E001C083E029960FB6F894DEBF72
:10C050000FBECDBFDF91CF911F910F91FF90EF9059
:10C06000DF90CF90BF90AF909F908F907F906F9018
:10C070005F9008950F931F93CF93DF93CDB7DEB7F3
:10C0800028970FB6F894DEBF0FBECDBF182F062F2E
:10C0900098E0ECE0F3E0DE01119601900D929A95A4
:10C0A000E1F7242F332727FD309541E752E0249F05
:10C0B000C001259F900D349F900D112464E670E01F
:10C0C0000E94378DCB0144E6049F800D911D112401
:10C0D000FE013196AE01475F5F4F619170E0261718
:10C0E000370711F4019603C0E417F507B1F71123E0
:10C0F00019F091958195910928960FB6F894DEBFB5
:10C100000FBECDBFDF91CF911F910F910895EF9298
:10C11000FF920F931F93CF93DF93CDB7DEB72B978B
:10C120000FB6F894DEBF0FBECDBFF82EE92E682FF4
:10C13000792F88E08F0D0E94685F882319F084E3CF
:10C1400091E243C066E471E48FE090E00E94F26007
:10C150008E01075F1F4F9801AE01465F5F4FBE0122
:10C16000655F7F4F8F2D9E2D0E948A5F8111E7CFE3
:10C1700088E0ECE0F3E0DE01119601900D928A95E3
:10C18000E1F7498521E732E0429FC001439F900DCE
:10C19000112464E670E00E94378D8A8594E6899FB9
:10C1A000600D711D1124FE0131968191481303C069
:10C1B0006F5F7F4F03C0E017F107B9F78B858823C6
:10C1C00019F0719561957109CB012B960FB6F89412
:10C1D000DEBF0FBECDBFDF91CF911F910F91FF90BA
:10C1E000EF900895DC01CB0181159105A105B10502
:10C1F00029F081509040A040B040D9F708959B01AC
:10C20000AC011092B90060E072E18AE790E00E9410
:10C210004B8D205131094109510956954795379564
:10C2200027952093B800089594EA9093BC0040EAC3
:10C2300056E861E070E09091BC0097FD0BC0415062
:10C24000510961097109411551056105710599F798
:10C2500081E008959091B900987F983011F0903165
:10C26000B9F78093BB0084E88093BC0080EA96E82D
:10C27000A1E0B0E02091BC0027FD08C00197A10912
:10C28000B1090097A105B105A9F7E2CF8091B900E6
:10C29000887F883111F08034D9F680E0089524EA4F
:10C2A00034E844E92093BC009091BC0097FFFCCF98
:10C2B0009091B900987F983011F0903199F7809360
:10C2C000BB003093BC009091BC0097FFFCCF9091D5
:10C2D000B900987F903211F0983539F44093BC0042
:10C2E0009091BC0094FDFCCFDDCF08950C941461B7
:10C2F00084E98093BC008091BC0084FDFCCF08954C
:10C300008093BB0084E88093BC008091BC0087FFD1
:10C31000FCCF9091B900987F81E0983209F480E0D9
:10C32000089584EC8093BC008091BC0087FFFCCF13
:10C330008091BB00089584E88093BC008091BC008C
:10C3400087FFFCCF8091BB000895E0E1DC01FD9107
:10C35000CD01F0933F01E150C9F780913C018F7D01
:10C3600080933C0180913C01877F80933C01FB01DD
:10C3700080E1919190933E018150D9F780913C01E9
:10C38000806880933C0180913D0180FFFCCF40514B
:10C39000510980913C01806280933C0180913C0175
:10C3A000877F80933C01141615069CF4FB0180E105
:10C3B000919190933E018150D9F780913C01806822
:10C3C00080933C0180913D0180FFFCCF4051510999
:10C3D000EACFF90180E190913E0191938150D9F724
:10C3E00081E090E008950F931F93CF93DF93EC01CA
:10C3F0008CE70E944F618CE70E9480618E01005F94
:10C400001F4F89910E948061C017D107D1F7DF913A
:10C41000CF911F910F910C947861813019F440E015
:10C4200050E002C040EC50E060E070E08CE790E04B
:10C430000C94BF11813019F44EE050E002C048E086
:10C4400050E060E070E08CE790E00C94BF1141E0B8
:10C4500050E060E070E08CE790E00E94BF116AE677
:10C460007AE080E090E00C94F26048E350E060E015
:10C4700070E08CE790E00E94BF1149E350E060E07B
:10C4800070E08CE790E00E94BF1144E150E060E072
:10C4900070E08CE790E00E94BF1148E750E060E058
:10C4A00070E08CE790E00E94BF114EE550E060E044
:10C4B00070E08CE790E00E94BF114DE650E060E034
:10C4C00070E08CE790E00E94BF116CE17AE186E0B9
:10C4D00090E00E94F2604CE050E060E070E08CE799
:10C4E00090E00E94BF1141E050E060E070E08CE716
:10C4F00090E00E94BF1146E050E060E070E08CE701
:10C5000090E00E94BF116AE67AE080E090E00C942F
:10C51000F260CF93DF93CDB7DEB7A2970FB6F89452
:10C52000DEBF0FBECDBF81E1E0E4F9E0DE0152964F
:10C5300001900D928A95E1F781E1E1E5F9E0DE01F4
:10C54000119601900D928A95E1F70E943562CE0115
:10C5500042960E94F36182E00E940D626AE67AE0F0
:10C5600080E090E00E94F260CE0101960E94F361AB
:10C5700060E17EEA88E290E00E94F26080E00E9442
:10C580001A6260E17EEA88E290E00E94F2604EE08A
:10C5900050E060E070E08CE790E00E94BF11A2964E
:10C5A0000FB6F894DEBF0FBECDBFDF91CF910895D7
:10C5B000CF92DF92EF92FF920F931F93CF93DF936F
:10C5C00000D01F92CDB7DEB7F82E042F122F2130E6
:10C5D00031F0223031F0243031F0283031F090E069
:10C5E00005C091E003C092E001C093E00C3059F027
:10C5F0000E3011F4946007C0003111F4986003C04C
:10C60000023109F49C60613059F0623011F490629B
:10C6100007C0633011F4906403C0643009F490667D
:10C620009068692F70E023E030E0AE014F5F5F4F0C
:10C630008F2D90E00E94D61169E07AE180E090E0D1
:10C640000E94F2608F2D8160F82E0E9414610E947A
:10C65000916189830E9491618A83023119F40E9459
:10C6600091618B830E94916187FDF1CF0E949B6154
:10C670000E94786169E07AE180E090E00E94F260D7
:10C680008F2D0E9414610E94916189830E949161A3
:10C690008A83023119F40E949B618B830E949B6103
:10C6A0000E94786139812A81023149F5832F90E017
:10C6B000A0E0B0E04B817727662731FF0EC030E065
:10C6C000322F2227620F731F811D911D640F711D70
:10C6D000811D911D8C6F9F6F0BC030E0322F222780
:10C6E000620F731F811D911D640F711D811D911DAE
:10C6F0000E94718A20E83FEF4FEF57E420C0632F7C
:10C7000070E0762F6627620F711D882777FD809570
:10C71000982F0E94718A0C3029F420E030EE4FEF00
:10C7200054E40DC00E3029F420E038EF4FEF55E40B
:10C7300006C0003131F420E03EEF4FEF56E40E9496
:10C74000D2892FE632E143E050E40E94538C6B0122
:10C750007C01612F70E080E090E00E94718A9B0173
:10C76000AC01C701B6010E94D2890F900F900F90C3
:10C77000DF91CF911F910F91FF90EF90DF90CF90BD
:10C780000895E6E4F1E080812081908130818295F6
:10C7900086958695837022952F70822B832B929598
:10C7A0009F70892B08950F931F93CF93DF9300D031
:10C7B000CDB7DEB746E06CE080E00E94036789E118
:10C7C0008093C4001092C50082E08093C00080E096
:10C7D0000E9490670E942F6684B784B784B784B79D
:10C7E00084B7E3EDF1E322E432E4318320833A9627
:10C7F0008DB79EB70A97E817F907B8F382E699E074
:10C800009F938F9381E391E19F938F930E94149460
:10C810000E9468750E94235560E070E086E892E00F
:10C820000E94CB550E94FF58E0911403F09115032C
:10C8300009950E94C16390E00E94A475CE01019603
:10C840000E9464650F900F900F900F90882341F025
:10C8500081E191E19F938F930E9414940F900F9028
:10C86000CE0101960E9492530E9472658C010E9433
:10C870006E65AE014F5F5F4FB8010E945A6A0E9419
:10C88000DE640E943B6A0E9476650E94946B84E09D
:10C8900091E19F938F930E9414948A811F928F93AA
:10C8A00000E011E11F930F930E94149489811F925D
:10C8B0008F931F930F930E9414948EEF90E19F9398
:10C8C0008F930E9414940E94A875E0915103F091F7
:10C8D00052030995E0914303F09144030995E091D7
:10C8E0002A03F0912B0309950E949B6B182F0E943D
:10C8F000386A1F921F931F928F93809150038F93DA
:10C9000080914F038F93809142038F9380914103D5
:10C910008F9383EE90E19F938F930E941494E09104
:10C920005B03F0915C030FB6F894DEBF0FBECDBF82
:10C93000309791F00995BC0180E890E00E94238D2A
:10C940007F936F9380ED90E19F938F930E94149457
:10C950000F900F900F900F908EEC90E19F938F931C
:10C960000E94149460E070E08CED92E00E94CB5540
:10C9700080EF92E00E94787486EC90E19F938F9311
:10C980000E9414940F900F900F900F900F900F90A3
:10C99000DF91CF911F910F9108957F936F939F9394
:10C9A0008F9380EC90E19F938F930E9414940F904B
:10C9B0000F900F900F900F900F9008951F93CF93AB
:10C9C000DF93CDB7DEB7A0970FB6F894DEBF0FBEEA
:10C9D000CDBF8DE590E00E948095182F282F35EF70
:10C9E000380F303108F0982F9095291709F461C05D
:10C9F0008CE491E19F938F930E941494E1E9F1E11B
:10CA00000F900F90DE01119684918D93319681E104
:10CA1000E939F807C9F7F89448E050E069E770E0B1
:10CA2000CE0101960E948695E3E8F1E1DE011196C0
:10CA300084918D93319681E1E139F807C9F74EE091
:10CA400050E06BE670E0CE0101960E948695E9E722
:10CA5000F1E1DE01119684918D93319681E1E33805
:10CA6000F807C9F74AE050E061E670E0CE010196B0
:10CA70000E9486956DEC7BEA8BE590E00E949E9586
:10CA800060E070E089E590E00E949E9560E088E5B6
:10CA900090E00E94909560E070E08FE590E00E9449
:10CAA0009E951AE16AE175EE8DE590E00E949E95F3
:10CAB0007894812FA0960FB6F894DEBF0FBECDBF3D
:10CAC000DF91CF911F910895F89442E050E069E71B
:10CAD00070E00E946895789480E008958BE590E07E
:10CAE0000C94809589E590E00C94809588E590E021
:10CAF0000C94789540916129509162296091632945
:10CB00007091642990E0A0E0B0E0480F591F6A1FBF
:10CB10007B1F40936129509362296093632970932E
:10CB2000642940915D2950915E2960915F2970913F
:10CB30006029480F591F6A1F7B1F40935D2950933E
:10CB40005E2960935F29709360292091012B222335
:10CB5000A1F04091592950915A2960915B29709117
:10CB60005C29480F591F6A1F7B1F40935929509316
:10CB70005A2960935B2970935C2908951F920F9244
:10CB80000FB60F9211240BB60F922F933F934F9332
:10CB90005F936F937F938F939F93AF93BF93EF9325
:10CBA000FF93809174139091751301969093751370
:10CBB00080937413809173138F5F80937313803805
:10CBC000A9F4109273138091612990916229A09128
:10CBD0006329B09164290196A11DB11D809361293B
:10CBE00090936229A0936329B09364298091012BCB
:10CBF0008823E1F0809172138F5F809372138038E5
:10CC0000A9F4109272138091592990915A29A091F8
:10CC10005B29B0915C290196A11DB11D8093592912
:10CC200090935A29A0935B29B0935C290E945B588A
:10CC3000892B11F00E946E57FF91EF91BF91AF9138
:10CC40009F918F917F916F915F914F913F912F9124
:10CC50000F900BBE0F900FBE0F901F901895F89479
:10CC60001092B60016BC83EF87BD82E084BD94E0CD
:10CC700095BD95B395BB80936E007894089580918F
:10CC8000741390917513209174133091751382175A
:10CC90009307A9F70895009751F022E330E00000D0
:10CCA0002150310921153105D1F70197F4CF0895AD
:10CCB0000F931F93CF93DF93EC010E943F668C018B
:10CCC0000E943F66801B910B8C179D07C8F3DF9174
:10CCD000CF911F910F91089508950F931F93609125
:10CCE0006129709162298091632990916429009152
:10CCF000612910916229209163293091642960177C
:10CD000071078207930759F71F910F9108951F929A
:10CD10000F920FB60F9211241092B2020F900FBE15
:10CD20000F901F9018951F920F920FB60F9211241B
:10CD30000BB60F922F933F934F935F936F937F9315
:10CD40008F939F93AF93BF93EF93FF93E091A802CC
:10CD5000F091A9028081E091B302F091B402309782
:10CD600009F00995FF91EF91BF91AF919F918F913C
:10CD70007F916F915F914F913F912F910F900BBEDB
:10CD80000F900FBE0F901F9018951F920F920FB625
:10CD90000F9211241092BF020F900FBE0F901F90A0
:10CDA00018951F920F920FB60F9211240BB60F9287
:10CDB0002F933F934F935F936F937F938F939F93A3
:10CDC000AF93BF93EF93FF93E091B502F091B6025A
:10CDD0008081E091C002F091C102309709F009957D
:10CDE000FF91EF91BF91AF919F918F917F916F9143
:10CDF0005F914F913F912F910F900BBE0F900FBEFF
:10CE00000F901F9018959DE0899FF0011124E8551F
:10CE1000FD4FA281B3811C92A481B5816C93A68140
:10CE2000B78188ED8C93A085B1854C9312861486CA
:10CE3000138608959DE0899FF0011124E855FD4F68
:10CE400081E08287A081B1816C933A9680818111C3
:10CE5000FDCF08951F93CF93DF93182FEB01FE01B1
:10CE60008491882339F0FE016491812F0E941A6712
:10CE70002196F5CFDF91CF911F9108951F93CF9306
:10CE8000DF93182FEB018881882369F08A3021F421
:10CE90006DE0812F0E941A6769916D30A1F3812F97
:10CEA0000E941A67F0CFDF91CF911F910895CF9321
:10CEB000DF93CDB7DEB79E01285F3F4F4E815F8184
:10CEC00060E470E086E793E10E94D19466E773E145
:10CED0008D810E943E67DF91CF910895CF93C82F37
:10CEE0008A3031F46DE08091B6130E941A6702C057
:10CEF0008D3029F06C2F8091B6130E941A6780E064
:10CF000090E0CF9108959DE0899FF0011124E855AC
:10CF1000FD4F748763870895682F80E00C941A672B
:10CF20008093B6138AE992E09093CE318093CD310D
:10CF3000089584B7877F84BF88E10FB6F894809303
:10CF40006000109260000FBE08952FE088E190E02D
:10CF50000FB6F894A895809360000FBE20936000F0
:10CF60000895A895089588E10FB6F894809360001D
:10CF7000109260000FBE0895F89428E088E190E0D8
:10CF80000FB6F894A895809360000FBE20936000C0
:10CF9000FFCF80916C2980916C2990E0089540E04A
:10CFA0006FE181E491E00C94306DE9E3F1E0808180
:10CFB00080818D7F80838DE090E00197F1F723E001
:10CFC00040E06FE182E491E00E943A6D83E090E0FE
:10CFD0000197F1F708959091390191FD0AC0282F2A
:10CFE000803108F02FE040E06FE085E491E00C94A0
:10CFF0003A6D08958091390181FD0EC040E06FE1E6
:10D0000081E491E00E94306D282F2F7E81E090E036
:10D01000213021F080E0089580E090E00895809133
:10D02000390181FD10C040E06FE181E491E00E9490
:10D03000306D8F3131F0982F9F7E915081E092308A
:10D0400018F480E0089581E008950E940F68882315
:10D05000E1F30895CF93DF93C82F0E9425680E94C3
:10D06000CF67D82FC81789F1C83019F40E94D56747
:10D0700025C0C93121F4863189F429E005C0C631C3
:10D0800069F4893159F426E040E06FE182E491E0EF
:10D090000E943A6DE3E0F0E03197F1F72C2F40E089
:10D0A0006FE182E491E00E943A6DD83019F4E9E62C
:10D0B000F1E002C0E3E0F0E03197F1F70E94CF67C2
:10D0C0008C1719F083E490E002C080E490E0DF91D7
:10D0D000CF9108950E9425681092012B0E94D56778
:10D0E000809139018260809339018091842B88235B
:10D0F000D9F180919400909195004091952B509199
:10D10000962B84179507A0F48091612B9091622B48
:10D11000A091632BB091642B8C57914EAF4FBF4FB2
:10D120008093612B9093622BA093632BB093642B1D
:10D130002091940030919500241B350B8091612B38
:10D140009091622BA091632BB091642B820F931F5F
:10D15000A11DB11D8093612B9093622BA093632B33
:10D16000B093642B1092842B8091862B8823D9F165
:10D1700080919400909195004091992B50919A2B19
:10D1800084179507A0F48091692B90916A2BA09148
:10D190006B2BB0916C2B8C57914EAF4FBF4F809340
:10D1A000692B90936A2BA0936B2BB0936C2B2091DF
:10D1B000940030919500241B350B8091692B909140
:10D1C0006A2BA0916B2BB0916C2B820F931FA11D2A
:10D1D000B11D8093692B90936A2BA0936B2BB09316
:10D1E0006C2B1092862B08958091012B882381F05F
:10D1F00080913A14811104C00E940F68811106C009
:10D2000081E08093381481E090E008950E946A687C
:10D2100080E090E008958091940090919500909323
:10D220009A2B8093992B21E02093862B80913901B2
:10D2300081FD08C08091390181FD1AC086E10E94FC
:10D240002A6816C02093002B80919400909195003D
:10D250009093962B8093952B2093842B809139016A
:10D260008D7F809339018091002B8111FCCFE2CF1B
:10D2700081E08093012B08958091012B81110AC0D8
:10D2800080913A14882321F081E08093391402C000
:10D290000E940B6981E090E008951F93CF93DF9384
:10D2A0001F92CDB7DEB78FB7898380913A14811171
:10D2B00026C0F8948091012B882351F08091390188
:10D2C00081FD1BC00E940F688823B9F080E003C075
:10D2D0000E943C6981E02091470191E02E3008F0E6
:10D2E00090E0192F119581110E94F468107429F0B3
:10D2F00089818FBF81E090E004C089818FBF80E089
:10D3000090E00F90DF91CF911F9108958091391493
:10D31000882321F00E940B691092391480913814EF
:10D32000882321F00E946A681092381410923A14EF
:10D3300008950F931F93AB0121E020933A140091BD
:10D34000452B1091462B2091472B3091482B0F5F96
:10D350001F4F2F4F3F4F0093452B1093462B209389
:10D36000472B3093482B22E0260F27FF0CC08091DB
:10D37000FE2A9091FF2A01969093FF2A8093FE2A1D
:10D380000FEF1FEF07C0BC0187EB93E10E944D93A5
:10D3900000E010E00E948669C8011F910F91089576
:10D3A00080933C1408950E94CF67823011F082313F
:10D3B00011F480E0089581E0089508958FEF80933F
:10D3C0004E0122E044E060EF8CE691E00E943A6D6D
:10D3D00025E041E06EE08CE290E00E943A6D80E84A
:10D3E00080936F018091460180936D0121E045E0BB
:10D3F00060E284E491E00C943A6D8DEF93E0019744
:10D40000F1F70E94266D109275291092F72910925B
:10D41000792A1092742910927329E9E3F1E080814E
:10D420008E7F808380818D7F80838DE090E0019767
:10D43000F1F780818160808323E040E06FE182E446
:10D4400091E00E943A6D8DEF93E00197F1F78091A2
:10D450005D0180915E010E94DE6960E070E082EC17
:10D4600092E00E94CB550E940B6981E090E0089504
:10D4700080913B140895CF93DF931F92CDB7DEB711
:10D4800089830E942568898180933B14282F40E07E
:10D490006FE188E491E00F90DF91CF910C943A6DA9
:10D4A0000E943B6A8091390181FD03C086E00C94A3
:10D4B0002A680895FA018093620190936301609352
:10D4C0006001709361013097C1F0808180936B019E
:10D4D000818180936A018281809369018381809335
:10D4E00068018481809367018581809366018681CC
:10D4F00080936501878180936401089582EC92E0B6
:10D500000E94EC5581E080936C2980916D29909167
:10D510006E29019690936E2980936D2981E090E0A9
:10D5200008958091742992E8899FF0011124EB58A5
:10D53000F64D10828F5F833018F48093742902C0F7
:10D5400010927429E091742982E8E89FF001112477
:10D55000EB58F64D808181110C947E6A10926C29F3
:10D5600008951F93CF93DF932091742912E8129F9F
:10D5700090011124D901AB58B64D4C91411103C013
:10D580000E94916A93C05091390151FD8FC0509112
:10D59000012B552309F48AC047FF16C00E94916AE7
:10D5A0008091352B9091362BA091372BB091382B51
:10D5B0000196A11DB11D8093352B9093362BA0931E
:10D5C000372BB093382B72C04330B0F40E94916A6D
:10D5D0008091312B9091322BA091332BB091342B31
:10D5E0000196A11DB11D8093312B9093322BA093F6
:10D5F000332BB093342B5AC050E0EA0122976C17BA
:10D600007D07B0F40E94916A80912D2B90912E2B72
:10D61000A0912F2BB091302B0196A11DB11D8093AD
:10D620002D2B90932E2BA0932F2BB093302B3EC0FD
:10D63000B9016A58764D0E944D93E09174291E9F5E
:10D64000F0011124EB50F64D8081809365290E94F2
:10D65000916A809147018093662990916B29992363
:10D6600011F0891710F480936B296091662970E09E
:10D6700084E00E94765D6091652970E083E00E94FD
:10D68000765D4091492B50914A2B60914B2B7091C4
:10D690004C2B4F5F5F4F6F4F7F4F4093492B509301
:10D6A0004A2B60934B2B70934C2B02C0C0E0D0E010
:10D6B000CE01DF91CF911F910895CF93DF93EC01BD
:10D6C000888199810097E9F08730954021F019828F
:10D6D000188283E026C06238C1F410926C290E943F
:10D6E000FD5C0E94645C60E870E00E94B16A1816FC
:10D6F00019066CF40E945F5CE0915503F0915603AB
:10D70000099587E095E09983888381E00AC080913C
:10D71000692990916A29019690936A2980936929D1
:10D72000F0CFDF91CF91089591E090933A140E9449
:10D73000EB670C9486698091390181FD06C040E059
:10D740006FE085E491E00C94306D80E108950F93D3
:10D750001F93CF93DF93182F21E020933A14009169
:10D76000012B8091390181FF16C080919400909126
:10D7700095009093962B8093952B2093842B209348
:10D78000002B809139018D7F809339018091002B8E
:10D790008111FCCF00E00E9425688091012B882335
:10D7A00009F43FC08091862B8823D9F180919400A1
:10D7B00090919500E091992BF0919A2B8E179F07ED
:10D7C000A0F44091692B50916A2B60916B2B709162
:10D7D0006C2B4C57514E6F4F7F4F4093692B50939A
:10D7E0006A2B60936B2B70936C2B2091940030917B
:10D7F00095002E1B3F0B4091692B50916A2B609135
:10D800006B2B70916C2B420F531F611D711D409348
:10D81000692B50936A2B60936B2B70936C2B109237
:10D82000862B8091390181FD03C089E10E942A681D
:10D8300086E00E94815D892B51F00E949B6BC82F6E
:10D8400086E00E94815D81500E94EB6702C0C0E0CB
:10D85000D0E020919400309195003093982B209344
:10D86000972B81E08093852BF89480913901826019
:10D8700080933901809139018D7F8093390162E075
:10D88000610F87EB93E10E94696D78942091FB2AE8
:10D890003091FC2A2F5F3F4F3093FC2A2093FB2AC4
:10D8A0000E94256845E060EE82E491E00E94306DC0
:10D8B000182F86E00E94815D892B19F08C2F0E9421
:10D8C000EB67002319F00E940B6902C00E946A688E
:10D8D0008091852B8823D9F18091940090919500B7
:10D8E000E091972BF091982B8E179F07A0F4409111
:10D8F000652B5091662B6091672B7091682B4C576C
:10D90000514E6F4F7F4F4093652B5093662B609322
:10D91000672B7093682B20919400309195002E1BFB
:10D920003F0B4091652B5091662B6091672B709156
:10D93000682B420F531F611D711D4093652B50933F
:10D94000662B6093672B7093682B1092852B8091C8
:10D95000012B882361F02091940030919500309341
:10D960009A2B2093992B81E08093862B07C023E08C
:10D9700040E06FE182E491E00E943A6D0E94866986
:10D980001130E9F01330A9F480913D2B90913E2B9A
:10D99000A0913F2BB091402B0196A11DB11D80930A
:10D9A0003D2B90933E2BA0933F2BB093402B12E046
:10D9B00009C0153031F0173029F411E003C010E030
:10D9C00001C013E0812F90E0DF91CF911F910F9163
:10D9D0000895CF93DF93EB010E949969009729F492
:10D9E000CE010E94A76B009751F02091FE2A309142
:10D9F000FF2A2F5F3F4F3093FF2A2093FE2ADF91AB
:10DA0000CF910895CF93DF938091012B811104C0B2
:10DA10000E943C69D1E001C0D0E00E94CF6786310E
:10DA200011F0813119F4C091470109C040E06FE164
:10DA300086E491E00E94306DC82FCC0FC80FD11141
:10DA40000E94F4688C2FDF91CF91089510923E14BC
:10DA500010923D14EFE6F0E08081806280830895AB
:10DA6000FC018081862390E002C0959587954A95B8
:10DA7000E2F70895F894FC015081362F3095532336
:10DA8000042E01C0220F0A94EAF72623522B50835A
:10DA90007894089540917B01FC014193A0E8B1E0A6
:10DAA00050E8540F9D012F5F3F4F6C9161935217C7
:10DAB00011F0D901F7CF4150E42FF0E0E058FE4FCC
:10DAC0002181FC01E058FF4F2083319621E0208323
:10DAD000089560938001E1E8F1E061589F012F5FB4
:10DAE0003F4FDC014D91CD014083621711F0F901E8
:10DAF000F5CF08951F920F920FB60F9211240BB617
:10DB00000F922F933F934F935F936F937F938F93D6
:10DB10009F93AF93BF93EF93FF93809147018093BF
:10DB200066298091732922E8829FC00111248B58B5
:10DB3000964D0E944A6D809173298F5F833018F44F
:10DB40008093732902C0109273290E947E6AFF910C
:10DB5000EF91BF91AF919F918F917F916F915F9165
:10DB60004F913F912F910F900BBE0F900FBE0F90D2
:10DB70001F9018951F920F920FB60F9211240F90BD
:10DB80000FBE0F901F9018951F920F920FB60F9215
:10DB900011240F900FBE0F901F9018951F920F9297
:10DBA0000FB60F9211240F900FBE0F901F90189573
:10DBB0001F920F920FB60F9211241092002B0F900C
:10DBC0000FBE0F901F9018951F920F920FB60F92D5
:10DBD00011241092002B0F900FBE0F901F901895DC
:10DBE0001F920F920FB60F9211248F9381E08093B2
:10DBF0006C298F910F900FBE0F901F9018951F9258
:10DC00000F920FB60F9211241092002B0F900FBE9F
:10DC10000F901F9018951F920F920FB60F9211241C
:10DC20008F939F9380913D1490913E140196909311
:10DC30003E1480933D149F918F910F900FBE0F90D3
:10DC40001F901895CF92DF92EF92FF920F931F9340
:10DC5000CF93DF937C018B016A018FE394E10E94F3
:10DC60008B56EC01009751F0EC81FD81309711F05B
:10DC7000C8010995CE010E943357F3CFA601B80120
:10DC8000C701DF91CF911F910F91FF90EF90DF902F
:10DC9000CF900C9415540F931F93CF93DF9300D024
:10DCA000CDB7DEB78091092B90910A2BA0910B2B59
:10DCB000B0910C2B0196A11DB11D8093092B90935F
:10DCC0000A2BA0930B2BB0930C2B0E94B5708C01E8
:10DCD0008FE394E10E948B56009779F0DC01129655
:10DCE000ED91FC911397309729F089839A830995D8
:10DCF0009A8189810E943357EFCF0115110549F0B0
:10DD0000C8010F900F90DF91CF911F910F910C944C
:10DD10000C540F900F90DF91CF911F910F910895A8
:10DD20000E94A8750E94FD5C0E94DC6E81E493E075
:10DD30009093042B8093032B0E94B3702FEF31E05C
:10DD400040E05EE160E074E082E090E00C947C7082
:10DD5000BC018FE394E10C94EB56BC018FE394E19A
:10DD60000C94D056CF93DF93EC014091052B50914A
:10DD7000062B6091072B7091082B4F5F5F4F6F4F01
:10DD80007F4F4093052B5093062B6093072B709386
:10DD9000082B0E94C870009761F00E947D5CE091A2
:10DDA0004503F0914603BE0182E29EE6099581E0BB
:10DDB00090E0DF91CF91089585E494E10C9487562B
:10DDC0000F93CF93DF93EC017B836A8318865F8385
:10DDD0004E83BC0185E494E10E94EB56E09141142E
:10DDE000F0914214309749F04C815D8101E020E0D0
:10DDF00030E068858A819B810995DF91CF910F91F1
:10DE00000895BC0185E494E10C94D0560F93DC0195
:10DE100018961C921897E0914114F0914214309793
:10DE200059F000E020E030E040E050E060E0129681
:10DE30008D919C91139709950F9108950F93DC0193
:10DE4000AB0114962D913C91159781E018968C9317
:10DE5000189715967C936E931497E0914114F09166
:10DE60004214309739F000E061E012968D919C9158
:10DE7000139709950F9108950F93DC01E0914114D8
:10DE8000F0914214309771F014964D915C91159772
:10DE900001E09A0118966C91189712968D919C91B9
:10DEA000139709950F910895E0914314F09144144C
:10DEB000309709F009940895909344148093431483
:10DEC00008959093421480934114089585E494E159
:10DED0000C948B56EF92FF920F931F93CF93DF9387
:10DEE0008C01EB017A0185E494E10E948B56009746
:10DEF000D9F0DC0112962D913C9113972C173D0718
:10DF000081F41696ED91FC911797309769F097017F
:10DF1000AE01B801DF91CF911F910F91FF90EF906B
:10DF200009940E943357E3CFDF91CF911F910F9156
:10DF3000FF90EF9008950895CF93DF93C8E7D4E161
:10DF40006881798120E030E04BEB5FE682E694E186
:10DF50000E940B590E94A675688179810E94238DC9
:10DF600020E030E04FEC5FE6BC0182E594E1DF9118
:10DF7000CF910C940B598091781490917914209141
:10DF8000761430917714880F991F2817390708F4F1
:10DF9000C90190937914809378140C949C6FCF935B
:10DFA000DF930E94FD5C0E94645CEC011982188280
:10DFB0000E94666F28813981009719F1FC01408524
:10DFC0004423F9F0FC0142815381F901EE0FFF1F58
:10DFD000EE0FFF1FEC0FFD1F53834283FC014481B2
:10DFE00055812F5F3F4FF901EE0FFF1FEE0FFF1F0F
:10DFF000EC0FFD1F51834083398328830E943357E0
:10E00000D9CFC901880F991F880F991F02960E94C6
:10E010005F5C88819981892B31F087E494E1DF91FD
:10E02000CF910C94E353DF91CF910895AF92BF92BB
:10E03000CF92DF92EF92FF920F931F93CF93DF93D4
:10E0400000D0CDB7DEB76B010E94645CFC0100819B
:10E0500011811A8309830C30110518F4E12CF12C7D
:10E060000DC01F930F9380E899E09F938F930E94B8
:10E0700002940F900F900F900F9021C0E016F106C0
:10E08000F1F00E94645CF701EE0FFF1FEE0FFF1F1F
:10E09000E80FF91FA280B3800E94645CFFEFEF1AC3
:10E0A000FF0AF701EE0FFF1FEE0FFF1FE80FF91F2A
:10E0B00040815181B501C6010E946A6FDFCF0F9088
:10E0C0000F90DF91CF911F910F91FF90EF90DF9014
:10E0D000CF90BF90AF9008950F93013059F4809185
:10E0E00072149091731490937914809378140F9113
:10E0F0000C949C6F0F910895EF92FF920F931F93D2
:10E10000CF93DF938B01EA0179014EE253E0BC012A
:10E1100087E494E10E94C753109373140093721420
:10E12000D0937514C0937414F0927714E09276141F
:10E130008CE690E7DF91CF911F910F91FF90EF90C8
:10E140000C94616F82E694E10E948F5982E594E11C
:10E150000E948F5987E494E10C94E15380917814E4
:10E160009091791408950C942154CF93DF93E0910A
:10E170003203F09133030995EC01009729F06A818D
:10E180007B8181E00E94765DCE01DF91CF91089581
:10E190000F931F93CF93DF93EC01E0913403F09141
:10E1A000350309958C016A817B8181E00E94765D4F
:10E1B00081E090E0012B11F480E090E0DF91CF91BD
:10E1C0001F910F910895E0913603F0913703099460
:10E1D00020E030E00296FC0132974081442331F088
:10E1E000FC0131974081240F311DF4CFC9010895FE
:10E1F000FC01208130E0322F22278181282B02C0B0
:10E20000220F331F6A95E2F7832F9927FA01E85C02
:10E21000FC4F208130E08223932328E030E0241B50
:10E22000350B02C0969587952A95E2F708956F926F
:10E230007F928F929F92AF92BF92CF92DF92EF9296
:10E24000FF920F931F93CF93DF938C01EB016A0131
:10E2500079012830310524F4A901B601CE014AC064
:10E26000590123E0B594A7942A95E1F7411551058A
:10E2700021F04801612C712C03C0D801FB0120C0A2
:10E2800048E050E0B601CE01860D971D0E94F8705F
:10E29000F40181934F01FFEF6F1A7F0A6A147B0428
:10E2A0007CF3C501B7FE02C080E090E0A701477093
:10E2B00055274115510511F1080F191FB60118C056
:10E2C000CF018C1B9D0B8A159B051CF481918D93AE
:10E2D000F7CFC501B7FE02C080E090E0A70147700C
:10E2E00055274115510551F0080F191F60E070E0E6
:10E2F0008C0F9D1F0E94F870F8018083DF91CF91F1
:10E300001F910F91FF90EF90DF90CF90BF90AF9053
:10E310009F908F907F906F9008958F929F92AF9271
:10E32000BF92CF92DF92EF92FF920F931F93CF9302
:10E33000DF9300D0CDB7DEB70E94645C8C0182E031
:10E3400090E00E94425C892B19F480E090E05DC06F
:10E35000F801818190E0982F88272081820F911DFC
:10E360000E9432547C01009781F30E94645C4C014E
:10E37000F7012681822F86958695869590E0422F1B
:10E38000477021E030E011F420E030E0820F931F6D
:10E390000E94425C892BC9F2F70104811581C12CCE
:10E3A000D12CF8018081882379F1F801A180B12C6A
:10E3B000B60133E0759567953A95E1F7A601477088
:10E3C0005527680D791D883168F09501CE010196B9
:10E3D0000E941771BE016F5F7F4FF80180810E941C
:10E3E0008A5D0DC01A8219829501CE0101960E94A4
:10E3F000177169817A81F80180810E94765DCA0C6B
:10E40000DB1C0E5F1F4FCDCFC7010F900F90DF9128
:10E41000CF911F910F91FF90EF90DF90CF90BF9021
:10E42000AF909F908F900895DC0150E0E0E1F0E024
:10E43000E61BF70BE21BF30B02C0440F551FEA95D6
:10E44000E2F78C91852B8C9311968C911197842BEC
:10E4500011968C9308956F927F928F929F92AF92B4
:10E46000BF92CF92DF92EF92FF920F931F93CF93C1
:10E47000DF938C016B01EA017901283031051CF42E
:10E480004881C8015CC0390153E0759467945A957E
:10E49000E1F76115710521F04E01A12CB12C03C0EB
:10E4A000D801FE0127C0F40141914F0128E030E07E
:10E4B000B601C8018A0D9B1D0E941472FFEFAF1AAE
:10E4C000BF0AA614B7047CF3C30177FE02C080E044
:10E4D00090E09701277033272115310509F43FC0DB
:10E4E000C80FD91F488150E0B601621B730B685FEB
:10E4F0007F4F1CC0CF018C1B9D0B861597051CF40C
:10E5000081918D93F7CFC30177FE02C080E090E048
:10E510009701277033272115310509F1C80FD91F3D
:10E52000488150E068E070E0621B730B02C05595B3
:10E5300047956A95E2F760E070E0800F911FDF91E8
:10E54000CF911F910F91FF90EF90DF90CF90BF90F0
:10E55000AF909F908F907F906F900C941472DF918A
:10E56000CF911F910F91FF90EF90DF90CF90BF90D0
:10E57000AF909F908F907F906F9008956F927F9251
:10E580008F929F92AF92BF92CF92DF92EF92FF92C3
:10E590000F931F93CF93DF9300D0CDB7DEB78C01DD
:10E5A000FC018681E82EE694E694E694F12C282F6F
:10E5B000277081E090E011F480E090E0E80EF91E11
:10E5C000C70102960E94C65C009709F445C00E94EC
:10E5D0006B5CF8012281FC012083F8012381FC019E
:10E5E00021830E946B5C02965C01A70160E070E0F1
:10E5F0000E945693F80104811581E12CF12CF80159
:10E600008081882339F1F8018180912C670163E0D2
:10E61000D594C7946A95E1F73701F7E06F22772424
:10E62000CA0CDB1C883128F00E94945D9401AC0177
:10E6300008C00E94815D9A8389839401AE014F5F77
:10E640005F4FB301C6010E942B72E80CF91C0E5FEC
:10E650001F4FD5CF81E090E00F900F90DF91CF91C9
:10E660001F910F91FF90EF90DF90CF90BF90AF90F0
:10E670009F908F907F906F900895E0915303F09159
:10E6800054030994E0912C03F0912D030994E09137
:10E690005703F09158030994E0915903F0915A03FC
:10E6A000099480E090E008950895E0912403F091AA
:10E6B0002503099480E090E008950F931F93CF9372
:10E6C000DF93CDB7DEB7E0970FB6F894DEBF0FBE8D
:10E6D000CDBF0E94B15C8C010E94645CAE014F5FB3
:10E6E0005F4F602F0E942D7B882309F446C088A9C4
:10E6F0009801281B3109C9010E94425C892BE9F16C
:10E700002E8121110CC0BE016A5E7F4F88E10E94FC
:10E710008A5DE0914703F091480309952EC08A85F0
:10E720009B858D3C3BEA930711F0019631F5223031
:10E7300019F088E090E002C082E090E001979C012F
:10E740002F5F3F4F12161306F4F6E1E0F0E0EC0FF6
:10E75000FD1FE80FF91F23852F3F81F3BE01645F82
:10E760007F4F89E10E948A5D89E10E94945D62E1A8
:10E7700079E20E948053892B31F6E0960FB6F89427
:10E78000DEBF0FBECDBFDF91CF911F910F910895D6
:10E79000AF92BF92CF92DF92EF92FF920F931F93AF
:10E7A000CF93DF93CDB7DEB7E0970FB6F894DEBF17
:10E7B0000FBECDBF8C016B01CE0101967C0180E3C1
:10E7C000F70111928A95E9F781E089838CE00E9434
:10E7D000815D8C831D821F8280917C1491E0980F53
:10E7E00090937C14898783E0B82EB8868DEC9BEAE1
:10E7F0009B878A8789E10E94945D60E073E00E94B4
:10E800008053892B31F082E08E838FEF8C878D8748
:10E8100009C089E10E94945DBC01CE010C960E9462
:10E820007753BE828DEC9BEA9D8B8C8B62E179E203
:10E83000CE0146960E9477530E94645C9FA78EA7E4
:10E840000E94B15C88ABC7010E94267AB82E90E086
:10E850000E94C65C892B31F10E946B5CBC014B2D80
:10E86000C7010E94447AE0901A03F0901B030E94B3
:10E87000BB5C5C010E946B5CB501F7010995011559
:10E88000110581F0009739F0019761F441E050E003
:10E8900064E070E004C041E050E060E070E0C60178
:10E8A000F8010995E0960FB6F894DEBF0FBECDBF14
:10E8B000DF91CF911F910F91FF90EF90DF90CF905C
:10E8C000BF90AF9008950E94A67580937C14E0914C
:10E8D0002403F09125030994892B29F0E091240366
:10E8E000F091250304C0E0912603F09127030994D9
:10E8F000CF93DF93EC0189919991009729F060E023
:10E9000070E00E94CB55F7CFDF91CF910895CF9360
:10E91000DF93EC0189919991009719F00E941D55A0
:10E92000F9CFDF91CF910895CF93DF93EC017B83F3
:10E930006A830E943F6699838883DF91CF9108950F
:10E94000FC018081918122813381820F931F918309
:10E9500080830895CF93DF93EC010E943F669983F3
:10E960008883DF91CF910895CF93DF93EC010E94CC
:10E970003F6628813981821B930B9C012F5F3F4F9B
:10E9800081E090E04A815B814217530710F080E0FC
:10E9900090E0DF91CF910895CF93DF93FC01C28186
:10E9A000D38180819181C80FD91F0E943F669E014B
:10E9B000281B390BC901DF91CF910895CF93DF93C5
:10E9C000EBE8FBE2CDE4DBE2AFE7BBE211921192B0
:10E9D00019921992199219921D928BE2E33AF80753
:10E9E000A9F7DF91CF910895CF93DF93FC01E15810
:10E9F000F44D40819C01220F331F220F331F44230B
:10EA000001F1A0919400B0919500FC01EE0FFF1F61
:10EA1000E557F44D80819181AD01481B590BCA0126
:10EA2000E901C35BD44D488159816A817B81480FDC
:10EA3000591F611D711D488359836A837B83B1838C
:10EA4000A083F901E35BF44D608171818281938140
:10EA5000DF91CF91089560E070E0CB010895FC0153
:10EA6000EE0FFF1FEE0FFF1FE35BF44D408351835A
:10EA7000628373830895CF93DF932FE73BE2CDE466
:10EA8000DBE2EBE8FBE2D9018D919D018823B9F02F
:10EA9000409194005091950080819181BA01681B4A
:10EAA000790B88819981AA81BB81860F971FA11D4F
:10EAB000B11D88839983AA83BB83518340832496A5
:10EAC0003296BBE22B383B07F1F6DF91CF910895E8
:10EAD0000C94B5790F931F93FC01CB0140917D14E9
:10EAE00050917E1433832283158304837183608362
:10EAF000F0937E14E0937D14452B11F40E94CF799E
:10EB000080E090E01F910F91089580917D14909185
:10EB10007E140097C1F010927E1410927D14DC01D7
:10EB200014966D917C9115971296ED91FC91139727
:10EB30000995E0917D14F0917E14309721F0808149
:10EB400091810C94CF7908950C94E08F0C94DC8F14
:10EB500084ED92E00E9402568CEC92E00C940256F6
:10EB6000CF93DF930E94715C892BA9F08CEC92E02B
:10EB70000E942056EC01009721F10E94B15C99831C
:10EB800088830E94AC5C9B838A83CE0104960E949A
:10EB9000ED5B8CAB14C084ED92E00E942056EC013A
:10EBA000009779F002960E94FF5B99838883BE01EB
:10EBB0006E547F4FCE018E579F4F0E94545DCE0101
:10EBC00002C080E090E0DF91CF910895BC016E54C7
:10EBD0007F4F8E579F4F0C94545DCF93DF93EC0182
:10EBE000BC0184ED92E00E946A56BE01892B19F0A7
:10EBF00084ED92E009C08CEC92E00E946A56892B69
:10EC000039F0BE018CEC92E0DF91CF910C94455627
:10EC1000DF91CF9108950F931F93CF93DF93EC0172
:10EC2000BC0184ED92E00E946A56892B91F0FE01AE
:10EC300061917191CF010E94105DBE016E547F4FB2
:10EC4000CE018E579F4FDF91CF911F910F910C9462
:10EC5000655DBE018CEC92E00E946A56892BD1F072
:10EC60000E94FD5C688179818A819B810E94105D90
:10EC70008CA990E00E94C65C0CA910E00E946B5C1D
:10EC8000BE016C5F7F4FA801DF91CF911F910F9163
:10EC90000C944D93DF91CF911F910F910895CF93D5
:10ECA000DF93EC01BC0184ED92E00E946A56892B4F
:10ECB00019F0CE0102960CC0BE018CEC92E00E94CD
:10ECC0006A56892B19F08A819B8102C080E090E00E
:10ECD000DF91CF910895FC01808191810895860F85
:10ECE000911D860F911D8E579F4F0895860F911D80
:10ECF000860F911D8E579F4FFC0180819181089551
:10ED000008958CED9AE10E944458892B21F08CEDF6
:10ED10009AE10C9431580895E091C81AF091C91AFB
:10ED2000309709F0099480E00895EF92FF920F93D5
:10ED30001F93CF93DF937C01EA01FC0180819181D5
:10ED4000009741F08C30934071F1F70111821082ED
:10ED500083E0F2C080E024E0829FF0011124E653BA
:10ED6000F54E118210828F5F8430A8F38093C71A0A
:10ED700080910212909103129093DB1A8093DA1A19
:10ED80000E9416558093A32B60E470E08CED9AE10D
:10ED90000E941D580E94A27C8CE093E0F7019183B1
:10EDA000808381E0C9C06230D9F48091A42B909116
:10EDB000A52B892B89F38091B52B863029F480917E
:10EDC000CD2B81FD0E94817681E00E94DF7D8091C4
:10EDD000A42B9091A52B892BF9F20E94A578DCCF6A
:10EDE000633060F5611114C02097B1F2D093B23056
:10EDF000C093B13083E00E94DF7D8091A42B90917D
:10EE0000A52B892B11F00E948C760E948176C4CFAD
:10EE1000613011F6209709F4BFCFD093AE30C09384
:10EE2000AD3085E00E94DF7D8091A42B9091A52BD1
:10EE3000892B09F4B1CF0E948C76AECF6738E9F503
:10EE40001092C61A0AEC1AE18091C61A8430B8F4FE
:10EE5000F801828193818C179D0749F4808191810B
:10EE60000E94AC7DF80111821082138212820C5F25
:10EE70001F4F8091C61A8F5F8093C61AE5CFECECC6
:10EE8000F0E3838194818C179D0719F41482138217
:10EE90001082B09621E3EC34F20799F7E9E4F1E34C
:10EEA000818592858C179D0711F4158214823D96F9
:10EEB00081E3EB3CF807A1F76FCF683809F06CCF1E
:10EEC000CC5DDA4109F068CF8CED9AE10E9444589C
:10EED000892B09F461CF1092C61AE091C61AE4306A
:10EEE00008F05ACF20E2E29FF0011124ED54FF4CCC
:10EEF000818D8823D9F08CED9AE10E943158809160
:10EF0000C61AE0E28E9FC00111248D549F4C90934D
:10EF1000B2308093B13082E00E94DF7D8091A42BDB
:10EF20009091A52B892B11F00E948C768091C61AA6
:10EF30008F5F8093C61AD1CFDF91CF911F910F9130
:10EF4000FF90EF9008959093C91A8093C81A08957E
:10EF5000209102123091031260E0EAECFAE1643091
:10EF600098F4408151814817590759F442815381DF
:10EF70004217530731F46093C51A118210820C9422
:10EF8000AC7D34966F5FEBCF6093C51A089540E077
:10EF9000EAECFAE14430A8F451E0540F20813181C9
:10EFA000232B61F44093C41A918380832091021231
:10EFB00030910312338322830C94C67D3496452FFF
:10EFC000E9CF4093C41A08952091021230910312A0
:10EFD000FC01358F248F778F668F08952091021260
:10EFE00030910312FC01328721877487638708956B
:10EFF000CF93DF93EA010E944F7D009749F0209163
:10F00000021230910312FC0132872187D487C38713
:10F01000DF91CF9108950F931F93CF93DF9300D08B
:10F0200000D0CDB7DEB78C01AB018FEF89838A8327
:10F030008B838C83B801CE0101960E94F8770097EC
:10F0400019F0FC01158304830F900F900F900F901F
:10F05000DF91CF911F910F91089540E050E062E061
:10F060008CED92E00E94BC551092A52B1092A42B1F
:10F070000895AC0161E08CED92E00C949E55AC01DA
:10F0800060E08CED92E00C949E550F931F93CF930C
:10F09000DF938A010E94CE7CEC01009759F08091A9
:10F0A0000212909103129D8F8C8F1F8F0E8FCE01B5
:10F0B0000E943F78CE01DF91CF911F910F9108956B
:10F0C000CF93DF93A091B130B091B230109719F087
:10F0D000ED016C9605C0C091AD30D091AE3029964F
:10F0E0008091AC3086FF22C01092C31A40E0EAEC57
:10F0F000FAE14430B8F42081318114968D919C91CD
:10F1000015972817390759F482819381009739F0B0
:10F110004093C31A998388831B821A8205C0349650
:10F120004F5FE7CF4093C31A0E948176888199810F
:10F13000009741F04A815B816091A32BDF91CF91D1
:10F140000C94BC55DF91CF9108950F931F93CF93EB
:10F15000DF938091B52B863009F071C08091A42B8C
:10F160009091A52B8115954009F069C0C4E9D2E0C2
:10F17000D093A52BC093A42B02E00093AE2B14E9EF
:10F180001093AF2B1092D12B1092D02B0E949C7C0D
:10F19000809590959093D12B8093D02B1092B72B84
:10F1A0001092B62B0E948B7C809590959093B72BF4
:10F1B0008093B62B0E948C76D093A52BC093A42B62
:10F1C0000093AE2B1093AF2BA091AF30B091B03025
:10F1D000FD01E459FD4F8CE692E001900D920197FC
:10F1E000E1F76CE672E084EC9BE20E944A7C80913D
:10F1F000A82B8093C42B8091A92B8093C52B809141
:10F20000AA2B8093C62B8091AB2B8093C72B109297
:10F21000D12B1092D02B0E949C7C8095909590933E
:10F22000D12B8093D02B1092B72B1092B62B0E942B
:10F230008B7C809590959093B72B8093B62BDF9124
:10F24000CF911F910F910C948C76FC01680F791F60
:10F2500080E048E1E617F70781F0219198E0322F2E
:10F260003827532F517030FD84278695513009F48B
:10F2700080682695915099F7EDCF08951F920F92CF
:10F280000FB60F9211240BB60F922F933F934F930B
:10F290005F936F937F938F939F93AF93BF93EF93FE
:10F2A000FF9380919400909195009093902B809380
:10F2B0008F2B81E08093812B80917100807D8093E2
:10F2C00071000E9485758091812B8823D9F18091EE
:10F2D00094009091950040918F2B5091902B841722
:10F2E0009507A0F48091552B9091562BA091572B08
:10F2F000B091582B8C57914EAF4FBF4F8093552BE9
:10F300009093562BA093572BB093582B2091940099
:10F3100030919500241B350B8091552B9091562BE5
:10F32000A091572BB091582B820F931FA11DB11D97
:10F330008093552B9093562BA093572BB093582B1B
:10F340001092812BFF91EF91BF91AF919F918F917F
:10F350007F916F915F914F913F912F910F900BBED5
:10F360000F900FBE0F901F9018959FB7F894E1E78C
:10F37000F0E08081807D808388B38F6288BB1092AB
:10F380009000E1E9F0E01082109292001092950056
:10F39000109294008081856080839FBF08952FB76D
:10F3A000F894909399008093980088B38F6288BBFB
:10F3B000E1E7F0E08081826080832FBF0895CF93E2
:10F3C000DF93FC01DB0185E0EB0119928A95E9F7F7
:10F3D0008581837011F082E08C938781837021F0A6
:10F3E00082E012968C9312978581837081F08781D9
:10F3F000837069F0238934898185928528173907BC
:10F4000031F481E0848312961C92129701C0148219
:10F4100085818370823021F0833021F080E003C049
:10F4200082E001C088E011968C93119787818370E8
:10F43000823021F0833021F080E003C082E001C0FF
:10F4400088E013968C93DF91CF910895CF93DF934B
:10F4500000D000D01F92CDB7DEB7BE016F5F7F4FE7
:10F460000E94DF7989819A81890F8D5F9B81890F45
:10F470009C81890F9D81890F0F900F900F900F90A5
:10F480000F90DF91CF9108954F925F926F927F928C
:10F490008F929F92AF92BF92CF92DF92EF92FF92A4
:10F4A0000F931F93CF93DF9300D000D000D0CDB740
:10F4B000DEB78C017B01BE016F5F7F4F4E830E94E0
:10F4C000DF79B981AA815B804C808B2F90E0039615
:10F4D0002A2F30E0820F931F850D911D642D70E05F
:10F4E000860F971F5D81850F911D4E8150E0481753
:10F4F00059070CF49AC0F801818180FB662460F8FA
:10F50000712C43E0660C771C4A95E1F7828180FB01
:10F51000882480F8912C54E0880C991C5A95E1F7C6
:10F52000862880818770882A838180FBAA24A0F89E
:10F53000B12C85E0AA0CBB1C8A95E1F78A2884814E
:10F5400080FBCC24C0F8D12C96E0CC0CDD1C9A9525
:10F55000E1F78C28F7018082F80145814370F4E0DF
:10F560004F9FA0011124F80186818370F0E18F9FE5
:10F57000C0011124482BF8018781F0E48F9FC0015E
:10F580001124482BF7014183F8018085F70182831C
:10F59000B23059F4F8018185F7018383F80182853F
:10F5A000F701848395E0C92E02C083E0C82EB0E045
:10F5B00080E090E0200F311FDB2EDC0C0197BA17A2
:10F5C00061F0A901480F591FFA01B384A7014D0D3D
:10F5D000511DFA01B082BF5FEFCF9D2DF2E05F12A7
:10F5E0000EC0D701AD0DB11DF80183898C9381E068
:10F5F0008D0DD701A80FB11D9E5F84898C9340E0CB
:10F6000020E030E0060F171F842F890F21503109A9
:10F61000441561F0D801A20FB31F55965C91D70134
:10F62000A80FB11D5C934F5FEFCF80E026960FB619
:10F63000F894DEBF0FBECDBFDF91CF911F910F9128
:10F64000FF90EF90DF90CF90BF90AF909F908F9002
:10F650007F906F905F904F900895BF92CF92DF920E
:10F66000EF92FF920F931F93CF93DF937C01D62EDF
:10F67000EA0182E0861708F0B1C0F701808186FBBD
:10F68000BB24B0F89181292F269526952370C92E89
:10F69000C294C694C69453E0C522382F377038837D
:10F6A00083FB332730F9398384FB332730F93A83DE
:10F6B00085FB882780F98B83BC822D83892F8295D7
:10F6C00083708E83CF8282818887222389F1338160
:10F6D000848190E0982F8827830F911D9A878987CE
:10F6E00087010B5F1F4F223071F460E073E0CE01A1
:10F6F0000B960E947753F70186818B8785818C87D3
:10F700000E5F1F4F20C02330F1F4F7013D9680E0DB
:10F7100090E03E2F2F2F4291DE01A80FB91F1B96BC
:10F720004C93019688309105B1F7032F122F0BC02F
:10F7300087010D5F1F4F60E073E0CE010B960E94C2
:10F7400077531A861986CC20B9F1B1100DC0F80193
:10F750002081818190E0982F8827820F911D9C8BBA
:10F760008B8B0E5F1F4F04C089859A859C8B8B8B7A
:10F77000F2E0CF120EC060E073E0CE0145960E9429
:10F780007753F80181818D8B80818E8B0E5F1F4FA7
:10F790001BC0F3E0CF1218C0085F1F4FF80180E0D4
:10F7A00090E02291DE01A80FB91F55962C93019687
:10F7B00088309105B1F708C060E073E0CE0145964E
:10F7C0000E9477531C8A1B8AC8018E199F092D2D10
:10F7D000281B2FA71EA70DA7D81608F480E0DF91DD
:10F7E000CF911F910F91FF90EF90DF90CF90BF903E
:10F7F0000895FB0141505109460F571FE417F507C3
:10F8000078F4208130E0322F22276181260F311DCC
:10F81000820F931F8217930708F401963296EECF5A
:10F82000E417F50751F4208130E0322F2227820FB0
:10F83000931F8217930708F401960895CF93DF93DF
:10F84000C091AF2BD0E064972091AE2B30E0322FE7
:10F850002227C20FD31F48E050E068EB7BE29E01F5
:10F86000280F311DC9010E94F97BAE0160EC7BE2DB
:10F870000E94F97B009721F098278927982702C0DA
:10F880008FEF9FEFDF91CF9108959093F51A8093BA
:10F89000F41A0895FC015381560F5093AB2B872F18
:10F8A00099274281480F4093AA2BA181A093A92BAD
:10F8B000E081E093A82B242F30E02817390748F483
:10F8C00081E08A0F8093A92B811103C0EF5FE09341
:10F8D000A82B852F90E077278617970788F44F5F2E
:10F8E0004093AA2B41110CC08091A92B8F5F80936C
:10F8F000A92B811105C08091A82B8F5F8093A82B25
:10F900000895AB01BC0180E090E00E94F97B98274C
:10F9100089279827089544E150E06CEA7BE280E073
:10F9200090E00E94F97B009721F09827892798277B
:10F9300008958FEF9FEF089586E00C941E7C81E17F
:10F940000C941E7C80E0E82FF0E0EE0FFF1FED5CD2
:10F95000FE4C118210828F5F8430A8F380E090E229
:10F96000899FF0011124ED54FF4C118E8F5F84307C
:10F97000B0F380E094E09093EF1A8093EE1A80E069
:10F980009DE0989FF0011124E75BFE4C15821482E4
:10F990008F5F8A30B0F38093ED1A0895CF93209152
:10F9A000EE1A3091EF1A2F5F3F4F21154DE73407C4
:10F9B00010F020E030E1522F432FE3EBF0E3C0E002
:10F9C000C43059F0A18DAA2329F0A481B581A417D0
:10F9D000B50749F3CF5FB096F3CF3093EF1A20937A
:10F9E000EE1A1092ED1A20E0E0E0F0E02430E8F4A6
:10F9F00030E2239FD0011124AD54BF4C59963C9165
:10FA00005997311104C02093ED1AFD0110C0373011
:10FA100041F4309739F05A964C915A97328D3417F9
:10FA200008F0DF012F5FFD01E1CF2093ED1A309741
:10FA300099F122E0218F2091F01A24872091F11A68
:10FA400025872091F21A26872091F31A278728ED1F
:10FA500034E0338B228B358B248B21E030E0318BEB
:10FA6000208B138E228F23E0208F168A20E1278B94
:10FA70002091EE1A3091EF1A32272327322735834F
:10FA8000248377836683DC014D915D916D917C9138
:10FA90004083518362837383CF01CF910895CF93C5
:10FAA000DF932091EE1A3091EF1A2F5F3F4F21150F
:10FAB0004DE7340710F020E030E1522F432FEDE402
:10FAC000F1E3C0E0CA3041F0A081B181CF5F3D9643
:10FAD000A417B507B9F7E9CF3093EF1A2093EE1AC0
:10FAE00040E05DE04A30A0F4A1E0A40F549FF00193
:10FAF0001124E75BFE4C24813581232B39F440939C
:10FB0000ED1A309741F480E090E023C04A2FEACF0D
:10FB10004093ED1AF8CF2091EE1A3091EF1A322768
:10FB2000232732273583248377836683009729F43C
:10FB3000108211821282138209C0EC01888199819E
:10FB4000AA81BB8180839183A283B38380E4808771
:10FB5000CF01DF91CF91089540E04430A0F4E42F2D
:10FB6000F0E051E0540FEE0FFF1FED5CFE4C2081E2
:10FB700031812817390729F44093ED1A1182108238
:10FB80000895452FEACF4093ED1A089540E04430A0
:10FB900098F4E42FF0E051E0540FEE0FFF1FED5CFE
:10FBA000FE4C20813181232B29F44093ED1A91835F
:10FBB00080830895452FEBCF4093ED1A0895AF92BF
:10FBC000BF92CF92DF92EF92FF920F931F93CF934A
:10FBD000DF93C091B130D091B230843009F4DCC1F0
:10FBE00024ED3BE23093B0302093AF303093A72B1D
:10FBF0002093A62B833059F4898D8F70833009F0C0
:10FC00006BC088899989892B09F0DFC67FC0823053
:10FC100009F080C08091F31A8F5F8093F31A8111ED
:10FC200013C08091F21A8F5F8093F21A81110CC079
:10FC30008091F11A8F5F8093F11A811105C0809134
:10FC4000F01A8F5F8093F01A1092A52B1092A42BBC
:10FC50001092483110924731298D822F8D7F853047
:10FC600041F48A8D8F5F8A8F843109F0AEC6198E78
:10FC7000ACC6222309F4A9C688899989892B09F47D
:10FC800041C08A8D9FEF980F9A8F81119EC68B8DF0
:10FC9000883031F09FEF920F923048F4853039F47C
:10FCA000198E80E88093AC300E94607847C585301B
:10FCB00038F493E0082E01C0990F0A94EAF701C0C6
:10FCC00090E39A8F8F5F8B8F822F8F708330A1F09C
:10FCD00048F4813009F44FC3823009F076C610929F
:10FCE000CD2B4CC3863009F4C8C4883009F4C5C490
:10FCF000843009F06AC6C1C484E08093AC300E94AD
:10FD000060784EC52F70233009F05FC688E080937D
:10FD1000AC3009C5853019F5E091AD30F091AE30C9
:10FD200084819581892B09F450C61092B2301092CB
:10FD3000B13088EC9BE29093B0308093AF309093D9
:10FD4000A72B8093A62B1092483110924731109226
:10FD5000A52B1092A42B88E08093AC301BC180911E
:10FD6000AC2B853409F031C60091AE2B10E0102F7A
:10FD700000278091AF2B080F111D8091A42B90912B
:10FD8000A52B8017910708F420C61093A52B00938C
:10FD9000A42B8091B22B8F7309F017C68091B32BDF
:10FDA000811113C68091433190914431C0915D031C
:10FDB000D0915E038C179D0759F4409145315091C5
:10FDC000463120915F033091600342175307A1F041
:10FDD0002091BC2B3091BD2B2817390709F0F5C5B0
:10FDE0002091BE2B3091BF2B8091453190914631AF
:10FDF0002817390709F0E9C50E948B7C019609F0A4
:10FE0000E4C58091B52B863009F429C18131E9F12F
:10FE1000813009F0DAC58091C02B883009F0D5C552
:10FE20001092C02B8091C22B9091C32B873F3FEF44
:10FE3000930710F0099601C008969093C32B809306
:10FE4000C22B8091B82B9091B92BA091BA2BB09175
:10FE5000BB2B8093BC2B9093BD2BA093BE2BB09358
:10FE6000BF2B8091433190914431A0914531B091A5
:10FE700046318093B82B9093B92BA093BA2BB093B3
:10FE8000BB2B80E48093B42B7DC50C5111091093DA
:10FE9000A52B0093A42B88EC9BE29093B030809329
:10FEA000AF308091C62B9091C72B892B29F00E94EF
:10FEB0009F7C019609F089C52091C22B3091C32BFC
:10FEC0002115310509F481C589E491E39093AE30A1
:10FED0008093AD30A090C02BB090C12B40915F03B8
:10FEE000509160036091610370916203A09163037C
:10FEF000B09164030091B82B1091B92BE090BA2B0C
:10FF0000F090BB2BE091AD30F091AE3081E3EB3C53
:10FF1000F80708F05AC584819581009721F12817C8
:10FF2000390709F586819781009719F0A816B90657
:10FF3000D1F4808191818C179D0729F4C280D380F0
:10FF4000C416D506B1F08617970729F4C280D3806E
:10FF5000CA16DB0671F00817190729F4828193810C
:10FF6000E816F90631F03D96F093AE30E093AD30EF
:10FF7000C9CF1092B2301092B13082E08093AC3091
:10FF800088EC9BE29093A72B8093A62B109248318C
:10FF9000109247310E9460788091473190914831AA
:10FFA000009709F412C59C01245E3F4F3093A52BA6
:10FFB0002093A42B3093AE2B2093AF2BE091AD3048
:10FFC000F091AE3020852093B42B21E12093B52B06
:10FFD00008969827892798279093C52B8093C42B40
:10FFE0001092C72B1092C62B848195819093C12BC0
:10FFF0008093C02B868197819093C32B8093C22BD3
:020000021000EC
:100000008091433190914431A0914531B091463176
:100010008093B82B9093B92BA093BA2BB093BB2BA2
:1000200080819181A281B3818093BC2B9093BD2B61
:10003000A093BE2BB093BF2B84ED9BE29093B03086
:100040008093AF300E949F7C80959095009711F42B
:100050008FEF9FEF9093C72B8093C62B93C40E9482
:100060009C7C019609F0B1C48091C22B9091C32B66
:10007000009709F4AAC42091C02B3091C12B2115FF
:10008000310509F4A2C44091B82B5091B92B60916D
:10009000BA2B7091BB2BECECF0E3C3EBD0E3F08018
:1000A000FF20A9F0AC81BD818A179B0781F4AE8146
:1000B000BF812A173B0759F4A881B9814A175B070A
:1000C00031F4AA81BB816A177B0709F46FC1A0963E
:1000D000B096A1E3C333DA0711F72091CD2B2F732C
:1000E0002230D9F49093EB1A8093EA1A40E044301E
:1000F00090F4E42FF0E0EE0FFF1FED5CFE4C20814A
:1001000031814F5F8217930791F71092ED1A20E02B
:10011000C0E0D0E07EC04093ED1A8091CD2B82FDEF
:1001200054C484E18093CD2B88E290E09093A52B7A
:100130008093A42B80E58093CC2B8091C72B90914A
:10014000CB2B9093C72B3091C62B9091CA2B9093B9
:10015000C62B3093CA2B2091C52B9091C92B90931D
:10016000C52B2093C92B9091C42B9093ED1A4091ED
:10017000C82B4093C42B9093C82B8F5F8093CB2BBD
:1001800081110FC081E0830F8093CA2B811109C0B8
:1001900081E0820F8093C92B811103C09F5F9093F0
:1001A000C82B8091C02B9091C12B9093EB1A809318
:1001B000EA1A2091C22B3091C32B3093C12B20938C
:1001C000C02B9093C32B8093C22B8091B82B90911E
:1001D000B92BA091BA2BB091BB2B8093BC2B9093E1
:1001E000BD2BA093BE2BB093BF2B80914331909138
:1001F0004431A0914531B09146318093B82B909312
:10020000B92BA093BA2BB093BB2BA1C3373089F085
:100210002F5F2430C0F430E2239FC0011124FC0181
:10022000ED54FF4C318D3111F1CF2093ED1AEF01D8
:100230000CC0209721F0428D3A8D341748F7EC011D
:10024000CD54DF4CE5CF2093ED1A209709F4BDC3C0
:10025000D093B230C093B13083E08A8F888F1E8AEA
:1002600084E08F8B1B8E8091C22B9091C32B9D833A
:100270008C838091C02B9091C12B9F838E83809122
:10028000B82B9091B92BA091BA2BB091BB2B88833E
:100290009983AA83BB8381E0898F8091F01A8C8730
:1002A0008091F11A8D878091F21A8E878091F31ACE
:1002B0008F8781E090E0998B888B8091C72B8B870B
:1002C0008091C62B8A878091C52B89878091C42B0A
:1002D000888781E090E00E9449858091CC2B282F6F
:1002E000207F30E0213531050CF445C082958F70B8
:1002F00090E00597880F991F880F991F3091EC1A8D
:1003000020E0E22FF0E0E817F9078CF5E455F44D12
:1003100030A5311105C02093ED1A1092EC1A2BC0B4
:10032000313011F42F5FEDCF3230E1F441A544308C
:10033000C9F42093ED1A3093EC1A82A590E0982F1F
:10034000882723A5822B9093EB1A8093EA1A893D84
:10035000A4E09A0710F088ED94E09B8B8A8B9D8B2C
:100360008C8B09C041A5442311F0240FCACF2093E0
:10037000ED1A3093EC1A80E18093CD2B8091CD2B38
:1003800082608093CD2B82E08093D42B84E0809395
:10039000D52B8093D62B88ED8093D72B8CE290E0E1
:1003A0009093A52B8093A42B80E67EC2D093B2308D
:1003B000C093B1301092AC309091CD2B92FF03C01E
:1003C000198E80E21AC28091CC2B82958F70880F93
:1003D000880F8093ED1A081B11090451110910931D
:1003E000A52B0093A42B8F2D8F70823029F4892F99
:1003F0008F73823139F41FC0813021F4892F8F73BC
:100400008230C9F0012B19F4892F8370A1F020915B
:10041000C42B888528133EC22091C52B89852813BB
:1004200039C22091C62B8A85281334C22091C72B4C
:100430008B8528132FC294FF4AC06889798961157A
:10044000710509F444C0CE010C960E944A7C30919B
:10045000C82B8091A82B38133AC02091C92B8091CA
:10046000A92B281334C09091CA2B8091AA2B9813E2
:100470002EC08091CB2B4091AB2B841328C03C879E
:100480002D879E878F878B8D81111AC02E89888D2D
:100490009A8D891B922F969596959695891B280F74
:1004A0002E8B87FD81959F89392F36953695931B25
:1004B000980F9F8B822F869586958695890F888FBA
:1004C00081E08093AC30888D8A8F198A188A498D93
:1004D000842F8F7090E0FC013197E830F10508F02F
:1004E00074C2E057FF4F0C948C8D8091AC3080FF2C
:1004F00014C083E0898F80E48093AC30198A188A15
:100500008091A42B9091A52B009709F408C122E4B7
:100510002093AC300E94498502C18091CD2B8F730E
:10052000823009F052C227CF8091AC3080FF70C07A
:100530008091CD2B8F73823109F06AC08091CC2BD2
:10054000282F207F30E0213531050CF445C08295FD
:100550008F7090E00597880F991F880F991F309131
:10056000EC1A20E0E22FF0E0E817F9078CF5E455EB
:10057000F44D30A5311105C02093ED1A1092EC1AFC
:100580002BC0313011F42F5FEDCF3230E1F441A5B3
:100590004430C9F42093ED1A3093EC1A82A590E010
:1005A000982F882723A5822B9093EB1A8093EA1A21
:1005B000893D24E0920710F088ED94E09B8B8A8BB4
:1005C0009D8B8C8B09C041A5442311F0240FCACF09
:1005D0002093ED1A3093EC1A83E0898F8091C42B1D
:1005E00088878091C52B89878091C62B8A878091C7
:1005F000C72B8B8781E090E00E94498582E480933D
:10060000AC30198A188A1092A52B1092A42B87C09F
:1006100080E28093AC300E946078E091B130F0913C
:10062000B230118E7ACD8091CD2B80FF28C044FD51
:1006300026C088899989892B09F0C7C18091A42B8C
:100640009091A52B01960E9449852091AC30822F74
:1006500080618093AC308091A42B9091A52B892B45
:1006600019F022612093AC300E94607881E090E024
:10067000998B888B88E0898F1B8E81E10CC185FF67
:100680001CC08091D22B90E0982F88272091D32BEB
:10069000822B2091AF303091B030280F391F30932A
:1006A000B0302093AF302091A42B3091A52B281B84
:1006B000390B3093A52B2093A42B8091A42B9091E0
:1006C000A52B009749F044FD07C02091AC30226073
:1006D0002093AC300E9449858091CE2B90E0982FDA
:1006E00088272091CF2B820F911D9093EB1A809336
:1006F000EA1A2C893D892817390710F0892B21F433
:100700003093EB1A2093EA1A8091EA1A9091EB1A2F
:100710009B8B8A8B8091AC30837009F456C1109208
:100720004831109247310E9460788091AC3085FF4B
:1007300007C01092483110924731198E84E1ABC046
:1007400084FF0AC0109248311092473181E090E056
:10075000998B888B84E08FCF20914731309148313D
:1007600021153105E1F080FF02C0198A188A8889B5
:100770009989009781F48A899B898217930720F4CD
:10078000909348318093473180914731909148311F
:10079000998B888B04C090934831809347311B8E8E
:1007A0008091A62B9091A72B9093B0308093AF307F
:1007B0008091473190914831892B59F088899989E6
:1007C000009739F088969093A52B8093A42B88E10D
:1007D0000BC08091AC3081FFF8C088E290E090932C
:1007E000A52B8093A42B80E18093CD2B5CC08091BE
:1007F000AC3080FFEAC0198E80E18093AC300E945B
:100800006078E3C08091A42B9091A52B009711F004
:100810000E9449859091CD2B8091AC3090FF0BC008
:1008200080FF06C087E0898F1A8E198A188A19C03E
:1008300086E0898F16C080FF1EC085E0898F198AE7
:10084000188AC3C08091A42B9091A52B009711F01A
:100850000E9449858091CD2B80FF0DC087E0898F54
:100860001A8E81E090E00E94498580E18093AC304F
:100870000E9460780FC08091A42B9091A52B892BAA
:1008800049F4A3C08091AC3080FF9FC087E0898F7E
:100890001A8E9BC080E18093CD2B88E290E09093EC
:1008A000A52B8093A42B80E58093CC2B8885809307
:1008B000C82B89858093C92B8A858093CA2B8B8509
:1008C0008093CB2B8C858093C42B8D858093C52BF7
:1008D0008E858093C62B8F858093C72B86E080936F
:1008E000B52B8C819D819093C12B8093C02B8E81E1
:1008F0009F819093C32B8093C22B80914331909121
:100900004431A0914531B09146318093B82B9093FA
:10091000B92BA093BA2BB093BB2B88819981AA8164
:10092000BB818093BC2B9093BD2BA093BE2BB09327
:10093000BF2B898D84FF05C01092CF2B1092CE2B38
:1009400006C084E08093CE2B88ED8093CF2B80E48B
:100950008093B42B8091A42B9091A52B9093AE2BD8
:100960008093AF2B1092D32B1092D22B1092D12BBD
:100970001092D02B0E949C7C809590959093D12BC7
:100980008093D02B85E48093AC2B1092AD2B1092EA
:10099000B32B1092B22B8091F41A9091F51A019614
:1009A0009093F51A8093F41A9093B02B8093B12B07
:1009B0001092B72B1092B62B0E948B7C809590954D
:1009C0009093B72B8093B62B04C01092A52B109256
:1009D000A42B1092AC30DF91CF911F910F91FF901B
:1009E000EF90DF90CF90BF90AF9008959827892720
:1009F000982708950E94928D0895FC018091A62B5E
:100A00009091A72B2CEA30E3281B390BAB0126175A
:100A100037070CF4A9011416150654F45093483105
:100A200040934731E817F90719F0BF010C944D9333
:100A3000089580E880936100109261000E94D36362
:100A40000E9433550E94B167809153299091542997
:100A5000009729F001979093542980935329C090CF
:100A60005529D0905629E0905729F09058290E9496
:100A70006D66C616D706E806F90611F30E946D6684
:100A8000609355297093562980935729909358293C
:100A9000D7CF2091B1303091B230BC01C901089656
:100AA0000E944A7CE091B130F091B2308091A82B45
:100AB00080878091A92B81878091AA2B8287809142
:100AC000AB2B838708952F923F924F925F926F9244
:100AD0007F928F929F92AF92BF92CF92DF92EF92CE
:100AE000FF920F931F93CF93DF93CDB7DEB763973A
:100AF0000FB6F894DEBF0FBECDBF7C011B016A01AB
:100B0000FC0117821682838181FF66C3BE016F5F7D
:100B10007F4F4B01F7019381F10193FD859193FF85
:100B200081911F01882309F453C3853239F493FD61
:100B3000859193FF81911F01853239F4B70190E0CF
:100B40000E94D09356016501E5CF10E0512C20E0C2
:100B50002032A0F48B3269F030F4803259F08332C5
:100B600069F420612CC08D3239F0803339F4216072
:100B700026C02260246023C0286021C027FD27C032
:100B800030ED380F3A3078F426FF06C0FAE01F9FA8
:100B9000300D1124132F13C06AE0569E300D11241E
:100BA000532E20620CC08E3221F426FD11C3206426
:100BB00006C08C3611F4206802C0883641F4F10179
:100BC00093FD859193FF81911F018111C1CF9BEB13
:100BD000980F933018F42061805E06C09BE9980F4F
:100BE000933008F0AAC12F7E26FF16E02F73722ED5
:100BF000853621F4F22FF0647F2E08C0863621F46A
:100C0000622F6068762E02C01111115077FE07C066
:100C10001C3348F444244394410E27E00BC01830A1
:100C200030F4212F06C027E04CE3442E03C027E018
:100C300017E0412C560174E0A70EB11CF60160814B
:100C4000718182819381042DA4010E9455926C01CF
:100C5000098100FF02C003FF06C071FC07C072FCDF
:100C600008C0612C08C03DE2632E05C02BE2622E55
:100C700002C090E2692E802F8C7099F1662011F0ED
:100C800084E001C083E0851510F0512C0BC0581A88
:100C900073FC08C0B70180E290E00E94D0935A94A0
:100CA000C9F7F3CF662029F0B701862D90E00E94A6
:100CB000D09303FD03C00DE911E102C009E911E180
:100CC000F72DF0717F2EF8018491882309F476C204
:100CD00071108052B70190E00E94D0930F5F1F4FB8
:100CE000F2CF77FE0FC04C0C04FF04C08A81813321
:100CF00009F44A94141474F5F8E0F41578F588E0D2
:100D0000482E2CC076FC2AC0812F90E08C159D05C2
:100D10009CF06CEFC6166FEFD60674F0772D7068F6
:100D2000772E0AC0E2E0F0E0EC0FFD1FE10FF11DAD
:100D30008081803319F411501111F4CF77FE0EC069
:100D400044244394410E812F90E0C816D9062CF418
:100D50001C1904C04424439401C010E077FE07C06E
:100D60001C141D043CF496012F5F3F4F05C025E085
:100D700030E002C021E030E0662011F02F5F3F4FED
:100D8000112331F0412F50E04F5F5F4F240F351F8B
:100D9000452D50E02417350714F4521A01C0512C88
:100DA000872D897049F4552039F0B70180E290E031
:100DB0000E94D0935A94F7CF662029F0B701862D70
:100DC00090E00E94D09373FC09C0552039F0B70120
:100DD00080E390E00E94D0935A94F7CF77FE5FC0F3
:100DE0009C2D8D2DD7FE02C090E080E0692E782EDC
:100DF00040E050E0C601841991099D878C879601D7
:100E000026193709280D391D812F90E0EE27FF277D
:100E1000E81BF90BFF87EE87FFEF6F167F0669F47B
:100E2000B7018EE290E02B8B3A8B488B598B0E9456
:100E3000D093598948893A892B89C614D70454F02C
:100E40006C857D85661577052CF4F901E40FF51F97
:100E5000818101C080E371E0671A71084F5F5F4FC5
:100E6000EE85FF856E167F066CF0B70190E02B8B48
:100E70003A8B488B598B0E94D0932B893A894889A9
:100E80005989CACF6C147D0439F49A81963318F4C9
:100E9000953311F404FF81E3B70190E04BC08A81E0
:100EA000813309F00F7EB70190E00E94D0931111B9
:100EB00005C074FE18C085E490E017C0B7018EE24B
:100EC00090E00E94D09382E066246394680EF4015F
:100ED000E80FF11D8081B70190E00E94D09311507E
:100EE00041F3862DF1CF85E690E0B7010E94D093C3
:100EF000D7FC05C0C114D10439F404FF05C0D19456
:100F0000C194D1088DE201C08BE2B70190E00E944C
:100F1000D09380E36AE0C616D1042CF08F5FFAE02C
:100F2000CF1AD108F7CFB70190E00E94D093B70154
:100F3000C601C0960E94D09341C1833631F08337F9
:100F400079F0833509F058C021C0560172E0A70E30
:100F5000B11CF6018081898301E010E0640114C0B6
:100F60005601F2E0AF0EB11CF601C080D18026FF21
:100F700003C0612F70E002C06FEF7FEFC6012B8BC3
:100F80000E947C938C012B892F7715C05601F2E0CB
:100F9000AF0EB11CF601C080D18026FF03C0612FC7
:100FA00070E002C06FEF7FEFC6012B8B0E943E9373
:100FB0008C012B892068722E23FD1AC0852D90E0AC
:100FC00008171907A8F4B70180E290E00E94D093B7
:100FD0005A94F4CFF60177FC859177FE81916F01E9
:100FE000B70190E00E94D09351105A94015011091A
:100FF0000115110579F7E2C0843611F0893651F5F3
:10100000560127FF09C0F4E0AF0EB11CF601608164
:101010007181828193810AC0F2E0AF0EB11CF601AA
:1010200060817181882777FD8095982F022F0F7638
:1010300097FF08C090958095709561957F4F8F4F71
:101040009F4F00682AE030E0A4010E940A95C82E54
:10105000C8183EC0022F853721F40F7E2AE030E009
:101060001DC0097F8F3691F018F4883559F0B0C053
:10107000803719F0883711F0ABC0006104FF09C058
:10108000046007C024FF08C0066006C028E030E006
:1010900005C020E130E002C020E132E0560107FF48
:1010A00009C0F4E0AF0EB11CF6016081718182814C
:1010B000938108C0F2E0AF0EB11CF601608171812E
:1010C00080E090E0A4010E940A95C82EC8180F770E
:1010D00006FF0BC0202F2E7FC11650F404FF0AC05C
:1010E00002FD08C0202F2E7E05C0DC2C202F03C05F
:1010F000DC2C01C0D12E24FF0DC0FE01EC0DF11D32
:101100008081803311F4297E09C022FF06C0D39468
:10111000D39404C0822F867809F0D39423FD13C0A2
:1011200020FF06C01C2DD51418F4150D1D19D52C43
:10113000D51468F4B70180E290E02B8B0E94D09325
:10114000D3942B89F5CFD51410F45D1801C0512C20
:1011500024FF12C0B70180E390E02B8B0E94D09354
:101160002B8922FF17C021FF03C088E590E002C051
:1011700088E790E0B7010CC0822F867859F021FDF6
:1011800002C080E201C08BE227FD8DE2B70190E052
:101190000E94D093C11638F4B70180E390E00E941A
:1011A000D0931150F7CFCA94F401EC0DF11D80815A
:1011B000B70190E00E94D093C110F5CF552009F4FB
:1011C000C2CCB70180E290E00E94D0935A94F6CF4F
:1011D000F7018681978102C08FEF9FEF63960FB66C
:1011E000F894DEBF0FBECDBFDF91CF911F910F915D
:1011F000FF90EF90DF90CF90BF90AF909F908F9037
:101200007F906F905F904F903F902F90089550582F
:10121000BB27AA270ED04EC23FD230F044D220F0D6
:1012200031F49F3F11F41EF4FFC10EF4E095E7FB8B
:10123000F5C1E92F50D280F3BA176207730784070C
:10124000950718F071F49EF568C20EF4E0950B2E28
:10125000BA2FA02D0B01B90190010C01CA01A00108
:101260001124FF27591B99F0593F50F4503E68F163
:101270001A16F040A22F232F342F4427585FF3CFA4
:10128000469537952795A795F0405395C9F77EF475
:101290001F16BA0B620B730B840BBAF09150A1F0BE
:1012A000FF0FBB1F661F771F881FC2F70EC0BA0F44
:1012B000621F731F841F48F4879577956795B795CC
:1012C000F7959E3F08F0B3CF9395880F08F09927C4
:1012D000EE0F979587950895DFD158F080E891E05B
:1012E00009F49EEFE0D128F040E851E059F45EEFB8
:1012F00009C09AC112C2E92FE078EDD168F3092E36
:10130000052AC1F3261737074807590738F00E2E6C
:1013100007F8E02569F0E025E0640AC0EF6307F80C
:10132000009407FADB01B9019D01DC01CA01AD019E
:10133000EF9347D0BFD10AD05F91552331F02BED09
:101340003FE049E450FD49EC63CF0895DF93DD278A
:10135000B92FBF7740E85FE31616170648075B070B
:1013600010F4D92FE5D19F938F937F936F934AD336
:10137000E0E3F1E06CD19ED12F913F914F915F91CD
:101380009ED2DD2349F09058A2EA2AED3FE049ECD5
:101390005FE3D0785D274DDFDF918CC11BD108F46E
:1013A00081E008950CD086C17ED140F075D130F037
:1013B00021F45F3F19F032C15111B0C135C18BD159
:1013C00098F39923C9F35523B1F3951B550BBB270C
:1013D000AA2762177307840738F09F5F5F4F220FB9
:1013E000331F441FAA1FA9F333D00E2E3AF0E0E8B2
:1013F00030D091505040E695001CCAF729D0FE2FFE
:1014000027D0660F771F881FBB1F2617370748078F
:10141000AB07B0E809F0BB0B802DBF01FF27935845
:101420005F4F2AF09E3F510568F0F8C077C15F3FDB
:10143000ECF3983EDCF3869577956795B795F7952D
:101440009F5FC9F7880F911D9695879597F9089525
:10145000E1E0660F771F881FBB1F621773078407C1
:10146000BA0720F0621B730B840BBA0BEE1F88F7D0
:10147000E095089519F40EF0D1C04FC1D5C033D115
:10148000C8F39638C0F707F80F92E8942BE33AEACE
:1014900048EB5FE716D20F920F920F924DB75EB7EF
:1014A0000F92CED1EDE5F1E0D2D04F915F91EF9167
:1014B000FF91E595EE1FFF1F49F0FE57E0684427B6
:1014C000EE0F441FFA95E1F74195550B3AD10F9075
:1014D00007FE2EC1089597FB0EF4A9D03EC0E894F4
:1014E00009C097FB3EF490958095709561957F4F6C
:1014F0008F4F9F4F9923A9F0F92F96E9BB2793951A
:10150000F695879577956795B795F111F8CFFAF429
:10151000BB0F11F460FF1BC06F5F7F4F8F4F9F4F5A
:1015200016C0882311F096E911C0772321F09EE8B8
:10153000872F762F05C0662371F096E8862F70E01E
:1015400060E02AF09A95660F771F881FDAF7880FF8
:101550009695879597F90895E894F92F96EBFF23D0
:1015600081F0121613061406440B9395F695879591
:101570007795679557954040FF23B9F71BC099278A
:101580000895882351F49850D2F7872B762F652F32
:10159000542F432F322F20E0B1F3121613061406F6
:1015A000440B88233AF09A95440F551F661F771F06
:1015B000881FCAF755234AF4440F551F11F460FFE2
:1015C00004C06F5F7F4F8F4F9F4F880F9695879511
:1015D00097F90895990F0008550FAA0BE0E8FEEF60
:1015E00016161706E807F907C0F012161306E407E7
:1015F000F50798F0621B730B840B950B39F40A26E0
:1016000061F0232B242B252B21F408950A2609F4BD
:10161000A140A6958FEF811D811D089597F99F67C1
:1016200080E870E060E008959FEF80EC0895909569
:1016300080957095609550954095309521953F4FD8
:101640004F4F5F4F6F4F7F4F8F4F9F4F0895DF93E7
:10165000CF931F930F93FF92EF92DF927B018C0148
:10166000689405C0DA2EEF012AD1FE01E894A59115
:101670002591359145915591AEF3EF01DADDFE01EB
:101680009701A801DA9479F7DF90EF90FF900F911E
:101690001F91CF91DF91089500240A941616170622
:1016A00018060906089500240A9412161306140653
:1016B00005060895092E0394000C11F4882352F0B6
:1016C000BB0F40F4BF2B11F460FF04C06F5F7F4F6E
:1016D0008F4F9F4F089557FD9058440F551F59F055
:1016E0005F3F71F04795880F97FB991F61F09F3F0F
:1016F00079F087950895121613061406551FF2CF38
:101700004695F1DF08C0161617061806991FF1CF87
:1017100086957105610508940895E894BB276627AE
:101720007727CB0197F9089555DF08F48FEF0895D7
:101730009B01AC0160E070E080E89FE333CE6ECFA8
:1017400064C1D1DFE8F39923D9F3940F511DBBF3A2
:101750009150504094F059F0882332F0660F771F73
:10176000881F91505040C1F79E3F510544F7880FA4
:10177000911D9695879597F908955F3FACF0983E37
:101780009CF0BB27869577956795B79508F4B1606F
:101790009395C1F7BB0F58F711F460FFE8CF6F5F67
:1017A0007F4F8F4F9F4FE3CFB9CF0AD029ED3BE555
:1017B0004EED5EE378C00EF028C136CF68942ECF90
:1017C00092DFC8F39923D1F3C6F3DF93CF931F932E
:1017D0000F93FF92C92FDD2788232AF02197660FE8
:1017E000771F881FDAF720E030E040E85FEB9FE3E7
:1017F000883920F0803E30F021968F7709DDE5E8CA
:10180000F1E003C005DDE2EBF1E021DF8B01BE0179
:10181000EC01FB2E6F5771097595771F880B990B9B
:1018200060DE28E132E741E35FE349D0AF2D980164
:10183000AE01FF900F911F91CF91DF91FADC3ACF6B
:10184000FA01DC01AA0FBB1F9B01AC01BF5728F4B2
:1018500022273327442750781FC0B75188F4AB2F75
:101860000024469537952795011CA395D2F30020B7
:1018700069F0220F331F441FB395DAF30DD0C7CCA4
:1018800061307105A0E88A07B94630F49B01AC01CC
:101890006627772788279078309621F02083318338
:1018A0004283538308950BD005CFF6DE28F0FBDE8C
:1018B00018F0952309F0B2CEB7CE11242FCF0BDF4D
:1018C000A0F3959FD1F3950F50E0551F629FF00153
:1018D000729FBB27F00DB11D639FAA27F00DB11DAC
:1018E000AA1F649F6627B00DA11D661F829F222735
:1018F000B00DA11D621F739FB00DA11D621F839FBC
:10190000A00D611D221F749F3327A00D611D231F91
:10191000849F600D211D822F762F6A2F11249F57DF
:1019200050408AF0E1F088234AF0EE0FFF1FBB1F02
:10193000661F771F881F91505040A9F79E3F5105A1
:1019400070F06CCEEBCE5F3FECF3983EDCF3869507
:1019500077956795B795F795E7959F5FC1F7FE2B4C
:10196000880F911D9695879597F90895FA01EE0FC6
:10197000FF1F30962105310599F16115710561F45C
:101980008038BFE39B0749F168949038810561F086
:101990008038BFEF9B0741F0992342F5FF3FE105F7
:1019A0003105210511F1E8940894E795D901AA239E
:1019B00029F4AB2FBE2FF85FD0F310C0FF5F70F497
:1019C000A695E0F7F73950F019F0FF3A38F49F7711
:1019D0009F930CD00F9007FC905808953EF024CEB2
:1019E00060E070E080E89FE308954FE79F775F93A2
:1019F0004F933F932F93E4DE2F913F914F915F914F
:101A000052DF3DCD9B01AC014ECF9F3F31F0915055
:101A100020F4879577956795B795880F911D9695D2
:101A2000879597F90895DB018F939F930E94B78D57
:101A3000BF91AF91A29F800D911DA39F900DB29F6A
:101A4000900D11240895AA1BBB1B51E107C0AA1FCA
:101A5000BB1FA617B70710F0A61BB70B881F991F4F
:101A60005A95A9F780959095BC01CD01089597FBF3
:101A7000072E16F4009407D077FD09D00E94238D1D
:101A800007FC05D03EF4909581959F4F0895709581
:101A900061957F4F0895A1E21A2EAA1BBB1BFD0181
:101AA0000DC0AA1FBB1FEE1FFF1FA217B307E4073D
:101AB000F50720F0A21BB30BE40BF50B661F771F95
:101AC000881F991F1A9469F7609570958095909575
:101AD0009B01AC01BD01CF010895052E97FB1EF4BB
:101AE00000940E94848D57FD07D00E944B8D07FC07
:101AF00003D04EF40C94848D5095409530952195EB
:101B00003F4F4F4F5F4F0895909580957095619529
:101B10007F4F8F4F9F4F0895EE0FFF1F0590F49159
:101B2000E02D099469279627692778278727782742
:101B300008950E94A18D332312F48A1B9B0B0C94F1
:101B4000B28DA29FB001B39FC001A39F700D811DF4
:101B50001124911DB29F700D811D1124911D0895B6
:101B60000E94A18DB7FF0895821B930B08950E94D8
:101B7000A18DA59F900DB49F900DA49F800D911DE8
:101B800011240895B7FF0C94B78D0E94B78D821B66
:101B9000930B0895DF93CF931F930F939A9DF02D8E
:101BA000219FF00D8B9DF00D8A9DE02DF10D039F7F
:101BB000F00D029FE00DF11D4E9DE00DF11D5E9DAB
:101BC000F00D4F9DF00D7F936F93BF92AF925F9397
:101BD0004F93D5010E94A18D8B01AC01D7010E94CA
:101BE000A18DEB01E80FF91FD6010E941A8E2F91EB
:101BF0003F91D6010E94A18DC60FD71FE81FF91F84
:101C0000AF91BF910E941A8E2F913F910E94A18D9A
